:020000040800F2
:10000000204E0020C12C0008494500085545000835
:100010005D450008654500086D45000800000000CA
:10002000000000000000000000000000754500080E
:1000300081450008000000008D4500089945000832
:10004000412D0008412D0008412D0008412D0008D8
:10005000412D0008412D0008412D0008412D0008C8
:10006000412D0008412D0008412D0008412D0008B8
:10007000412D0008412D0008412D0008412D0008A8
:10008000412D0008412D0008412D0008412D000898
:10009000412D0008412D0008412D0008412D000888
:1000A000412D0008412D0008412D0008412D000878
:1000B000412D0008412D0008412D0008412D000868
:1000C000412D0008412D0008412D0008412D000858
:1000D000A5450008412D0008412D0008412D0008CC
:1000E000412D0008412D0008412D0008412D000838
:1000F000412D0008412D0008412D0008412D000828
:10010000412D0008412D0008412D0008412D000817
:10011000412D0008412D0008412D0008412D000807
:10012000412D0008412D0008412D0008412D0008F7
:10013000412D0008412D0008412D0008412D0008E7
:10014000412D0008412D0008412D0008412D0008D7
:10015000412D0008412D0008412D0008412D0008C7
:10016000412D0008412D0008412D0008412D0008B7
:10017000412D0008412D0008412D0008412D0008A7
:10018000412D0008412D000890B484B000AF024614
:100190000B46FA71BB714FF00003FB60BB7903F0B3
:1001A00003034FEA83034FF00F0202FA03F3FB60ED
:1001B0004FF46053C4F20103BA794FEA9202D2B20B
:1001C00010464FF46052C4F20102B9794FEA91012E
:1001D000C9B201F1020152F82110FA686FEA020275
:1001E000114000F1020243F822104FF46053C4F2B0
:1001F0000103BA794FEA9202D2B210464FF460522C
:10020000C4F20102B9794FEA9101C9B201F10201C8
:1002100052F82110FC79BA7902F003024FEA820207
:1002200004FA02F2114300F1020243F8221007F12E
:100230001007BD4690BC704780B582B000AF4FF04C
:100240003A004FF0010104F013F84CF233733B60B5
:100250004FF002033B714FF002037B714FF000033C
:10026000BB714FF00003FB713B464FF44060C4F29A
:100270000200194604F0DEFB4FF44060C4F20200B5
:100280004FF000014FF00C0204F0B0FC4FF440605E
:10029000C4F202004FF001014FF00C0204F0A6FC82
:1002A0004FF44060C4F202004FF004014FF00C0222
:1002B00004F09CFC4FF44060C4F202004FF00501D2
:1002C0004FF00C0204F092FC4FF44060C4F20200C4
:1002D0004FF008014FF00C0204F088FC4FF440602E
:1002E000C4F202004FF009014FF00C0204F07EFC52
:1002F0004FF44060C4F202004FF00A014FF00C02CC
:1003000004F074FC4FF44060C4F202004FF00E01A0
:100310004FF00C0204F06AFC4FF44060C4F202009B
:100320004FF00F014FF00C0204F060FC4FF68073A9
:100330003B603B464FF48050C4F20200194604F083
:1003400079FB4FF48050C4F202004FF007014FF0E8
:100350000C0204F04BFC4FF48050C4F202004FF04A
:1003600008014FF00C0204F041FC4FF48050C4F23D
:1003700002004FF009014FF00C0204F037FC4FF47B
:100380008050C4F202004FF00A014FF00C0204F05A
:100390002DFC4FF48050C4F202004FF00B014FF0DF
:1003A0000C0204F023FC4FF48050C4F202004FF022
:1003B0000C014FF00C0204F019FC4FF48050C4F211
:1003C00002004FF00D014FF00C0204F00FFC4FF44F
:1003D0008050C4F202004FF00E014FF00C0204F006
:1003E00005FC4FF48050C4F202004FF00F014FF0B3
:1003F0000C0204F0FBFB4FF008033B603B464FF45C
:100400008050C4F20200194604F014FB4FF48050EF
:10041000C4F202004FF003014FF00C0204F0E6FBBF
:100420004FF080033B603B464FF44060C4F2020053
:10043000194604F0FFFA4FF44060C4F202004FF096
:100440000A014FF00C0204F0D1FB4FF008033B60AF
:100450004FF001033B714FF000037B714FF000033D
:10046000BB714FF00003FB713B464FF44060C4F298
:100470000200194604F0DEFA4FF400533B604FF0DF
:1004800001033B714FF001037B714FF00003BB711F
:100490004FF00003FB713B464FF44060C4F2020092
:1004A000194604F0C7FA4FF44060C4F202004FF45A
:1004B000005104F07FFB07F10807BD4680BD00BF77
:1004C00080B596B000AF4FF001004FF0010103F08E
:1004D000F9FE4FF001033B604FF000037B604FF0EB
:1004E0000903BB604FF00003FB604FF000033B616A
:1004F0004FF000037B614FF00003BB614FF000033E
:10050000FB614FF000033B624FF000037B624FF052
:100510001003BB624FF00003FB624FF000033B632C
:100520004FF000037B634FF00003BB634FF0000309
:10053000FB634FF480533B644FF000037B644FF048
:100540000003BB644FF00003FB643B463B653B4646
:100550007B6507F11C03184604F09AF94FF0000080
:100560004FF0010104F03CFA07F15807BD4680BD89
:1005700080B582B000AFFFF75FFEFFF7A1FF4FF03D
:10058000050000F0F3FD4FF44060C4F202004FF0AC
:10059000080104F01DFB4FF00A0000F0E7FD4FF4E6
:1005A0004060C4F202004FF0080104F003FB4FF07A
:1005B00010004FF0010100F01BF94FF01E004FF04A
:1005C000B20100F015F94FF028004FF0060100F0DD
:1005D0000FF94FF000004FF0010100F009F94FF062
:1005E000010047F2EF0100F003F94FF002004FF471
:1005F000C06100F0FDF84FF010004FF0000100F076
:10060000F7F84FF0050000F0B1FD4FF0110046F68D
:10061000200100F0EDF84FF0120040F6991100F0C3
:10062000E7F84FF026004FF4605100F0E1F84FF08A
:1006300007004FF0330100F0DBF84FF00C004FF0F3
:10064000050100F0D5F84FF030004FF0000100F048
:10065000CFF84FF0310040F2033100F0C9F84FF00D
:10066000320040F2074100F0C3F84FF0330040F28F
:10067000013100F0BDF84FF0340040F2013100F0DC
:10068000B7F84FF0350040F2034100F0B1F84FF0F9
:10069000360040F2077100F0ABF84FF037004FF42E
:1006A000806100F0A5F84FF03A004FF4206100F0AF
:1006B0009FF84FF03B004FF4805100F099F84FF055
:1006C0000D004FF00A0100F093F84FF00E004FF4C8
:1006D000385100F08DF84FF044004FF46F4100F0B6
:1006E00087F84FF045004FF0000100F081F84FF01F
:1006F000460040F23F1100F07BF84FF04E004FF003
:10070000000100F075F84FF04F004FF0000100F0CD
:100710006FF84FF022004FF0000100F069F84FF041
:1007200000037B6007E04FF0000000F083F87B6877
:1007300003F101037B607A6842F6FF33C0F20103E4
:100740009A42F0D940F21800C2F2000000F082F89C
:1007500007F10807BD4680BD80B582B000AF0246F4
:100760000B46FA807B71FB884FF04E00194600F073
:100770003FF87B799BB24FF04F00194600F038F8F4
:1007800007F10807BD4680BD80B582B000AFF88094
:1007900079717A803B71FA887B88D31A9BB203F116
:1007A00001039BB24FF04500194600F021F8FB8889
:1007B0004FF04600194600F01BF87B799AB23B795E
:1007C0009BB2D31A9BB203F101039BB29AB27B791D
:1007D0004FEA03239BB213439BB29BB24FF04400FA
:1007E000194600F005F807F10807BD4680BD00BFB7
:1007F00080B483B000AF02460B46FA71BB804FF065
:10080000C043FA7992B21A804FF00003C6F2100387
:10081000BA881A8007F10C07BD4680BC704700BF3C
:1008200080B400AF4FF0C0434FF022021A80BD46A3
:1008300080BC704780B483B000AF0346FB804FF0AC
:100840000003C6F21003FA881A8007F10C07BD46B0
:1008500080BC704780B483B000AF786040F6B4339A
:10086000C2F200037A681A6007F10C07BD4680BC2B
:10087000704700BF80B400AF40F6B433C2F200034B
:100880001B681846BD4680BC704700BF80B584B069
:1008900000AF0346FB804FF00003FB604FF01100F8
:1008A00046F62001FFF7A4FF40F23F104FF0000191
:1008B000FFF752FFFFF7B4FF4FF00003FB6009E0C2
:1008C0004FF00003C6F21003FA881A80FB6803F1A8
:1008D0000103FB60FA6842F6FF33C0F201039A425B
:1008E000EED907F11007BD4680BD00BF80B584B0CA
:1008F00000AFF88079717A803B717A793B79D318AF
:10090000DBB203F1FF33D9B2F8887A883B79FFF77D
:100910003BFF4FF0110046F62001FFF769FFFA8810
:100920007B7910461946FFF717FFFFF779FF4FF065
:100930000003FB6007E03B8B1846FFF77BFFFB687B
:1009400003F10103FB607B883A7902FB03F31A464B
:10095000FB689A42EFD840F23F104FF000014FF48D
:10096000A0724FF0F003FFF70FFF07F11007BD462D
:1009700080BD00BF80B584B000AFF88079717A8007
:100980003B714FF00003FB813B79002B06D14FF008
:1009900011004FF4D041FFF72BFF08E03B79012B0A
:1009A00005D14FF0110046F62801FFF721FFFA8824
:1009B0007B7910461946FFF7CFFEFFF731FF4FF066
:1009C0000003FB810BE040F6BA33C2F200031B8840
:1009D0001846FFF72FFFFB8903F10103FB81FA891A
:1009E0007B889A42EFD34FF0110046F62001FFF7C3
:1009F000FFFE07F11007BD4680BD00BF80B588B07F
:100A000000AFF88079717A803B717A88FB88D31ABD
:100A10009BB2FB833B799AB27B799BB2D31A9BB290
:100A2000BB83FA887B7910461946FFF795FEFFF7DE
:100A3000F7FE40F6BA33C2F200031B881846FFF7F0
:100A4000F9FEB7F91E3083EAE372A2EBE372B7F95D
:100A50001C30002BB8BF5B429A4261DBB7F91E30F5
:100A6000002B5DD0B7F91C3006EE903AB8EEE67A6E
:100A7000B7F91E3006EE903AF8EEE67AC7EE277A1E
:100A8000C7ED067A7B7907EE903AB8EEE77AFB88F5
:100A900007EE903AF8EEE76AD7ED067A66EEA77AA7
:100AA00077EE677AC7ED057AB7F91E30002B02DAC8
:100AB0004FF6FF7301E04FF00103FB832BE0FA8B4D
:100AC000FB88D318FB80FB8806EE903AB8EEE67AF6
:100AD000D7ED067A27EE277AD7ED057A77EE277AD3
:100AE00017EE900A06F044FF02460B4610461946E0
:100AF00005F010F80346DBB2FA8810461946FFF7F6
:100B00002BFEFFF78DFE40F6BA33C2F200031B88BE
:100B10001846FFF78FFEFA887B889A42CFD15DE0B6
:100B2000B7F91E3007EE903AB8EEE77AB7F91C3005
:100B300006EE903AF8EEE67AC7EE277AC7ED047A29
:100B4000FB8807EE903AB8EEE77A7B7907EE903AA9
:100B5000F8EEE76AD7ED047A66EEA77A77EE677A61
:100B6000C7ED037AB7F91C30002B02DA4FF6FF739A
:100B700001E04FF00103BB832CE0BB8BDAB27B7941
:100B8000D3187B717B7906EE903AB8EEE67AD7ED12
:100B9000047A27EE277AD7ED037A77EE277A17EED5
:100BA000900A06F0E5FE02460B461046194604F090
:100BB000B1FF03469AB27B7910461946FFF7CCFD88
:100BC000FFF72EFE40F6BA33C2F200031B88184628
:100BD000FFF730FE7A793B799A42CED107F12007B0
:100BE000BD4680BD80B400AF40F20203C2F20003F4
:100BF0001B881846BD4680BC704700BF80B400AF5C
:100C000040F6B833C2F200031B889BB21846BD46BB
:100C100080BC704780B483B000AF0346FB8040F2D5
:100C20000203C2F20003FA881A8007F10C07BD46DE
:100C300080BC704780B483B000AF0346FB8040F6B1
:100C4000BA33C2F20003FA881A8007F10C07BD46D6
:100C500080BC704780B483B000AF0346FB8040F691
:100C6000B833C2F20003FA881A8007F10C07BD46B8
:100C700080BC704790B585B002AFF88079717A80FA
:100C80003B71FB88C3F59F7303F1010398B2797937
:100C90007A883B793C8B0094FFF728FE07F10C071C
:100CA000BD4690BD80B582B000AFF88079717A8082
:100CB0003B71FB88C3F59F7303F1010398B2797907
:100CC0007A883B79FFF756FE07F10807BD4680BDDD
:100CD00080B582B000AFF88079717A803B71FB8873
:100CE000C3F59F7303F1010398B27B88C3F59F732B
:100CF00003F101039AB279793B79FFF77FFE07F19F
:100D00000807BD4680BD00BF80B582B000AFF88047
:100D100079717A803B71FB88C3F59F7303F10103FE
:100D200099B27A797B88084611461A464FF000033B
:100D3000FFF720FEFB88C3F59F7303F1010399B20F
:100D40003A797B79D318DBB203F1FF33DAB27B88CF
:100D5000084611461A464FF00003FFF70BFEFB88CA
:100D6000C3F59F7303F1010399B23B799BB27A7982
:100D7000084611461A464FF00103FFF7FBFDFB88BA
:100D8000C3F100039AB27B88D31A9BB203F5A07318
:100D900099B23B799BB27A79084611461A464FF0D0
:100DA0000103FFF7E7FD07F10807BD4680BD00BF5F
:100DB00080B588B000AFF88079713A71FB70FFF7A9
:100DC00059FD0346DB887B75FFF754FD03469B887E
:100DD0003B75FFF74FFD03461A683B79A3F12003EB
:100DE0004FEA4303797D01FB03F3D318BB613B7DDD
:100DF000082B02D94FF4004301E04FF080037B82BF
:100E0000FFF7F0FE03463B82FFF7F8FE0346FB8147
:100E1000FB88FB837B79BB834FF00003FB757AE093
:100E20004FF00003BB7543E0FB8BC3F59F7303F1E9
:100E300001039AB2BB8BDBB210461946FFF78CFC5C
:100E4000FFF7EEFCBB691B881A46798ABB7D41FA25
:100E500003F31340002B04D0FB891846FFF7EAFC8C
:100E600003E03B8A1846FFF7E5FCFB78002B04D132
:100E7000BB8B03F1FF33BB8316E0FB78012B04D15E
:100E8000FB8B03F10103FB830EE0FB78022B04D103
:100E9000BB8B03F10103BB8306E0FB78032B03D17B
:100EA000FB8B03F1FF33FB83BB7D03F10103BB75B8
:100EB000BA7D3B7D9A42B7D3FB78002B06D1FB8BE2
:100EC00003F10103FB837B79BB831CE0FB78012BDF
:100ED00006D1FB88FB83BB8B03F10103BB8312E0CC
:100EE000FB78022B06D1FB8B03F1FF33FB837B796D
:100EF000BB8308E0FB78032B05D1FB88FB83BB8B0E
:100F000003F1FF33BB83BB6903F10203BB61FB7DCC
:100F100003F10103FB75FA7D7B7D9A4280D307F1D3
:100F20002007BD4680BD00BF80B586B000AF3A60E7
:100F30000246FA800A467A713B71386807F092FAE5
:100F40000346FB81FFF796FC03469B88BB8197F81D
:100F50002030002B31D13B79002B13D1FB887B82D1
:100F60007B799AB2BB89F98901FB03F34FEAD3710C
:100F7000CB184FEA63039BB2D3189BB203F1FF3344
:100F80003B82B4E03B79012B04D1FB887B827B79E7
:100F90003B82ACE03B79022B40F0A980FB887B824E
:100FA0007B799AB2BB89F98901FB03F39BB2D31811
:100FB0009BB203F1FF333B8299E097F82030012B7D
:100FC0002ED13B79002B12D1BB89FA8902FB03F3A6
:100FD0004FEAD372D3184FEA63039BB2FA88D31A4D
:100FE0009BB203F101037B827B793B827FE03B79FB
:100FF000012B04D1FB887B827B793B8277E03B79B4
:10100000022B74D1BB89FA8902FB03F39BB2FA88E5
:10101000D31A9BB203F101037B827B793B8266E0AA
:1010200097F82030022B30D13B79002B13D1FB886D
:101030007B827B799AB2BB89F98901FB03F34FEA82
:10104000D371CB184FEA63039BB2D31A9BB203F15F
:1010500001033B824BE03B79012B04D1FB887B826F
:101060007B793B8243E03B79022B40D1FB887B823A
:101070007B799AB2BB89F98901FB03F39BB2D31A3E
:101080009BB203F101033B8231E097F82030032B40
:101090002DD13B79002B12D1BB89FA8902FB03F3D6
:1010A0004FEAD372D3184FEA63039AB2FB88D3187E
:1010B0009BB203F1FF337B827B793B8217E03B7964
:1010C000012B04D1FB887B827B793B820FE03B794B
:1010D000022B0CD1BB89FA8902FB03F39AB2FB887D
:1010E000D3189BB203F1FF337B827B793B824FF0B5
:1010F00000037B6131E03B8AD9B23A687B69D3183F
:101100001A78788A97F82030FFF752FE97F8203047
:10111000002B04D13A8ABB89D31A3B8219E097F895
:101120002030012B04D17A8ABB89D3187B8210E04E
:1011300097F82030022B04D13A8ABB89D3183B821E
:1011400007E097F82030032B03D17A8ABB89D31AA2
:101150007B827B6903F101037B61FA897B699A4297
:10116000C9D807F11807BD4680BD00BF80B485B05F
:1011700000AF78604FF00003FB607B6842F21072B2
:1011800002FB03F3FB6003E0FB6803F1FF33FB604A
:10119000FB68002BF8D107F11407BD4680BC7047EF
:1011A00080B49DB000AFF8607A600A467A813B81D6
:1011B0007B897B667B6EBB657B6E4FEA93037B66A8
:1011C0004FF00003BB664FF00003FB667B6E3B668F
:1011D000BA6E7B6ED3187B657A6D7B6ED3183B65D8
:1011E0003A6D7B6ED318FB64BB6E4FEAC303FA689B
:1011F000D31893ED007A3B6D4FEAC303FA68D31816
:10120000D3ED007A77EE277AC7ED127ABB6E4FEAFC
:10121000C303FA68D31893ED007A3B6D4FEAC3031A
:10122000FA68D318D3ED007A77EE677AC7ED117AB2
:10123000BB6E4FEAC30303F10403FA68D31893EDBE
:10124000007A3B6D4FEAC30303F10403FA68D31835
:10125000D3ED007A77EE277AC7ED107ABB6E4FEAAE
:10126000C30303F10403FA68D31893ED007A3B6DCE
:101270004FEAC30303F10403FA68D318D3ED007AED
:1012800077EE677AC7ED0F7A7B6D4FEAC303FA6892
:10129000D31893ED007AFB6C4FEAC303FA68D318B6
:1012A000D3ED007A77EE277AC7ED0E7ABB6E4FEA60
:1012B000C303FA68D31897ED127AD7ED0E7A77EE5A
:1012C000277AC3ED007A97ED127AD7ED0E7A77EE92
:1012D000677AC7ED127A7B6D4FEAC30303F104030B
:1012E000FA68D31893ED007AFB6C4FEAC30303F15D
:1012F0000403FA68D318D3ED007A77EE277AC7EDA6
:101300000D7ABB6E4FEAC30303F10403FA68D318E6
:1013100097ED107AD7ED0D7A77EE277AC3ED007A44
:1013200097ED107AD7ED0D7A77EE677AC7ED107AE0
:101330007B6D4FEAC30303F10403FA68D31893EDFE
:10134000007AFB6C4FEAC30303F10403FA68D31875
:10135000D3ED007A77EE677AC7ED0E7A7B6D4FEAB0
:10136000C303FA68D31893ED007AFB6C4FEAC3030A
:10137000FA68D318D3ED007A77EE677AC7ED0D7A65
:10138000FA6EFB6ED3183B633B6B4FEAC3037A687C
:10139000D3181B68FB623B6B4FEAC30303F10403E2
:1013A0007A68D3181B68BB627B6D4FEAC303FA6887
:1013B000D31897ED127AD7ED0B7A27EE277AD7ED6F
:1013C000106AD7ED0A7A66EEA77A77EE277AC3ED30
:1013D000007A7B6D4FEAC30303F10403FA68D31864
:1013E00097ED107AD7ED0B7A27EE277AD7ED126AB0
:1013F000D7ED0A7A66EEA77A77EE677AC3ED007AC0
:1014000097ED117AD7ED0E7A77EE277AC7ED127A3B
:1014100097ED117AD7ED0E7A77EE677AC7ED117AEC
:1014200097ED0F7AD7ED0D7A77EE677AC7ED107AE0
:1014300097ED0F7AD7ED0D7A77EE277AC7ED0F7A11
:10144000FB6E4FEAC3037A68D3181B687B62FB6E9E
:101450004FEAC30303F104037A68D3181B683B62A5
:101460003B6D4FEAC303FA68D31897ED127AD7EDB4
:10147000097A27EE277AD7ED106AD7ED087A66EE5B
:10148000A77A77EE277AC3ED007A3B6D4FEAC30364
:1014900003F10403FA68D31897ED107AD7ED097AAF
:1014A00027EE277AD7ED126AD7ED087A66EEA77A8B
:1014B00077EE677AC3ED007A3A6BFB6ED318FB6167
:1014C000FB694FEAC3037A68D3181B68BB61FB69E9
:1014D0004FEAC30303F104037A68D3181B687B61E6
:1014E000FB6C4FEAC303FA68D31897ED117AD7ED76
:1014F000067A27EE277AD7ED0F6AD7ED057A66EEE2
:10150000A77A77EE277AC3ED007AFB6C4FEAC30324
:1015100003F10403FA68D31897ED0F7AD7ED067A32
:1015200027EE277AD7ED116AD7ED057A66EEA77A0E
:1015300077EE677AC3ED007A3B89FA6ED318FB66C3
:10154000BB6E03F10103BB663B6E03F1FF333B66E9
:101550003B6E002B7FF43CAE3B894FEA83033B811B
:101560007B894FEA93039BB2FB65E3E17B6EBB652E
:101570007B6E4FEA93037B664FF00003FB664FF0F0
:1015800000033B66C7E1FA6EFB6ED3183B633A6B10
:10159000FB6ED318FB61FB6E4FEAC3037A68D31866
:1015A0001B687B62FB6E4FEAC30303F104037A6896
:1015B000D3181B683B623B6B4FEAC3037A68D318AE
:1015C0001B68FB623B6B4FEAC30303F104037A68B9
:1015D000D3181B68BB62FB694FEAC3037A68D31850
:1015E0001B68BB61FB694FEAC30303F104037A681C
:1015F000D3181B687B613B89FA6ED318FB663B6E80
:10160000BB667FE1BA6E7B6ED3187B657A6D7B6EAD
:10161000D3183B653A6D7B6ED318FB64BB6E4FEA03
:10162000C303FA68D31893ED007A3B6D4FEAC30306
:10163000FA68D318D3ED007A77EE277AC7ED127ADD
:10164000BB6E4FEAC303FA68D31893ED007A3B6D83
:101650004FEAC303FA68D318D3ED007A77EE677ABE
:10166000C7ED117ABB6E4FEAC30303F10403FA68B6
:10167000D31893ED007A3B6D4FEAC30303F10403E3
:10168000FA68D318D3ED007A77EE277AC7ED107A8F
:10169000BB6E4FEAC30303F10403FA68D31893ED5A
:1016A000007A3B6D4FEAC30303F10403FA68D318D1
:1016B000D3ED007A77EE677AC7ED0F7A7B6D4FEA4C
:1016C000C303FA68D31893ED007AFB6C4FEAC303A7
:1016D000FA68D318D3ED007A77EE277AC7ED0E7A41
:1016E000BB6E4FEAC303FA68D31897ED127AD7EDB1
:1016F0000E7A77EE277AC3ED007A97ED127AD7ED5E
:101700000E7A77EE677AC7ED127A7B6D4FEAC303E4
:1017100003F10403FA68D31893ED007AFB6C4FEAE7
:10172000C30303F10403FA68D318D3ED007A77EE0C
:10173000277AC7ED0D7ABB6E4FEAC30303F10403AA
:10174000FA68D31897ED107AD7ED0D7A77EE277AED
:10175000C3ED007A97ED107AD7ED0D7A77EE677AC0
:10176000C7ED107A7B6D4FEAC30303F10403FA68F7
:10177000D31893ED007AFB6C4FEAC30303F1040323
:10178000FA68D318D3ED007A77EE677AC7ED0E7A50
:101790007B6D4FEAC303FA68D31893ED007AFB6CB4
:1017A0004FEAC303FA68D318D3ED007A77EE677A6D
:1017B000C7ED0D7A7B6D4FEAC303FA68D31897ED36
:1017C000127AD7ED0B7A27EE277AD7ED106AD7ED8C
:1017D0000A7A66EEA77A77EE277AC3ED007A7B6DF8
:1017E0004FEAC30303F10403FA68D31897ED107AA4
:1017F000D7ED0B7A27EE277AD7ED126AD7ED0A7A62
:1018000066EEA77A77EE677AC3ED007A97ED117AE4
:10181000D7ED0E7A77EE277AC7ED127A97ED117A27
:10182000D7ED0E7A77EE677AC7ED117A97ED0F7ADA
:10183000D7ED0D7A77EE677AC7ED107A97ED0F7ACC
:10184000D7ED0D7A77EE277AC7ED0F7A3B6D4FEA29
:10185000C303FA68D31897ED127AD7ED097A27EE09
:10186000277AD7ED106AD7ED087A66EEA77A77EE79
:10187000277AC3ED007A3B6D4FEAC30303F10403FB
:10188000FA68D31897ED107AD7ED097A27EE277A00
:10189000D7ED126AD7ED087A66EEA77A77EE677A07
:1018A000C3ED007AFB6C4FEAC303FA68D31897EDD7
:1018B000117AD7ED067A27EE277AD7ED0F6AD7EDA2
:1018C000057A66EEA77A77EE277AC3ED007AFB6C8D
:1018D0004FEAC30303F10403FA68D31897ED0F7AB4
:1018E000D7ED067A27EE277AD7ED116AD7ED057A7C
:1018F00066EEA77A77EE677AC3ED007ABA6EBB6DB3
:10190000D318BB667A89BB6E9A423FF67BAE3B6EBC
:1019100003F101033B667B6E03F1FF323B6E9A429B
:10192000BFF431AE3B894FEA83033B81FB6D4FEA45
:101930009303FB65FB6D042B3FF618AE7B6EBB6516
:101940007B6E4FEA93037B664FF00003BB662BE18F
:10195000BA6E7B6ED3187B657A6D7B6ED3183B6550
:101960003A6D7B6ED318FB64BB6E4FEAC303FA6813
:10197000D31893ED007A3B6D4FEAC303FA68D3188E
:10198000D3ED007A77EE277AC7ED127ABB6E4FEA75
:10199000C303FA68D31893ED007A3B6D4FEAC30393
:1019A000FA68D318D3ED007A77EE677AC7ED117A2B
:1019B000BB6E4FEAC30303F10403FA68D31893ED37
:1019C000007A3B6D4FEAC30303F10403FA68D318AE
:1019D000D3ED007A77EE277AC7ED107ABB6E4FEA27
:1019E000C30303F10403FA68D31893ED007A3B6D47
:1019F0004FEAC30303F10403FA68D318D3ED007A66
:101A000077EE677AC7ED0F7A7B6D4FEAC303FA680A
:101A1000D31893ED007AFB6C4FEAC303FA68D3182E
:101A2000D3ED007A77EE277AC7ED0E7ABB6E4FEAD8
:101A3000C303FA68D31897ED127AD7ED0E7A77EED2
:101A4000277AC3ED007A97ED127AD7ED0E7A77EE0A
:101A5000677AC7ED127A7B6D4FEAC30303F1040383
:101A6000FA68D31893ED007AFB6C4FEAC30303F1D5
:101A70000403FA68D318D3ED007A77EE277AC7ED1E
:101A80000D7ABB6E4FEAC30303F10403FA68D3185F
:101A900097ED107AD7ED0D7A77EE277AC3ED007ABD
:101AA00097ED107AD7ED0D7A77EE677AC7ED107A59
:101AB0007B6D4FEAC30303F10403FA68D31893ED77
:101AC000007AFB6C4FEAC30303F10403FA68D318EE
:101AD000D3ED007A77EE677AC7ED0E7A7B6D4FEA29
:101AE000C303FA68D31893ED007AFB6C4FEAC30383
:101AF000FA68D318D3ED007A77EE677AC7ED0D7ADE
:101B00007B6D4FEAC303FA68D318BA6C1A607B6D19
:101B10004FEAC30303F10403FA68D3183A6C1A605E
:101B200097ED117AD7ED0E7A77EE277AC7ED127A14
:101B300097ED117AD7ED0E7A77EE677AC7ED117AC5
:101B400097ED0F7AD7ED0D7A77EE677AC7ED107AB9
:101B500097ED0F7AD7ED0D7A77EE277AC7ED0F7AEA
:101B60003B6D4FEAC303FA68D318BA6C1A603B6D39
:101B70004FEAC30303F10403FA68D3183A6C1A60FE
:101B8000FB6C4FEAC303FA68D3187A6C1A60FB6CDB
:101B90004FEAC30303F10403FA68D318FA6B1A601F
:101BA000BA6EBB6DD318BB667A89BB6DD21ABB6E99
:101BB0009A42BFF4CDAE07F17407BD4680BC7047B2
:101BC00080B49DB000AFF8607A600A467A813B81AC
:101BD0007B897B667B6EBB657B6E4FEA93037B667E
:101BE0004FF00003BB664FF00003FB667B6E3B6665
:101BF000BA6E7B6ED3187B657A6D7B6ED3183B65AE
:101C00003A6D7B6ED318FB64BB6E4FEAC303FA6870
:101C1000D31893ED007A3B6D4FEAC303FA68D318EB
:101C2000D3ED007A77EE277AC7ED127ABB6E4FEAD2
:101C3000C303FA68D31893ED007A3B6D4FEAC303F0
:101C4000FA68D318D3ED007A77EE677AC7ED117A88
:101C5000BB6E4FEAC30303F10403FA68D31893ED94
:101C6000007A3B6D4FEAC30303F10403FA68D3180B
:101C7000D3ED007A77EE277AC7ED107ABB6E4FEA84
:101C8000C30303F10403FA68D31893ED007A3B6DA4
:101C90004FEAC30303F10403FA68D318D3ED007AC3
:101CA00077EE677AC7ED0F7A7B6D4FEAC303FA6868
:101CB000D31893ED007AFB6C4FEAC303FA68D3188C
:101CC000D3ED007A77EE277AC7ED0E7ABB6E4FEA36
:101CD000C303FA68D31897ED127AD7ED0E7A77EE30
:101CE000277AC3ED007A97ED127AD7ED0E7A77EE68
:101CF000677AC7ED127A7B6D4FEAC30303F10403E1
:101D0000FA68D31893ED007AFB6C4FEAC30303F132
:101D10000403FA68D318D3ED007A77EE277AC7ED7B
:101D20000D7ABB6E4FEAC30303F10403FA68D318BC
:101D300097ED107AD7ED0D7A77EE277AC3ED007A1A
:101D400097ED107AD7ED0D7A77EE677AC7ED107AB6
:101D50007B6D4FEAC30303F10403FA68D31893EDD4
:101D6000007AFB6C4FEAC30303F10403FA68D3184B
:101D7000D3ED007A77EE677AC7ED0E7A7B6D4FEA86
:101D8000C303FA68D31893ED007AFB6C4FEAC303E0
:101D9000FA68D318D3ED007A77EE677AC7ED0D7A3B
:101DA000FA6EFB6ED3183B633B6B4FEAC3037A6852
:101DB000D3181B68FB623B6B4FEAC30303F10403B8
:101DC0007A68D3181B68BB627B6D4FEAC303FA685D
:101DD000D31897ED127AD7ED0B7A27EE277AD7ED45
:101DE000106AD7ED0A7A66EEA77A77EE677AC3EDC6
:101DF000007A7B6D4FEAC30303F10403FA68D3183A
:101E000097ED107AD7ED0B7A27EE277AD7ED126A85
:101E1000D7ED0A7A66EEA77A77EE277AC3ED007AD5
:101E200097ED117AD7ED0E7A77EE677AC7ED127AD1
:101E300097ED117AD7ED0E7A77EE277AC7ED117A02
:101E400097ED0F7AD7ED0D7A77EE277AC7ED107AF6
:101E500097ED0F7AD7ED0D7A77EE677AC7ED0F7AA7
:101E6000FB6E4FEAC3037A68D3181B687B62FB6E74
:101E70004FEAC30303F104037A68D3181B683B627B
:101E80003B6D4FEAC303FA68D31897ED127AD7ED8A
:101E9000097A27EE277AD7ED106AD7ED087A66EE31
:101EA000A77A77EE677AC3ED007A3B6D4FEAC303FA
:101EB00003F10403FA68D31897ED107AD7ED097A85
:101EC00027EE277AD7ED126AD7ED087A66EEA77A61
:101ED00077EE277AC3ED007A3A6BFB6ED318FB617D
:101EE000FB694FEAC3037A68D3181B68BB61FB69BF
:101EF0004FEAC30303F104037A68D3181B687B61BC
:101F0000FB6C4FEAC303FA68D31897ED117AD7ED4B
:101F1000067A27EE277AD7ED0F6AD7ED057A66EEB7
:101F2000A77A77EE677AC3ED007AFB6C4FEAC303BA
:101F300003F10403FA68D31897ED0F7AD7ED067A08
:101F400027EE277AD7ED116AD7ED057A66EEA77AE4
:101F500077EE277AC3ED007A3B89FA6ED318FB66D9
:101F6000BB6E03F10103BB663B6E03F1FF333B66BF
:101F70003B6E002B7FF43CAE3B894FEA83033B81F1
:101F80007B894FEA93039BB2FB65E3E17B6EBB6504
:101F90007B6E4FEA93037B664FF00003FB664FF0C6
:101FA00000033B66C7E1FA6EFB6ED3183B633A6BE6
:101FB000FB6ED318FB61FB6E4FEAC3037A68D3183C
:101FC0001B687B62FB6E4FEAC30303F104037A686C
:101FD000D3181B683B623B6B4FEAC3037A68D31884
:101FE0001B68FB623B6B4FEAC30303F104037A688F
:101FF000D3181B68BB62FB694FEAC3037A68D31826
:102000001B68BB61FB694FEAC30303F104037A68F1
:10201000D3181B687B613B89FA6ED318FB663B6E55
:10202000BB667FE1BA6E7B6ED3187B657A6D7B6E83
:10203000D3183B653A6D7B6ED318FB64BB6E4FEAD9
:10204000C303FA68D31893ED007A3B6D4FEAC303DC
:10205000FA68D318D3ED007A77EE277AC7ED127AB3
:10206000BB6E4FEAC303FA68D31893ED007A3B6D59
:102070004FEAC303FA68D318D3ED007A77EE677A94
:10208000C7ED117ABB6E4FEAC30303F10403FA688C
:10209000D31893ED007A3B6D4FEAC30303F10403B9
:1020A000FA68D318D3ED007A77EE277AC7ED107A65
:1020B000BB6E4FEAC30303F10403FA68D31893ED30
:1020C000007A3B6D4FEAC30303F10403FA68D318A7
:1020D000D3ED007A77EE677AC7ED0F7A7B6D4FEA22
:1020E000C303FA68D31893ED007AFB6C4FEAC3037D
:1020F000FA68D318D3ED007A77EE277AC7ED0E7A17
:10210000BB6E4FEAC303FA68D31897ED127AD7ED86
:102110000E7A77EE277AC3ED007A97ED127AD7ED33
:102120000E7A77EE677AC7ED127A7B6D4FEAC303BA
:1021300003F10403FA68D31893ED007AFB6C4FEABD
:10214000C30303F10403FA68D318D3ED007A77EEE2
:10215000277AC7ED0D7ABB6E4FEAC30303F1040380
:10216000FA68D31897ED107AD7ED0D7A77EE277AC3
:10217000C3ED007A97ED107AD7ED0D7A77EE677A96
:10218000C7ED107A7B6D4FEAC30303F10403FA68CD
:10219000D31893ED007AFB6C4FEAC30303F10403F9
:1021A000FA68D318D3ED007A77EE677AC7ED0E7A26
:1021B0007B6D4FEAC303FA68D31893ED007AFB6C8A
:1021C0004FEAC303FA68D318D3ED007A77EE677A43
:1021D000C7ED0D7A7B6D4FEAC303FA68D31897ED0C
:1021E000127AD7ED0B7A27EE277AD7ED106AD7ED62
:1021F0000A7A66EEA77A77EE677AC3ED007A7B6D8E
:102200004FEAC30303F10403FA68D31897ED107A79
:10221000D7ED0B7A27EE277AD7ED126AD7ED0A7A37
:1022200066EEA77A77EE277AC3ED007A97ED117AFA
:10223000D7ED0E7A77EE677AC7ED127A97ED117ABD
:10224000D7ED0E7A77EE277AC7ED117A97ED0F7AF0
:10225000D7ED0D7A77EE277AC7ED107A97ED0F7AE2
:10226000D7ED0D7A77EE677AC7ED0F7A3B6D4FEABF
:10227000C303FA68D31897ED127AD7ED097A27EEDF
:10228000277AD7ED106AD7ED087A66EEA77A77EE4F
:10229000677AC3ED007A3B6D4FEAC30303F1040391
:1022A000FA68D31897ED107AD7ED097A27EE277AD6
:1022B000D7ED126AD7ED087A66EEA77A77EE277A1D
:1022C000C3ED007AFB6C4FEAC303FA68D31897EDAD
:1022D000117AD7ED067A27EE277AD7ED0F6AD7ED78
:1022E000057A66EEA77A77EE677AC3ED007AFB6C23
:1022F0004FEAC30303F10403FA68D31897ED0F7A8A
:10230000D7ED067A27EE277AD7ED116AD7ED057A51
:1023100066EEA77A77EE277AC3ED007ABA6EBB6DC8
:10232000D318BB667A89BB6E9A423FF67BAE3B6E92
:1023300003F101033B667B6E03F1FF323B6E9A4271
:10234000BFF431AE3B894FEA83033B81FB6D4FEA1B
:102350009303FB65FB6D042B3FF618AE7B6EBB65EC
:102360007B6E4FEA93037B664FF00003BB6657E139
:10237000BA6E7B6ED3187B657A6D7B6ED3183B6526
:102380003A6D7B6ED318FB64BB6E4FEAC303FA68E9
:10239000D31893ED007A3B6D4FEAC303FA68D31864
:1023A000D3ED007A77EE277AC7ED127ABB6E4FEA4B
:1023B000C303FA68D31893ED007A3B6D4FEAC30369
:1023C000FA68D318D3ED007A77EE677AC7ED117A01
:1023D000BB6E4FEAC30303F10403FA68D31893ED0D
:1023E000007A3B6D4FEAC30303F10403FA68D31884
:1023F000D3ED007A77EE277AC7ED107ABB6E4FEAFD
:10240000C30303F10403FA68D31893ED007A3B6D1C
:102410004FEAC30303F10403FA68D318D3ED007A3B
:1024200077EE677AC7ED0F7A7B6D4FEAC303FA68E0
:10243000D31893ED007AFB6C4FEAC303FA68D31804
:10244000D3ED007A77EE277AC7ED0E7ABB6E4FEAAE
:10245000C303FA68D31897ED127AD7ED0E7A37EEE8
:10246000277AD7ED1E7A67EE277AC3ED007A97EDCB
:10247000127AD7ED0E7A77EE677AC7ED127A7B6D16
:102480004FEAC30303F10403FA68D31893ED007A0B
:10249000FB6C4FEAC30303F10403FA68D318D3EDCE
:1024A000007A77EE277AC7ED0D7ABB6E4FEAC30349
:1024B00003F10403FA68D31897ED107AD7ED0D7A7B
:1024C00037EE277AD7ED1E7A67EE277AC3ED007ACA
:1024D00097ED107AD7ED0D7A77EE677AC7ED107A1F
:1024E0007B6D4FEAC30303F10403FA68D31893ED3D
:1024F000007AFB6C4FEAC30303F10403FA68D318B4
:10250000D3ED007A77EE677AC7ED0E7A7B6D4FEAEE
:10251000C303FA68D31893ED007AFB6C4FEAC30348
:10252000FA68D318D3ED007A77EE677AC7ED0D7AA3
:102530007B6D4FEAC303FA68D31897ED127AD7ED93
:102540001E7A67EE277AC3ED007A7B6D4FEAC303EC
:1025500003F10403FA68D31897ED107AD7ED1E7AC9
:1025600067EE277AC3ED007A97ED117AD7ED0E7AF0
:1025700077EE677AC7ED127A97ED117AD7ED0E7A7A
:1025800077EE277AC7ED117A97ED0F7AD7ED0D7AAE
:1025900077EE277AC7ED107A97ED0F7AD7ED0D7A9F
:1025A00077EE677AC7ED0F7A3B6D4FEAC303FA689F
:1025B000D31897ED127AD7ED1E7A67EE277AC3ED1E
:1025C000007A3B6D4FEAC30303F10403FA68D318A2
:1025D00097ED107AD7ED1E7A67EE277AC3ED007A71
:1025E000FB6C4FEAC303FA68D31897ED117AD7ED65
:1025F0001E7A67EE277AC3ED007AFB6C4FEAC303BD
:1026000003F10403FA68D31897ED0F7AD7ED1E7A19
:1026100067EE277AC3ED007ABA6EBB6DD318BB663E
:102620007A89BB6DD21ABB6E9A42BFF4A1AE07F194
:102630007407BD4680BC704780B489B000AFF860B5
:102640007B600B467B8113463B814FF00003BB83CD
:102650007B894FEA53037B837B894FEA53039BB209
:1026600003F101033B834FF00003FB83E5E0FA8BAA
:10267000BB8B9A4280F08880FB8B4FEAC303FA68D9
:10268000D3181B687B61FB8B4FEAC303FA68D3182E
:10269000BA8B4FEAC202F9688A1812681A60BB8BBB
:1026A0004FEAC303FA68D3187A691A60FB8B4FEAC2
:1026B000C30303F10403FA68D3181B687B61FB8B27
:1026C0004FEAC30303F10403FA68D318BA8B4FEA45
:1026D000C20202F10402F9688A1812681A60BB8B00
:1026E0004FEAC30303F10403FA68D3187A691A6046
:1026F000FA8B3B8BD3184FEAC303FA68D3181B68D5
:102700007B61FA8B3B8BD3184FEAC303FA68D3186B
:10271000B98B3A8B8A184FEAC202F9688A18126894
:102720001A60BA8B3B8BD3184FEAC303FA68D318ED
:102730007A691A60FA8B3B8BD3184FEAC30303F113
:102740000403FA68D3181B687B61FA8B3B8BD318A0
:102750004FEAC30303F10403FA68D318B98B3A8B29
:102760008A184FEAC20202F10402F9688A18126854
:102770001A60BA8B3B8BD3184FEAC30303F10403EF
:10278000FA68D3187A691A60FB8B03F101034FEAE8
:10279000C303FA68D3181B687B61FB8B03F1010349
:1027A0004FEAC303FA68D318B98B7A8B8A184FEAB9
:1027B000C202F9688A1812681A60BA8B7B8BD31828
:1027C0004FEAC303FA68D3187A691A60FB8B03F1E6
:1027D00001034FEAC30303F10403FA68D3181B682B
:1027E0007B61FB8B03F101034FEAC30303F1040395
:1027F000FA68D318B98B7A8B8A184FEAC20202F1B1
:102800000402F9688A1812681A60BA8B7B8BD31895
:102810004FEAC30303F10403FA68D3187A691A6014
:102820007B681B88BB833B894FEA43037A68D318D4
:102830007B60FB8B03F10203FB83FA8B7B8BA3F1A1
:1028400002039A427FF613AF07F12407BD4680BC0E
:10285000704700BF90B589B002AFF860B9607A6088
:10286000FB685B697B61FB689B79012B28D1FB6866
:102870009B881946FB68DA68FB681B69F868806802
:102880007C6800940190B86800F064F97B6919884D
:102890007B695A687B699B897869006900907868D0
:1028A000FFF78EF9FB68DB79012B2ED17B69198844
:1028B0007B69DA897B699B687868FFF7BDFE24E055
:1028C0007B6919887B695A687B699B89B868FEF7C0
:1028D00067FCFB68DB79012B08D17B6919887B6970
:1028E000DA897B699B68B868FFF7A6FEFB689B885E
:1028F0001946FB68DA68FB681B69F86880687C68C1
:1029000000940190B86800F005F807F11C07BD4677
:1029100090BD00BF80B491B000AFF860B9607A603C
:102920003B60BB6C03F108033B63BB684FEA0313D6
:10293000A3F10403BA6CD318FB62FB6803F108032C
:10294000BB62BB684FEAC303A3F10403FA68D31860
:102950007B62BB684FEAC303FA68D318FA6812684F
:102960001A60BB684FEAC30303F10403FA68D31883
:10297000FA6852681A60FB6C4FEAC3037A68D3188E
:10298000BB63FB6C4FEAC3033A68D3187B63BB6835
:1029900003F1FF33FB63A6E0BB6B1B683B62BB6BC1
:1029A00003F10403BB63BB6B1B68FB61BB6A93ED64
:1029B000007AD7ED087A67EE277AC7ED067ABB6A08
:1029C00093ED007AD7ED077A67EE277AC7ED057A9F
:1029D000BB6A03F10403BB62BB6A93ED007A7B6AB6
:1029E000D3ED007A37EE277AD7ED077A67EE277AAC
:1029F00097ED067A77EE677AC7ED067ABB6A93EDB4
:102A0000007AD7ED087A67EE277A97ED057A77EEA8
:102A1000277AC7ED057ABB6A03F10403BB627B6BBF
:102A20001B683B617B6A93ED007AD7ED047A67EE11
:102A3000277A97ED057A77EE677AC7ED057A7B6A94
:102A4000A3F104037B627B6A93ED007AD7ED077AEA
:102A500067EE277A97ED057A77EE677AC7ED057A04
:102A60007B6A93ED007AD7ED047A67EE277A97EDCB
:102A7000067A77EE277AC7ED067A7B6AA3F104031C
:102A80007B623B6BBA691A603B6B03F104033B63E7
:102A90003B6B7A691A603B6B03F104033B63D7ED30
:102AA000057AF1EE677AFB6AC3ED007AFB6AA3F15F
:102AB0000403FB62FB6ABA691A60FB6AA3F10403B0
:102AC000FB62FB6C4FEAC3037A6BD3187B63FB6C2E
:102AD0004FEAC303A3F10403BA6BD318BB63FB6BC8
:102AE00003F1FF33FB63FB6B002B7FF455AFBB6837
:102AF0004FEAC303BA6CD318FA6892ED007AFA6809
:102B000002F10402D2ED007A77EE677AC3ED007A23
:102B1000BB684FEAC30303F10403BA6CD3184FF048
:102B200000021A60FB6893ED007AFB6803F104036E
:102B3000D3ED007A77EE277ABB6CC3ED007ABB6CDD
:102B400003F104034FF000021A6007F14407BD4689
:102B500080BC704780B48FB000AFF860B9607A6015
:102B60003B60FB68FB62BB684FEAC30303F10403ED
:102B7000FA68D318BB627B687B633B683B6396E073
:102B80007B6B1B687B627B6B03F104037B637B6B5A
:102B90001B683B62FB6A93ED007AD7ED097A67EE1A
:102BA000277AC7ED077AFB6AD3ED007AB1EE677A30
:102BB000D7ED087A67EE277AC7ED067AFB6A03F14C
:102BC0000403FB62FB6A93ED007ABB6AD3ED007AE3
:102BD00037EE277AD7ED087A67EE277A97ED077AEE
:102BE00077EE277AC7ED077AFB6A93ED007AD7ED87
:102BF000097A67EE277A97ED067A77EE277AC7ED9E
:102C0000067AFB6A03F10403FB623B6B1B687B6182
:102C1000BB6A93ED007AD7ED057A67EE277A97EDD8
:102C2000067A77EE677AC7ED067ABB6AA3F10403EA
:102C3000BB62BB6A93ED007AD7ED057A67EE277A1F
:102C400097ED077A77EE277AC7ED077ABB6A93ED9F
:102C5000007AD7ED087A67EE277A97ED067A77EE55
:102C6000277AC7ED067ABB6AA3F10403BB623B6C0B
:102C7000FA691A603B6C03F104033B643B6CBA696C
:102C80001A603B6C03F104033B647B6C4FEAC303A3
:102C90003A6BD3183B637B6C4FEAC303A3F1040385
:102CA0007A6BD3187B63BB6803F1FF33BB60BB68EF
:102CB000002B7FF465AF07F13C07BD4680BC704731
:102CC00080B582B000AF46F6A813C0F601037B6062
:102CD00040F20003C2F200033B600BE07B681A681D
:102CE0003B681A603B6803F104033B607B6803F1B7
:102CF00004037B603A6840F6B433C2F200039A42A0
:102D0000ECD30C480C494FF000028842B8BF40F8A1
:102D1000042BFFF6FAAFDFF82400016841F47001DC
:102D2000016001F0B7FF00F0A3F807F10807BD4606
:102D300080BD0000B40B00201C46002088ED00E0A0
:102D400080B400AFFEE700BF80B588B000AF024698
:102D50000B46FA71BB71FA794DF61C33C0F60003CD
:102D600053F8223018464FF0010101F081FA4FF478
:102D700080404FF0010101F0F9FA4FF000033B777A
:102D80004FF00003FB77FA794DF61833C0F60003D5
:102D900033F81230BB61FA7940F21403C2F2000337
:102DA00053F8222007F118031046194601F042FE9D
:102DB000BB79012B3AD1FA794DF62433C0F60003E2
:102DC0009A5CF9794DF62833C0F600035B5C104637
:102DD0001946FDF7D9F9FA794DF62033C0F600030C
:102DE00033F812303B614FF000033B754FF008039E
:102DF0007B754FF00103BB7507F11003184602F015
:102E0000B5FAFA794DF62C33C0F600039B5C3B73A0
:102E10004FF00F037B734FF00F03BB734FF00103B1
:102E2000FB7307F10C03184602F050FB07F1200773
:102E3000BD4680BD80B582B000AF0346FB71FA7914
:102E400040F21403C2F2000353F82220F9794DF640
:102E50001833C0F6000333F811301046194601F05C
:102E60008BFE0346184607F10807BD4680BD00BF2C
:102E7000B0B586B002AF01F0D7F901F0B9F901F0B1
:102E80003BF901F083F943F28813C2F200034FF4D7
:102E9000FA421A8043F28813C2F200034FF0000294
:102EA000C4F220129A6043F28813C2F200034FF07A
:102EB0000002C4F27A625A6043F28813C2F200033D
:102EC0004FF001029A8143F28813C2F200034FF0DF
:102ED0000102DA8143F28810C2F2000002F024FC01
:102EE0004FF00103009342F20410C2F2000044F2DA
:102EF000C011C2F200014FF400724FF0000301F064
:102F0000B3FA4FF000004FF00001FFF71DFFFDF78F
:102F10002FFB4FF00000FDF7B9FC4FF00000FDF76C
:102F200079FE40F22000C2F20000FDF793FC4FF45E
:102F3000FC60FDF78FFE4FF0010300934FF0A000FF
:102F40004FF01E014DF63032C0F600024FF0000384
:102F5000FDF7EAFF4FF0010300934FF0A0004FF0A0
:102F600032014DF64832C0F600024FF00003FDF783
:102F7000DBFF40F23000C2F20000FDF76BFC4FF4C3
:102F8000FC60FDF767FE4FF0010300934FF0A000D7
:102F90004FF046014DF65832C0F600024FF00003E4
:102FA000FDF7C2FF4FF0010300934FF0A0004FF078
:102FB0005A014DF66C32C0F600024FF00003FDF7E7
:102FC000B3FF40F23000C2F20000FDF743FC4FF6C1
:102FD000E070FDF73FFE4FF0010300934FF0A000BB
:102FE0004FF096014DF67C32C0F600024FF0000320
:102FF000FDF79AFF00BF4FF00000FFF71BFF0346ED
:10300000002BF8D000BF4FF00000FFF713FF03467E
:10301000012BF8D04FF6FF70FDF70CFE4CF2186054
:10302000FDF718FE4FF00000FDF730FC4FF00103F4
:1030300000934FF020004FF005014DF69832C0F696
:1030400000024FF00103FDF76FFF4FF01F004FF03C
:1030500013014FF481724FF03F03FDF755FE4FF01F
:10306000000300934FF020004FF014014FF48072E2
:103070004FF03D03FDF7FEFD4FF01F004FF08101C3
:103080004FF481724FF06703FDF73EFE4FF00003EF
:1030900000934FF020004FF082014FF480724FF008
:1030A0006503FDF7E7FD4FF00003BB6019E044F254
:1030B0001823C2F20003BA684FEA82029B184FF04D
:1030C00000021A6041F60453C2F20003BA684FEAE4
:1030D00082029B184FF000021A60BB6803F10103E3
:1030E000BB60BB68FF2BE2D941F26F23C3F6832399
:1030F0003B604FF00003FB6043F28413C2F2000315
:103100004FF001021A7000F038BDFB6803F10103B3
:10311000FB60FB68B3F5806F02D94FF00103FB60E1
:103120004FF00000FFF786FE0346012B63D100BF7E
:103130004FF00000FFF77EFE0346012BF8D043F26C
:103140008413C2F200031B7803F10103DAB243F2E5
:103150008413C2F200031A7043F28413C2F2000314
:103160001B78022B0FD14FF0010300934FF020008A
:103170004FF005014DF6B032C0F600024FF00103EA
:10318000FDF7D2FE2CE043F28413C2F200031B7859
:10319000032B0FD14FF0010300934FF020004FF0AD
:1031A00005014DF6C832C0F600024FF00103FDF7ED
:1031B000BBFE15E043F28413C2F200031B78042B1C
:1031C0000ED14FF0010300934FF020004FF00501A6
:1031D0004DF6E032C0F600024FF00103FDF7A4FE09
:1031E00043F28413C2F200031B78042B00F2E6843E
:1031F0004FF00103FB6043F28413C2F200031B781B
:10320000012B45D14FF00003BB603BE0D7ED037AC3
:10321000B8EE677ADFEDBD7A27EE277AD7ED027A2E
:10322000F8EE677A27EE277AD7ED007A67EE277AED
:1032300017EE900A04F09CFB02460B461046194616
:1032400002F0BAFC02460B46104619464FF0000247
:103250004FF00003C4F23E0304F0DEFB02460B46CF
:103260001046194604F0BAFE024643F2C013C2F2F9
:103270000003B9684FEA81015B181A60BB6803F16B
:103280000103BB60BA6840F2FF139A42BED919E24B
:1032900043F28413C2F200031B78022B77D14FF064
:1032A0000003BB606DE0D7ED037AB8EE677ADFED1F
:1032B000977A27EE277AD7ED027AF8EE677A27EE2B
:1032C000277AD7ED007A67EE277A17EE900A04F096
:1032D0004FFB02460B461046194602F06DFC0246B3
:1032E0000B46104619464FF000024FF00003C4F29F
:1032F000340304F091FB02460B4614461D46D7EDFD
:10330000037AB8EE677ADFED827A27EE277AD7ED77
:10331000027AF8EE677A27EE277AD7ED007A67EE21
:10332000277A17EE900A04F023FB02460B4610465C
:10333000194602F041FC02460B46104619464FF072
:1033400000024FF00003C4F2240304F065FB0246C0
:103350000B462046294604F0ADF902460B461046BE
:10336000194604F03BFE024643F2C013C2F20003CA
:10337000B9684FEA81015B181A60BB6803F1010369
:10338000BB60BA6840F2FF139A428CD99AE143F2CB
:103390008413C2F200031B78032B40F0AB804FF084
:1033A0000003BB609FE0D7ED037AB8EE677ADFEDEC
:1033B000577A27EE277AD7ED027AF8EE677A27EE6A
:1033C000277AD7ED007A67EE277A17EE900A04F095
:1033D000CFFA02460B461046194602F0EDFB0246B4
:1033E0000B46104619464FF000024FF00003C4F29E
:1033F0002E0304F011FB02460B4614461D46D7ED82
:10340000037AB8EE677ADFED427A27EE277AD7EDB6
:10341000027AF8EE677A27EE277AD7ED007A67EE20
:10342000277A17EE900A04F0A3FA02460B461046DC
:10343000194602F0C1FB02460B46104619464FF0F2
:1034400000024FF00003C4F2240304F0E5FA024640
:103450000B462046294604F02DF902460B46144639
:103460001D46D7ED037AB8EE677ADFED2A7A27EEAC
:10347000277AD7ED027AF8EE677A27EE277AD7ED2A
:10348000007A67EE277A17EE900A04F071FA024686
:103490000B461046194602F08FFB02460B461046BB
:1034A00019464FF000024FF00003C4F2140304F079
:1034B000B3FA02460B462046294604F0FBF80246C2
:1034C0000B461046194604F089FD024643F2C0132C
:1034D000C2F20003B9684FEA81015B181A60BB6849
:1034E00003F10103BB60BA6840F2FF139A427FF612
:1034F0005AAFE7E043F28413C2F200031B78042BB7
:1035000040F0E0804FF00003BB60D5E0DB0FC94026
:10351000DB0F4941E4CB9641DB0FC9410000484233
:10352000D7ED037AB8EE677A5FED087A27EE277A4F
:10353000D7ED027AF8EE677A27EE277AD7ED007A90
:1035400067EE277A17EE900A04F012FA02460B464D
:103550001046194602F030FB02460B46104619464B
:103560004FF000024FF00003C4F22E0304F054FAAF
:1035700002460B4614461D46D7ED037AB8EE677A2D
:103580005FED1D7A27EE277AD7ED027AF8EE677A9B
:1035900027EE277AD7ED007A67EE277A17EE900AA2
:1035A00004F0E6F902460B461046194602F004FB09
:1035B00002460B46104619464FF000024FF000033A
:1035C000C4F2240304F028FA02460B46204629469A
:1035D00004F070F802460B4614461D46D7ED037AF8
:1035E000B8EE677A5FED357A27EE277AD7ED027A63
:1035F000F8EE677A27EE277AD7ED007A67EE277A1A
:1036000017EE900A04F0B4F902460B46104619462C
:1036100002F0D2FA02460B46104619464FF000025D
:103620004FF00003C4F2080304F0F6F902460B461B
:103630002046294604F03EF802460B4614461D4635
:10364000D7ED037AB8EE677A5FED4D7A27EE277AE9
:10365000D7ED027AF8EE677A27EE277AD7ED007A6F
:1036600067EE277A17EE900A04F082F902460B46BD
:103670001046194602F0A0FA02460B4610461946BB
:1036800004F018F802460B462046294604F012F8CA
:1036900002460B461046194604F0A0FC024643F2CF
:1036A000C013C2F20003B9684FEA81015B181A60C7
:1036B000BB6803F10103BB60BA6840F2FF139A4292
:1036C0007FF62EAF4FF00000FDF7B4FA4FF0000385
:1036D000BB6039E0BB689BB203F1200398B244F2AF
:1036E0001823C2F20003BA684FEA82029B1893EDD6
:1036F000007A5FED767A77EE277AFCEEE77A17EEBE
:10370000903A9BB2D9B2BB689BB203F121039AB243
:10371000BB6803F1010444F21823C2F200034FEA2C
:1037200084041B1993ED007A5FED847A77EE277A93
:10373000FCEEE77A17EE903A9BB2DBB2FDF7C8FADF
:10374000BB6803F10103BB60BB68FE2BC2D94FF617
:10375000E070FDF76FFA4FF00003BB6039E0BB6823
:103760009BB203F1200398B243F2C013C2F20003EC
:10377000BA684FEA82029B1893ED007A5FED997A5E
:1037800077EE277AFCEEE77A17EE903A9BB2D9B241
:10379000BB689BB203F121039AB2BB6803F1010439
:1037A00043F2C013C2F200034FEA84041B1993EDE5
:1037B000007A5FEDA67A77EE277AFCEEE77A17EECD
:1037C000903A9BB2DBB2FDF783FABB6803F10103C9
:1037D000BB60BB68FE2BC2D943F28413C2F2000364
:1037E0001B78012B1AD143F22010C2F200004DF6D3
:1037F000F831C0F60001FA6804F00CFE4FF0010346
:1038000000934FF020004FF0640143F22012C2F207
:1038100000024FF00103FDF787FBADE043F2841394
:10382000C2F200031B78022B1DD1FB684FEA430351
:1038300043F22010C2F200004DF60441C0F6000130
:10384000FA6804F0E7FD4FF0010300934FF0200009
:103850004FF0640143F22012C2F200024FF0010364
:10386000FDF762FB88E043F28413C2F200031B7889
:10387000032B3CD1FB684FEA430343F22010C2F212
:1038800000004DF60441C0F60001FA6804F0C2FDE4
:103890004FF0010300934FF020004FF0640143F21A
:1038A0002012C2F200024FF00103FDF73DFBFA685F
:1038B00013464FEA43039B1843F22010C2F2000064
:1038C0004DF61C41C0F600011A4604F0A3FD4FF06E
:1038D000010300934FF020004FF06E0143F22012DD
:1038E000C2F200024FF00103FDF71EFB44E043F279
:1038F0008413C2F200031B78042B3DD1FB684FEA0E
:10390000430343F22010C2F200004DF60441C0F61A
:103910000001FA6804F07EFD4FF0010300934FF0C0
:1039200020004FF0640143F22012C2F200024FF077
:103930000103FDF7F9FAFA6813464FEA43039A18B0
:10394000FB684FEA830343F22010C2F200004DF6F9
:103950002841C0F6000104F05DFD4FF00103009323
:103960004FF020004FF06E0143F22012C2F200022D
:103970004FF00103FDF7D8FA4FF00003BB6027E0DA
:1039800043F2C013C2F20003BA684FEA82029B18E6
:103990001A6844F21823C2F20003B9684FEA8101A1
:1039A0005B181A6040F60453C2F20003BA684FEA8B
:1039B00082029B181A6841F60453C2F20003B968E8
:1039C0004FEA81015B181A60BB6803F10103BB6019
:1039D000BB68FF2BD4D942F20410C2F2000043F2BC
:1039E000C011C2F2000142F22012C2F20002FEF740
:1039F00031FF42F22010C2F2000040F60451C2F240
:103A000000014FF4007200F061FE40F60450C2F273
:103A100000004FF4007143F2BC12C2F2000244F203
:103A20001423C2F2000301F0C3FD4FF00003BB609A
:103A300023E040F60453C2F20003BA684FEA820260
:103A40009B1893ED007ADFEDBF7A27EE277A43F2D9
:103A5000BC13C2F20003D3ED007AC7EE277A40F61A
:103A60000453C2F20003BA684FEA82029B18C3ED06
:103A7000007ABB6803F10103BB60BA6840F2FF1330
:103A80009A42D6D94FF00000FDF7D4F84FF000036A
:103A9000BB602AE0BB689BB203F1200399B2BB680C
:103AA0009BB203F120039AB2BB6803F1010041F617
:103AB0000453C2F200034FEA80001B18D3ED007AD2
:103AC000FCEEE77A17EE903A9BB2D8B24FF6E67367
:103AD000CFF6FF731B1ADBB208464FF0E601FDF785
:103AE000F7F8BB6803F10103BB60BB68FF2BD1D9BA
:103AF0004FF4FC60FDF79EF84FF00003BB602AE036
:103B0000BB689BB203F1200399B2BB689BB203F17F
:103B100020039AB2BB6803F1010040F60453C2F2DD
:103B200000034FEA80001B18D3ED007AFCEEE77A21
:103B300017EE903A9BB2D8B24FF6E673CFF6FF730A
:103B40001B1ADBB208464FF0E601FDF7C1F8BB686F
:103B500003F10103BB60BB68FF2BD1D94FF0000319
:103B6000BB6003E0BB6803F10103BB60BA684FF6BA
:103B7000FF73C0F201039A42F4D943F28413C2F2F4
:103B800000031B78012B3FF4C0AA43F28413C2F256
:103B900000031B78022B3FF4B8AA43F28413C2F24D
:103BA00000031B78032B3FF4B0AA43F28413C2F244
:103BB00000031B78042B3FF4A8AA00E000BF4FF6D7
:103BC000FF70FDF737F84CF21860FDF743F84FF03F
:103BD0000000FCF75BFE4FF0010300934FF0640020
:103BE0004FF005014DF64042C0F600024FF00103D0
:103BF000FDF79AF94FF00003BB6019E044F2182377
:103C0000C2F20003BA684FEA82029B184FF000022A
:103C10001A6041F60453C2F20003BA684FEA820206
:103C20009B184FF000021A60BB6803F10103BB60F0
:103C3000BB68FF2BE2D94FF000037B604FF015000B
:103C40004FF0140100F00EF94FF46050C4F2000080
:103C50004FF0010101F0E2FA4FF00000FFF7EAF83F
:103C60000346012B08D100BF4FF00000FFF7E2F838
:103C70000346012BF8D0EAE040F6C033C2F200035D
:103C80001B68002B00F09A804FF00003BB601CE023
:103C90007B684FEA4312BB68D21844F2D413C2F2D5
:103CA0000003B96833F8113007EE103AF8EE477A9E
:103CB00043F2C013C2F200034FEA82029B18C3ED25
:103CC000007ABB6803F10103BB60BB681F2BDFD91F
:103CD0007B6803F101037B607B68102B67D94FF091
:103CE00000037B604FF0000000F0B0F942F20410D6
:103CF000C2F2000043F2C011C2F2000142F22012EF
:103D0000C2F20002FEF7A6FD42F22010C2F200004D
:103D100040F60451C2F200014FF4007200F0D6FCEC
:103D200009484FF4007143F2BC12C2F2000244F29F
:103D30001423C2F2000301F03BFC4FF00003BB6010
:103D40002CE000BF0000C842080D002000000C431A
:103D50008096984BBB6803F10102BB6803F1010137
:103D600040F60453C2F200034FEA81015B1893ED61
:103D7000007A5FED0A7A27EE277A5FED0B7AC7EEBD
:103D8000277A40F60453C2F200034FEA82029B18DE
:103D9000C3ED007ABB6803F10103BB60BA6840F26F
:103DA000FF139A42D6D94FF4FC6000F04FF940F669
:103DB000C033C2F200034FF000021A6044F2142331
:103DC000C2F200031B6803F10103184603F0AEFDC5
:103DD00002460B46104619464FF000024FF0000312
:103DE000C4F2400303F018FE02460B461046194683
:103DF0004FF000024FF0814303F038FF02460B46BC
:103E000043F22010C2F200004DF65041C0F600010E
:103E100004F000FB4FF0010300934FF064004FF0FB
:103E20000F0143F22012C2F200024FF00103FDF72E
:103E30007BF84FF00003BB6003E0BB6803F10103B4
:103E4000BB60BA684FF6FF739A42F6D904E74FF4A5
:103E50006050C4F200004FF0000101F0DFF9FFF7FD
:103E6000D9B800BF80B586B002AF02460B46FA80D3
:103E70007B7142F21C13C2F20003FA881A8040F6EA
:103E80000053C2F200037A791A704FF6FF70FCF704
:103E9000D1FEFB8803F10A039AB27B7903F10A038E
:103EA000DBB2104619464FF481724FF09803FCF7CD
:103EB0002BFFFB8803F10B039AB27B7903F10B0311
:103EC000DBB24FF000010091104619464FF48072AA
:103ED0004FF09603FCF7CEFE40F23000C2F2000035
:103EE000FCF7B8FC4CF21860FCF7B4FE4FF000038E
:103EF000FB605EE0FB684FEA0313184603F026FD03
:103F000002460B46104619464FF000024FF00003E0
:103F1000C4F2400303F080FD02460B4610461946EA
:103F20004FF000024FF0814303F0A0FE02460B4623
:103F300043F22010C2F200004DF66041C0F60001CD
:103F400004F068FAFB689BB24FEA03139AB2FB884D
:103F5000D3189BB203F10A039AB27B79A3F15E03F3
:103F6000DBB2104619464FF005024FF00103FCF793
:103F700099FEFB689BB24FEA03139AB2FB88D318F1
:103F80009BB203F10E039AB27B79A3F15403DBB227
:103F90004FF0020100911046194643F22012C2F27E
:103FA00000024FF00103FCF7BFFFFB6803F10103C0
:103FB000FB60FB68102B9DDDFB689BB24FEA03138F
:103FC0009AB2FB88D3189BB203F10E039AB27B79A5
:103FD000A3F15403DBB24FF00201009110461946E1
:103FE0004DF66842C0F600024FF00103FCF79CFF5B
:103FF0004FF00003FB6022E0FB8803F105039AB257
:10400000FB68DBB219464FEAC101CB1A19464FEAE9
:10401000411019460346CB18D9B27B79CB18DBB2D5
:10402000A3F15F03DBB2104619464FF005024FF0D3
:104030000003FCF737FEFB6803F10103FB60FB683C
:10404000062BD9DD07F11007BD4680BDB0B584B0A1
:1040500000AF0346FB80FB881846FCF7EBFD4FF0F2
:104060000003FB6041E0FB689AB242F21C13C2F20B
:1040700000031B88D3189BB203F10B0398B240F6E0
:104080000053C2F200031B78A3F16003D9B2FB68AE
:104090009AB242F21C13C2F200031B88D3189BB2DF
:1040A00003F10B039AB240F60053C2F200031C78EE
:1040B000FB6803F1010540F60453C2F200034FEA26
:1040C00085055B19D3ED007AFCEEE77A17EE903A9E
:1040D0009BB2DBB2E31ADBB2A3F16003DBB2FCF705
:1040E000F7FDFB6803F10103FB60FB68FF2BBADD02
:1040F00007F11007BD46B0BD80B582B000AF4FF4E8
:1041000080633B604FF002033B714FF00003BB71D3
:104110004FF00003FB714FF001037B713B464FF4FE
:104120008060C4F20200194600F084FC4FF00803DE
:104130003B604FF002033B714FF00003BB714FF047
:104140000003FB714FF001037B713B464FF40060AD
:10415000C4F20200194600F06DFC4FF48060C4F216
:1041600002004FF00A014FF0050200F03FFD4FF44E
:104170000060C4F202004FF003014FF0050200F0AE
:1041800035FD07F10807BD4680BD00BF80B584B08E
:1041900000AF4FF46050C4F2000000F0F1FE4FF4A5
:1041A0007A43BB604FF020037B804FF00003BB805D
:1041B0004FF00803BB814FF440733B804FF0000386
:1041C000FB803B464FF46050C4F20000194600F0FB
:1041D0001BFF4FF46050C4F200004FF060014FF03D
:1041E000010201F049F807F11007BD4680BD00BF8C
:1041F00080B582B000AF4FF4C06001F053F94FF0CA
:1042000024033B714FF00103FB714FF000037B71FE
:104210004FF00103BB7107F10403184601F056F992
:1042200007F10807BD4680BD80B500AF41F206002A
:104230004FF0010100F01CF84FF480404FF00101F5
:1042400000F06AF84FF0010000F002F880BD00BFF6
:1042500080B483B000AF0346FB714FF06803C4F233
:104260004723FA791A6007F10C07BD4680BC7047F6
:1042700080B483B000AF78600B46FB70FB78002BF6
:104280000CD04FF46053C4F202034FF46052C4F2F6
:104290000202116B7A680A431A630DE04FF460530F
:1042A000C4F202034FF46052C4F20202116B7A6846
:1042B0006FEA02020A401A6307F10C07BD4680BC90
:1042C000704700BF80B483B000AF78600B46FB70CE
:1042D000FB78002B0CD04FF46053C4F202034FF470
:1042E0006052C4F20202916B7A680A439A630DE04D
:1042F0004FF46053C4F202034FF46052C4F202025E
:10430000916B7A686FEA02020A409A6307F10C0720
:10431000BD4680BC704700BF80B483B000AF7860FA
:104320000B46FB70FB78002B0CD04FF46053C4F2AB
:1043300002034FF46052C4F20202116C7A680A431D
:104340001A640DE04FF46053C4F202034FF460525C
:10435000C4F20202116C7A686FEA02020A401A641F
:1043600007F10C07BD4680BC704700BF80B483B026
:1043700000AF78600B46FB70FB78002B0CD04FF43D
:104380006053C4F202034FF46052C4F20202516C53
:104390007A680A435A640DE04FF46053C4F2020392
:1043A0004FF46052C4F20202516C7A686FEA020262
:1043B0000A405A6407F10C07BD4680BC704700BF35
:1043C00080B483B000AF78600B46FB70FB78002BA5
:1043D0000CD04FF46053C4F202034FF46052C4F2A5
:1043E0000202116A7A680A431A620DE04FF46053C0
:1043F000C4F202034FF46052C4F20202116A7A68F6
:104400006FEA02020A401A6207F10C07BD4680BC3F
:10441000704700BF80B483B000AF78600B46FB707C
:10442000FB78002B0CD04FF46053C4F202034FF41E
:104430006052C4F20202516A7A680A435A620DE07D
:104440004FF46053C4F202034FF46052C4F202020C
:10445000516A7A686FEA02020A405A6207F10C0751
:10446000BD4680BC704700BF80B586B000AFF86025
:10447000B9607A603B604FF00003FB757B689BB2CC
:104480001A46FB681A607B689BB24FEA53039AB2E4
:10449000FB689A80FA684DF67043C0F60003D3605B
:1044A000FA684FF67043C0F6000313613B68DAB256
:1044B000FB689A713B6ADAB2FB68DA71FB681B68C9
:1044C000B3F5007F0AD0B3F5006F02D0802B0AD07D
:1044D0000EE0FB684FF001029A600DE0FB684FF0C0
:1044E00004029A6008E0FB684FF010029A6003E053
:1044F0004FF0FF03FB7500BFFB68BA685A61FB68A9
:104500009B79002B0CD0FB685A69FB689B8810468E
:1045100019464FF001024FF0000301F087F80BE05D
:10452000FB685A69FB689B88104619464FF00002E9
:104530004FF0000301F07AF8FB7D5BB2184607F1FB
:104540001807BD4680BD00BF80B400AFBD4680BC2B
:10455000704700BF80B400AFFEE700BF80B400AF7B
:10456000FEE700BF80B400AFFEE700BF80B400AF3D
:10457000FEE700BF80B400AFBD4680BC704700BFFF
:1045800080B400AFBD4680BC704700BF80B400AFB0
:10459000BD4680BC704700BF80B400AFBD4680BC44
:1045A000704700BF80B582B000AF4FF46050C4F2D6
:1045B00000004FF0600100F095FE0346002B5FD035
:1045C0004FF46050C4F2000000F048FE0346FB8048
:1045D00040F6BC33C2F200031A68FB88D9B240F639
:1045E0000043C2F20003995402F1010240F6BC33C9
:1045F000C2F200031A6040F6BC33C2F200031A682C
:10460000FB884FEA13239BB2D9B2FB884FEA0323FE
:10461000DBB20B43DBB2D9B240F60043C2F2000377
:10462000995402F1010240F6BC33C2F200031A6051
:1046300040F6BC33C2F200031B68FF2B20D940F6C2
:10464000BC33C2F200034FF000021A604FF0320395
:10465000BB80BB8840F60040C2F2000044F2D41197
:10466000C2F200011A4643F28813C2F2000301F0BD
:10467000DFF840F6C033C2F200034FF001021A60C7
:1046800007F10807BD4680BD80B582B000AF87ED59
:10469000010A3860D7ED017AF5EEC07AF1EE10FA32
:1046A00008DD786801F0D4FA02463B681A604FF0E2
:1046B000000305E03B684FF000021A604FF0FF0373
:1046C0005BB2184607F10807BD4680BD80B588B0CB
:1046D00000AFF860B9607A607B684FEA9303FB61D2
:1046E0009BE0FB681B68BB61FB6803F10403FB6094
:1046F000FB681B687B61FB6803F10403FB6097EDBB
:10470000067AD7ED067A27EE277AD7ED056AD7ED38
:10471000057A66EEA77A77EE277ABB68BA6802F167
:104720000402BA60B0EE670A1846FFF7ADFFFB68F7
:104730001B68BB61FB6803F10403FB60FB681B683B
:104740007B61FB6803F10403FB6097ED067AD7ED0C
:10475000067A27EE277AD7ED056AD7ED057A66EE59
:10476000A77A77EE277ABB68BA6802F10402BA60CA
:10477000B0EE670A1846FFF787FFFB681B68BB614E
:10478000FB6803F10403FB60FB681B687B61FB684B
:1047900003F10403FB6097ED067AD7ED067A27EE66
:1047A000277AD7ED056AD7ED057A66EEA77A77EE18
:1047B000277ABB68BA6802F10402BA60B0EE670AF1
:1047C0001846FFF761FFFB681B68BB61FB6803F1DC
:1047D0000403FB60FB681B687B61FB6803F1040357
:1047E000FB6097ED067AD7ED067A27EE277AD7EDAC
:1047F000056AD7ED057A66EEA77A77EE277ABB6869
:10480000BA6802F10402BA60B0EE670A1846FFF710
:104810003BFFFB6903F1FF33FB61FB69002B7FF476
:1048200060AF7B6803F00303FB6129E0FB681B6852
:10483000BB61FB6803F10403FB60FB681B687B61E1
:10484000FB6803F10403FB6097ED067AD7ED067A67
:1048500027EE277AD7ED056AD7ED057A66EEA77AB7
:1048600077EE277ABB68BA6802F10402BA60B0EE4C
:10487000670A1846FFF708FFFB6903F1FF33FB6186
:10488000FB69002BD2D107F12007BD4680BD00BFD8
:1048900080B483B000AF78604FF020437A6812682C
:1048A000796848687968896808437968C9680843FD
:1048B00079680969084379684969084379688969A9
:1048C00008437968C96908437968096A08437968BF
:1048D000496A08437968896A08437968C96A08435C
:1048E0007968096B014343F822107B689B68082BA9
:1048F0000DD14FF020437A6812684FF0204178685C
:10490000006851F8201041F0400143F822104FF0A8
:1049100020437A68126802F101027968496B0868DD
:104920007968496B49684FEA011108437968496B16
:1049300089684FEA012108437968496BC9684FEAE1
:10494000014108437968496B09694FEA01510843FD
:104950007968496B49694FEA016108437968496B95
:104960008969014343F822107B68DB6AB3F5804F05
:1049700027D14FF48273CAF200037A68126879680B
:10498000896B08687968896B49684FEA01110843A7
:104990007968896B89684FEA012108437968896BD6
:1049A00009694FEA015108437968896B49694FEAFF
:1049B000016108437968896B8969014343F82210D2
:1049C00009E04FF48273CAF200037A6812686FF04C
:1049D000704143F8221007F10C07BD4680BC7047B8
:1049E00080B483B000AF78600B46FB70FB78002B7F
:1049F0000CD04FF020434FF02042796852F821202C
:104A000042F001017A6843F822100EE04FF0204294
:104A10004FF02043796853F821104FF6FE73C0F22F
:104A20000F030B40796842F8213007F10C07BD46AF
:104A300080BC704780B487B000AF786039604FF0B9
:104A400000037B614FF000033B614FF00003FB600C
:104A50004FF000037B6186E07B694FF0010202FAB0
:104A600003F33B613B681A683B691340FB60FA68DB
:104A70003B699A4273D17B681A687B694FEA4303AA
:104A80004FF0030101FA03F36FEA03031A407B6856
:104A90001A607B681A683B681B7919467B694FEA84
:104AA000430301FA03F31A437B681A603B681B79DE
:104AB000012B03D03B681B79022B34D17B689A68A9
:104AC0007B694FEA43034FF0030101FA03F36FEAF6
:104AD00003031A407B689A607B689A683B685B793D
:104AE00019467B694FEA430301FA03F31A437B68D3
:104AF0009A607B685A687B699BB24FF0010101FAAA
:104B000003F36FEA03031A407B685A607B685A68B4
:104B10003B689B7919467B699BB201FA03F39BB210
:104B20001A437B685A607B68DA687B699BB24FEAFC
:104B300043034FF0030101FA03F36FEA03031A4042
:104B40007B68DA607B68DA683B68DB7919467B69E9
:104B50004FEA430301FA03F31A437B68DA607B6987
:104B600003F101037B617B690F2B7FF675AF07F1C2
:104B70001C07BD4680BC704780B485B000AF78602C
:104B80000B467B804FF00003FB737B681A697B88C0
:104B90001340002B03D04FF00103FB7302E04FF0F2
:104BA0000003FB73FB7B184607F11407BD4680BC6E
:104BB000704700BF80B483B000AF78600B467B8045
:104BC0007B687A881A8307F10C07BD4680BC704762
:104BD00080B483B000AF78600B467B807B687A88B6
:104BE0005A8307F10C07BD4680BC704780B485B07E
:104BF00000AF786013460A467A807B704FF000035E
:104C0000FB604FF00003BB607A787B8803F00703FA
:104C10004FEA830302FA03F3FB607B884FEAD30376
:104C20009BB21A467B884FEAD3039BB219467B6836
:104C300001F1080153F821107B8803F007034FEAC4
:104C400083034FF00F0000FA03F36FEA03031940E8
:104C50007B6802F1080243F822107B884FEAD303F5
:104C60009BB21A467B6802F1080253F82220FB68C7
:104C70001343BB607B884FEAD3039BB21A467B6821
:104C800002F10802B96843F8221007F11407BD4683
:104C900080BC704780B500AF4FF46D43CEF2000387
:104CA0004FF46D42CEF20002D2F8882042F4700236
:104CB000C3F888204FF46053C4F202034FF46052EB
:104CC000C4F20202126842F001021A604FF460530B
:104CD000C4F202034FF000029A604FF46053C4F232
:104CE00002034FF46052C4F20202126822F084728E
:104CF00022F480321A604FF46053C4F2020343F28C
:104D00001002C2F200425A604FF46053C4F2020330
:104D10004FF46052C4F20202126822F480221A6038
:104D20004FF46053C4F202034FF00002DA6000F067
:104D300009F84FF46D43CEF200034FF000629A6021
:104D400080BD00BF80B483B000AF4FF000037B6034
:104D50004FF000033B604FF46053C4F202034FF482
:104D60006052C4F20202126842F480321A604FF4B8
:104D70006053C4F202031B6803F400333B607B689A
:104D800003F101037B603B68002B03D17B68B3F523
:104D9000A06FECD14FF46053C4F202031B6803F41C
:104DA0000033002B03D04FF001033B6002E04FF0D3
:104DB00000033B603B68012B40F082804FF460535E
:104DC000C4F202034FF46052C4F20202126C42F0C9
:104DD00080521A644FF4E043C4F200034FF4E042FF
:104DE000C4F20002126842F480421A604FF4605329
:104DF000C4F202034FF46052C4F2020292689A6055
:104E00004FF46053C4F202034FF46052C4F2020242
:104E1000926842F400429A604FF46053C4F2020375
:104E20004FF46052C4F20202926842F4A0529A60B7
:104E30004FF46053C4F2020345F20842C0F24072DC
:104E40005A604FF46053C4F202034FF46052C4F24C
:104E50000202126842F080721A6000BF4FF4605381
:104E6000C4F202031B6803F00073002BF6D04FF46A
:104E70007053C4F2020340F205621A604FF46053AB
:104E8000C4F202034FF46052C4F20202926822F0AC
:104E900003029A604FF46053C4F202034FF460526D
:104EA000C4F20202926842F002029A6000BF4FF41C
:104EB0006053C4F202039B6803F00C03082BF6D185
:104EC0004FF46053C4F202034FF46052C4F2020282
:104ED000926822F400029A604FF46053C4F2020315
:104EE0004FF48142C3F20002C3F884204FF46053B0
:104EF000C4F202034FF46052C4F20202126842F09C
:104F000080621A6000BF4FF46053C4F202031B6852
:104F100003F00063002BF6D007F10C07BD4680BC00
:104F2000704700BF80B485B000AF786040F6C433EE
:104F3000C2F200031B68002B08D140F6C433C2F252
:104F4000000344F62062C2F200021A6040F6C43345
:104F5000C2F200031B68FB6040F6C433C2F20003D8
:104F60001A687B68D21840F6C433C2F200031A6094
:104F7000FB68184607F11407BD4680BC704700BFA8
:104F800080B582B000AF78607A684FF44053C4F2C5
:104F900001039A420CD14FF480504FF00101FFF70A
:104FA00039FA4FF480504FF00001FFF733FA26E052
:104FB0007A684FF46053C4F200039A420CD14FF464
:104FC00080404FF00101FFF7FBF94FF480404FF0B4
:104FD0000001FFF7F5F912E07A684FF47053C4F25C
:104FE00000039A420BD14FF400404FF00101FFF74C
:104FF000E7F94FF400404FF00001FFF7E1F907F146
:105000000807BD4680BD00BF80B48BB000AF78609C
:1050100039604FF000037B834FF00203FB844FF0B5
:105020000003BB844FF001037B844FF00003FB615E
:105030004FF000037B614FF000033B614FF0000332
:10504000FB604FF00003BB607B689B8B9BB223F43B
:105050007B6323F00F039AB27B689A837B684FF0DF
:1050600002021A847B689B8B7B833B689B68022BC4
:1050700006D14FF00003BB844FF00203FB849AE09B
:105080003B689B88002B03D14FF001037B8402E037
:105090004FF002037B844FF46053C4F202039B6819
:1050A00003F40003002B0BD04FF46053C4F202034F
:1050B0004FF46052C4F20202926822F400029A6035
:1050C0004FF46053C4F20203D3F8842047F6C07350
:1050D00013404FEA93134FEAC3534FEAD353FB6095
:1050E0004FF46053C4F20203D3F8843003F0E0437A
:1050F0004FEA137303F00703BB604FF46053C4F22D
:1051000002035B6803F03F033B614FF49053C0F22E
:105110007A033A69B3FBF2F3FA6802FB03F2BB6865
:10512000B2FBF3F37B613B68DB88B3F5007F13D1FF
:105130007B694FEA132213464FEA83039B184FEA19
:1051400043031A463B689B68B2FBF3F39BB203F13F
:1051500005039BB2FB6115E07B8C4FEA43137A6930
:10516000B2FBF3F213464FEA83039B184FEA430363
:105170001A463B689B68B2FBF3F39BB203F105034D
:105180009BB2FB61FA694CF6CD43CCF6CC43A3FB52
:1051900002134FEAD303FB61FB699BB203F00103E7
:1051A000BB84BB8CFA69D31A4FEA5303FB84BB8CD4
:1051B0004FEA0323BB84FB8C012B02D9FB8CFF2B12
:1051C00005D94FF00203FB844FF00003BB843B681A
:1051D000DA88BB8C13439AB2FB8C13439AB27B6878
:1051E0001A843B681A883B6859883B6898883B68F2
:1051F0009B8903439BB20B439BB213439AB27B8BB5
:1052000013439BB243F400637B837B687A8B9A835E
:1052100007F12C07BD4680BC704700BF80B483B047
:1052200000AF78600B46FB70FB78002B08D07B68E2
:105230009B8B9BB243F480639AB27B689A8307E0AE
:105240007B689B8B9BB223F480639AB27B689A83C2
:1052500007F10C07BD4680BC704700BF80B483B027
:1052600000AF78607B689B899BB2184607F10C07FA
:10527000BD4680BC704700BF80B485B000AF786089
:1052800013460A46FA70BB704FF00003FB814FF0E3
:105290000003BB81FB784FEA1313DBB2FB81FB8970
:1052A0004FF0010202FA03F3BB81BB78002B08D058
:1052B0007B689B889AB2BB8913439AB27B689A80B9
:1052C0000AE07B689B889AB2BB896FEA03039BB2B2
:1052D00013409AB27B689A8007F11407BD4680BCE0
:1052E000704700BF80B485B000AF78600B46FB709C
:1052F0004FF00003FB734FF00003BB814FF000033E
:105300007B814FF000033B81FB7803F00F034FF0EC
:10531000010202FA03F3BB81FB784FEA1313DBB2FD
:105320007B817B894FF0010202FA03F37B817B686A
:105330009B889AB27B8913403B817B681B899AB218
:10534000BB8913409BB2002B06D03B89002B03D0B6
:105350004FF00103FB7302E04FF00003FB73FB7B94
:10536000184607F11407BD4680BC704780B485B06D
:1053700000AF78604FF00003FB604FF47053C4F24D
:105380000103FB607B689B79002B78D04FF470534E
:10539000C4F201034FF47052C4F2010211687A683A
:1053A00012686FEA02020A401A604FF47053C4F2A6
:1053B00001034FF47052C4F2010251687A68126816
:1053C0006FEA02020A405A607B681B79FA68D318B8
:1053D000FB60FB68FA6811687A6812680A431A6011
:1053E0004FF47053C4F201034FF47052C4F201023F
:1053F00091687A6812686FEA02020A409A604FF474
:105400007053C4F201034FF47052C4F20102D16828
:105410007A6812686FEA02020A40DA607B685B7998
:10542000102B1AD14FF47053C4F201034FF4705291
:10543000C4F2010291687A6812680A439A604FF4D4
:105440007053C4F201034FF47052C4F20102D168E8
:105450007A6812680A43DA601FE04FF47053C4F2AE
:105460000103FB607B685B79FA68D318FB60FB681B
:10547000FA6811687A6812680A431A600DE07B685E
:105480001B79FA68D318FB60FB68FA6811687A68C0
:1054900012686FEA02020A401A6007F11407BD465B
:1054A00080BC704780B483B000AF78604FF46D4328
:1054B000CEF200037A6842F0BF6242F40032DA6052
:1054C00007F10C07BD4680BC704700BF80B485B0B3
:1054D00000AF78604FF00003FB734FF00003BB7325
:1054E0004FF00F037B737B68DB78002B45D04FF4C4
:1054F0006D43CEF20003DB686FEA030303F4E0635D
:105500004FEA1323FB73FB7BC3F10403BB737A7B6A
:10551000FB7B42FA03F37B737B685B781A46BB7BA9
:1055200002FA03F3FB737B689A787B7B1340DAB251
:10553000FB7B1343FB73FB7B4FEA0313FB734FF4BB
:105540006143CEF200037A6812789B18FA7B83F8E5
:1055500000234FF46143CEF200037A6812784FEAD9
:105560005212D2B27968097801F01F014FF00100A0
:1055700000FA01F143F8221014E04FF46143CEF237
:1055800000037A6812784FEA5212D2B27968097829
:1055900001F01F014FF0010000FA01F102F12002B9
:1055A00043F8221007F11407BD4680BC704700BFC6
:1055B00080B489B000AFF860B9607A603B604FF0AA
:1055C00000037B61FB681B68FB61FB6803F104035C
:1055D000FB60BB6803F1FF33BB61FB681B683B6189
:1055E000FB6803F10403FB6097ED077AD7ED047ABB
:1055F000B4EEE77AF1EE10FA05D53B69FB61BA68C3
:10560000BB69D31A7B61BB6903F1FF33BB61BB6923
:10561000002BE2D17B68FA691A603B687A691A60EC
:1056200007F12407BD4680BC704700BF80B485B039
:1056300000AF786079807A703B704FF00003FB73A5
:105640007B687A881A807A6844F24063C0F6010366
:1056500053607B687A789A707B683A78DA707B68F6
:105660001B88402B2DD0402B02DC102B39D048E07A
:10567000B3F5807F15D0B3F5806F42D17B684FF0D2
:1056800001029A817B684FF00102DA817A684DF25B
:105690008073C0F6000393607B684FF06A521A6112
:1056A00033E07B684FF004029A817B684FF004027C
:1056B000DA817B68194A9A607B684FF06E521A61F2
:1056C00023E07B684FF010029A817B684FF0100254
:1056D000DA817B68124A9A607B684FF072521A61D5
:1056E00013E07B684FF040029A817B684FF04002E4
:1056F000DA817B680B4A9A607B684FF076521A61B8
:1057000003E04FF0FF03FB7300BFFB7B5BB2184667
:1057100007F11407BD4680BC704700BF86D700085C
:105720009ED70008FED700082DE9F84F3C4A3D4BB4
:1057300005461A601B683C4A0026934211D13B4A39
:10574000476800F110041360E6600661A6606660B9
:10575000A661666126613846002102F023FE08B189
:1057600026E0FEE738464FF0874102F087FC02F062
:10577000FFF880463846894602F0FAF8064628883F
:105780000F4602F0E3F824A3D3E9002302F06EFAF7
:1057900002460B463046394601F08CFF02460B4666
:1057A0004046494602F062FA02F0F8FBA08300E0AE
:1057B000A683AF680021384602F0F4FD10BB2E88A6
:1057C000300202F0C3F8824638468B4602F0D0F829
:1057D00011A3D3E9002302F01FF980463046894621
:1057E00002F0B4F802460B464046494601F062FF1B
:1057F00002460B465046594602F038FA02F0CEFBFC
:10580000E08301E00023E3832A884FF47A73B2FB3C
:10581000F3F32384BDE8F88F1F85EB51B81E1940C0
:10582000C2A507F400300240CDB5E8B5C80B002092
:105830002DE9F04FA1B01F92B04A1E911168B04AF5
:10584000914200D0FEE703F11002546911690B94F4
:10585000D468089191680694D48B059199899569CB
:105860000D9406244C430995958B4FEA81094FEA24
:10587000C10B0C954D0005EB010809EB010A1894CA
:10588000C1EB0B0C00241F6956681295CDF85880A7
:10589000CDF84C90CDF85CA0CDF854B0CDF864C0F4
:1058A00007940391019313E190F80080DFF860A260
:1058B000039D1AF80840DDF8489036190A9610F84A
:1058C00005C0904E1AF80C4016F80850169904EBD3
:1058D0004504E7190E9710F809408B4F1AF8045049
:1058E00017F8088010F801B0454416F80C8017F836
:1058F0000C9005EB48051AF80B8016F804C0C1445B
:1059000009EB4C0C139BCDF83CC010F803903C5DA8
:105910001AF809C016F80B80644404EB48080F9C81
:10592000CDF840804444DDF85C801C9410F808C039
:1059300017F80B801AF80C401899444416F809809F
:1059400017F8099004EB480404EB050BCDF874B08C
:1059500010F801801AF808B0D94416F80CB009EB19
:105960004B0BCDF844B00E9B17F80CC05B44DDF830
:1059700064B01B9310F80B9016F808B01AF809A041
:105980000F99D4440CEB4B0BDDF828C04FEA051AF5
:10599000DC44CDF868C0C5EB0A0A17F808C04FF020
:1059A0000A0808FB01AA16F80960119BCDF850B04F
:1059B0009A44DDF840B00CEB460604EB440CE2449C
:1059C00017F809704FF0060909FB0BAA06990A9B04
:1059D0008A444FF01C0C0CFB03AA0E994FF0150BD8
:1059E0000BFB01AA1D9BCDF828A04FF02E0A0AFB45
:1059F00003FA1C99302303FB01AA05991A9B514411
:105A00004FF0240A0AFB03131B99CA440AFB013115
:105A100006910F9905EB450509FB015925012C1B42
:105A2000109BA14408FB0399149C119D0CFB049945
:105A30000BFB05990E990A9B0D9C49440591A3F512
:105A4000003A64B1089D0B990D9B6C1A54445C4359
:105A500048BFFF342412CDF82CA00894A2460C9C19
:105A600064B1099DC4F580746C430C9901FB0A4430
:105A7000002CB8BFFF3424120994A2461F9B03FBDD
:105A80000AFABAF1000F04DD0AF1080A4FEA2A1AED
:105A900006E0BAF1080C48BF0AF1070C4FEA2C1ACD
:105AA000019DDDF81C80EC8947F6BC7C04FB08F402
:105AB000164DE245B8BFD4461E99159BAC45A8BF0C
:105AC000654608F1010821F81450C018CDF81C8073
:105AD000148C079DA542FFF6E7AE019B05991F6157
:105AE000069B9160D360089D0B99099B56601561D8
:105AF00051619361204621B0BDE8F08FC80B0020B2
:105B0000CDB5E8B538010020380000204480FFFF03
:105B10003802002070B5C1F30A5521F07F46A5F286
:105B2000FF3426F470060029ACBF01234FF0FF3389
:105B3000132C024646F480160DDC002C36DB4FF4A5
:105B4000002141FA04F18E19C4F1140426FA04F07C
:105B500000FB03F070BD1E2C0ED8332C0FDDA5F218
:105B60001340A5F2334506FA00F602FA05F246EABA
:105B7000020000FB03F070BD02F0E8F970BDA5F271
:105B800013454FF0004121FA05F10A18C4F134041D
:105B900028BF0136202C18BF22FA04F006FA05F6B9
:105BA00008BF0020304300FB03F070BDB4F1FF3F9D
:105BB0000CBF1846002070BD30B542F2FB1421F036
:105BC0000045C3F6E974A54287B002460B461CDDCA
:105BD0004FF6FF74C7F6EF74A54203DD01F068FDD0
:105BE00007B030BD02AA00F08BF800F003000128D6
:105BF0001DD0022810D008BB01230093DDE902016B
:105C0000DDE9042301F04CFBEAE7002200920023C7
:105C1000002201F045FBE3E701210091DDE90423C7
:105C2000DDE9020101F03CFB01F10041D8E7DDE9CB
:105C30000201DDE9042300F00FFBD1E7DDE90201F9
:105C4000DDE9042300F008FB01F10041C8E700BFD3
:105C500030B52DED028B284C8BB008EE100A00F009
:105C600093FA94F900300133054609D018EE100A72
:105C700001F0E2FC20B1B5EEC08AF1EE10FA04D4D6
:105C800028460BB0BDEC028B30BD1C4A012118EE3A
:105C9000100A002500910192089501F069FE247810
:105CA000CDE90401CDE902018CB90022002343ECC7
:105CB000172B8DED067B684601F036FC88B10898FD
:105CC000A0B9DDE9060102F089F90546D8E7002010
:105CD000002102460B4601F0C9FF022CCDE9060166
:105CE000E9D102F091FB21230360E8E702F08CFB8D
:105CF00008990160E5E700BF38030020406601080D
:105D00002DE9F04F42F2FB1321F00046C3F6E97390
:105D10009E428FB004460D468B460F46904640F398
:105D2000A9804DF67B12C4F202029642894629DC14
:105D30000029E1A3D3E9002340F3D28101F0B8FCAC
:105D400042F2FB14C3F6F974A64282468B4600F079
:105D5000AA80DBA3D3E9002301F0AAFC04460D4688
:105D6000504622462B465946C8E9004501F0A0FCA2
:105D7000D3A3D3E9002301F09BFC4FF0010AC8E94B
:105D8000020181E042F2FB13C4F239139E4240F358
:105D9000AA804FF6FF72C7F6EF72964278DC4FEAA0
:105DA000265AAAF2164AA6EB0A510F46064602F0F8
:105DB000CDF801F0CBFD04460D4622462B46304679
:105DC0003946CDE9084501F073FC00230022C4F2F6
:105DD000701301F021FE0F46064602F0B7F801F0FD
:105DE000B5FD04460D4622462B4630463946CDE9E0
:105DF0000A4501F05DFC00230022C4F2701301F09B
:105E00000BFE00220023CDE90C0102F06DF8002802
:105E100000F08981032620462946002200230AAF8C
:105E2000013E02F061F840B177E90201002200234F
:105E3000013E02F059F80028F6D1A74A0223009348
:105E4000019208A852464146334600F031FBB9F1B1
:105E5000000F824618DAD8F80400D8F80C1000F1C8
:105E6000004201F10043C8F80420C8F80C30CAF120
:105E7000000A09E0C2E900450023002243EC172B89
:105E800088ED027B4FF0000A50460FB0BDE8F08F5E
:105E900002460B4601F00CFC4FF0000AC8E9020173
:105EA000C8E90001F0E77EA3D3E9002301F000FC7C
:105EB0007DA3D3E9002306460F4601F0F9FB044613
:105EC0000D4622462B4630463946C8E9004501F0CA
:105ED000EFFB75A3D3E9002301F0EAFB4FF0010AC1
:105EE000C8E90201D0E701F093FA71A3D3E90023D6
:105EF00004460D4601F090FD00230022C3F6E07336
:105F000001F0D8FB02F022F8824601F01FFD6AA3DF
:105F1000D3E90023CDE9040101F07EFD02460B46E2
:105F20002046294601F0C4FB65A3D3E900230446BB
:105F30000D46DDE9040101F06FFDBAF11F0FCDE957
:105F400002012046294631DC0AF1FF37634A52F844
:105F50002730B3422AD0DDE9022301F0A9FB024633
:105F60000B46C8E9002383460F465A463B46204667
:105F7000294601F09DFBDDE9022301F099FBB9F10F
:105F8000000F02460B46C8E90223BFF67DAF07F1BA
:105F9000004701F10042C8F800B0C8F80470C8F822
:105FA0000800C8F80C20CAF1000A6DE7DDE90223F9
:105FB00001F07EFB36150B460F46C1F30A5102462F
:105FC0008346701A1028C8E90023CEDD34A3D3E934
:105FD0000023DDE9040101F01FFDCDE90201DDE947
:105FE00002232046294601F063FBCDE90601DDE9E5
:105FF00006232046294601F05BFBDDE9022301F080
:1060000057FB29A3D3E9002304460D46DDE904012B
:1060100001F002FD22462B4601F04AFBCDE90201C8
:10602000DDE90223DDE9060101F042FB0246834679
:10603000C1F30A50361A0B46312E0F46C8E9002329
:1060400040F3938020A3D3E90023DDE9040101F0AC
:10605000E3FC06460F4632463B46DDE9060101F009
:1060600027FB04460D4622462B46DDE9060101F0DA
:106070001FFB32463B4601F01BFB15A3D3E900236F
:1060800006460F46DDE9040101F0C6FC32463B46F8
:1060900001F00EFBCDE90201204629465BE700BF77
:1060A0000000601A61B4D03D7370032E8A19A33BBF
:1060B00083C8C96D305FE43F00004054FB21F93FC5
:1060C0003163621A61B4D03D0000002E8A19A33BEF
:1060D000C14920259A837B39C866010848660108B2
:1060E00001F0E8FA42F2FB13C3F6F9739E428246CE
:1060F0008B461AD01EA3D3E9002301F0DBFA044635
:106100000D46504622462B465946C8E9004501F047
:10611000CFFA17A3D3E9002301F0CCFA4FF0FF3AEE
:10612000C8E90201B0E6032687E613A3D3E90023FA
:1061300001F0C0FA12A3D3E9002306460F4601F08E
:10614000B9FA04460D4622462B4630463946C8E980
:10615000004501F0ADFA0AA3D3E9002301F0AAFA41
:106160004FF0FF3AC8E902018EE6DDE90645FCE69C
:106170003163621A61B4D03D0000601A61B4D03D51
:106180007370032E8A19A33B20F00042B2F1FF4F37
:10619000F0B407EE900A03464BD2002A45D00028FF
:1061A00050DBC115B2F5000F09D210F400044ED136
:1061B0005B0001341802FBD5C4F10100091823F07B
:1061C0007F4525F40006A1F17F07F90746F4000298
:1061D00048BF520053004FF0807400267F109C424D
:1061E000304629DD5B004FF4000218248518510861
:1061F0009D4204F1FF3402DCA8185B1BB6185B005B
:1062000042189A4202DC9B1A501876185B004A0822
:10621000013CEBD113B106F001017618701000F1CA
:106220007C5606EBC75607EE906A17EE900AF0BC54
:10623000704747EEA77AF8E74FF0007003F17F430D
:106240002646CFE737EEE70AC0EE007AEDE70120F9
:10625000B4E700BF000000002DE9F04F21F0004935
:10626000B9F1795F85B006460F4604460D46924661
:106270009B466DDA01F06AFE002800F0F880324695
:106280003B463046394601F0C7FB7DA3D3E90023E6
:1062900004460D4601F0C0FB7BA3D3E9002301F0C7
:1062A00009FA22462B4601F0B7FB79A3D3E9002374
:1062B00001F0FEF922462B4601F0AEFB76A3D3E9AE
:1062C000002301F0F7F922462B4601F0A5FB74A349
:1062D000D3E9002301F0ECF922462B4601F09CFBA8
:1062E00071A3D3E9002301F0E5F922462B4601F022
:1062F00093FBCDE900010023002220462946C3F686
:10630000E07301F089FBDDE90023804689462046E1
:10631000294601F081FB524604460D465B46304655
:10632000394601F079FB02460B462046294601F02A
:10633000BFF902460B464046494601F0B9F90B4603
:1063400000210246C3F6F071002001F0B1F980E0AF
:1063500002460B4601F060FB49A3D3E90023044643
:106360000D4601F059FB48A3D3E9002301F0A2F93F
:1063700022462B4601F050FB45A3D3E9002301F050
:1063800097F922462B4601F047FB43A3D3E90023AC
:1063900001F090F922462B4601F03EFB40A3D3E9E1
:1063A000002301F085F922462B4601F035FB3EA380
:1063B000D3E9002301F07EF92B46224601F02CFBA5
:1063C00043F23233C3F6D3739945CDE9000192DD30
:1063D0000020C3F6E97081453EDCA9F5001189462D
:1063E000002100220020C3F6F0714B46904601F0D8
:1063F0005FF9CDE902010023204629460022C3F6B9
:10640000E07301F009FB42464B4601F051F9DDE92A
:106410000023804689462046294601F0FDFA52466F
:1064200004460D465B463046394601F0F5FA024611
:106430000B462046294601F03BF902460B464046F2
:10644000494601F035F902460B46DDE9020101F04B
:106450002FF905B0BDE8F08F9FED077B4FF00009E5
:106460008DED027B4FF00008C3F6D279C3E700211F
:106470000020C3F6F071ECE7000000000000E73FE9
:10648000D43888BEE9FAA8BDC4B1B4BD9EEE213EA1
:10649000AD529C804F7E923E9015CB19A001FA3EE2
:1064A0007751C1166CC1563F4C5555555555A53FB2
:1064B0002DE9F04F4AF6AB25ADF51B7DD41EC2F693
:1064C000AA2585FB0465E417A49F304E0A91C4EB0E
:1064D000A50525EAE5749A4656F827600D94E3432E
:1064E0000AF1FF37069703EB4305834602EBC5002D
:1064F000069A0D99089612EB06090990C7EB01045C
:1065000046D4A144A59EC4EB0908002C06EB8405E3
:1065100009F1010908F00108C0F2A186286801F01C
:1065200015FA013420AE04274C45E6E902012FD0CC
:10653000B8F1000F21D0002CC0F29586E85901F087
:1065400005FA013404374C45E6E9020115D11FE094
:10655000E85901F0FBF90437013406F10808C6E9EF
:1065600002010FD4E85901F0F1F9013404374C4528
:10657000C8E9020108F108060AD0002CE8DA002078
:106580000021E8E700200021EFE700BFD067010805
:10659000089B002B68DB0899CDF80CA072A800EBD3
:1065A000C1020DF5E0790492069D002DC0F2DD8256
:1065B000039C22AE06EBC40757E902230AF1FF3C15
:1065C000DBE900010CF0010801F026FA02460B4657
:1065D0000020002101F06EF80126083F56450446D0
:1065E0000D46DE4638D0B8F1000F12D077E902230D
:1065F000DBE9020101F010FA02460B46204629466B
:1066000001F058F80226564504460D460BF1080ED7
:1066100022D0F04657E90223D8E9020101F0FCF943
:1066200002460B462046294601F044F857E9042368
:1066300004460D46D8E9040101F0EEF902460B4686
:106640002046294601F036F80236103F56450446EA
:106650000D4608F11008DDD1E9E90245039B0499D4
:10666000581C894503909FD1089E0EAA02EB860410
:1066700002920B940396039D039AEB009AA8C1180B
:10668000002A059351E9286740F3BB80059D0DF56D
:10669000E479A944039D00230DAC04EB850C002292
:1066A000C3F6706330463946CDF804C001F0B4F942
:1066B00001F04CFC01F04AF900230022C4F27013EF
:1066C00004460D4601F0A8F902460B46304639460D
:1066D00000F0EEFF01F03AFC0DF138082B46C8F847
:1066E0000000224679E9020100F0E4FFDDF804C071
:1066F000E04506460F46CCF3800300F082805BB392
:1067000000230022C3F67063CDF804C001F084F9C1
:1067100001F01CFC01F01AF900230022C4F27013EE
:1067200004460D4601F078F902460B4630463946DC
:1067300000F0BEFF01F00AFC0DF13C082246C8F84B
:1067400000002B4679E9020100F0B4FFDDF804C037
:10675000E04506460F4654D0CDF810B0D346E24689
:1067600000230022C3F670633046394601F054F925
:1067700001F0ECFB01F0EAF800230022C4F27013F0
:1067800004460D4601F048F902460B4630463946AC
:1067900000F08EFF01F0DAFB22462B46C8F8040019
:1067A00079E9020100F086FF00230022C3F670633E
:1067B00006460F4601F030F901F0C8FB01F0C6F8BB
:1067C00000230022C4F2701304460D4601F024F9A0
:1067D00002460B463046394600F06AFF01F0B6FB30
:1067E0002246C8F808002B4679E9020100F062FF52
:1067F00008F10808D04506460F46B1D1DA46DDF863
:1068000010B0099A3046394600F092FE00224FF04F
:106810007F5306460F4601F0FFF800F0FDFD002310
:106820000022C4F2200301F0F7F802460B4630467E
:10683000394600F03DFF04460D4601F087FB8046D7
:1068400001F084F802460B462046294600F030FF4E
:10685000099C002C06460F4640F34B81039B0DF12B
:10686000380C5A1EC4F118055CF8223043FA05F1C1
:1068700001FA05F01B1AC4F117044CF822308844C1
:1068800043FA04F5002D5ADD039A002A08F10108A5
:1068900040F375810EAB029803EB82010C1A53F89A
:1068A000042B201FC0F38000002422B1C2F18074A9
:1068B00043F8044C01248B422BD068B10F9A043367
:1068C000002C00F00D81C2F1FF1000F57F4443F869
:1068D000044C01248B421CD053F8042BC2F1FF104E
:1068E00000F57F4014B9C2F1807012B143F8040C76
:1068F000012453F8042BC2F1FF1000F57F401CB9AE
:10690000C2F18070002AE5D001248B4243F8040CC8
:10691000E2D1099B002B0FDD012B00F01081022B2F
:106920000AD103990EAB481E53F8202022F07F4174
:1069300021F4400243F82020022D00F0E38030468D
:1069400039460022002301F0CFFA002800F04684E7
:106950000398089F441EA74222DC0DF1380E0EEB6F
:1069600080010B460B9E53F8042D881B011FB34278
:10697000C1F3800011D030B153F8046D0B998B42F4
:1069800042EA060209D00B9E53F8040D53F8041D89
:106990000243B34242EA0102F6D1002A40F0F380FA
:1069A000089C0DF13809671E59F82730002B40F07C
:1069B000E88009EB8702012052F8046D0130002EB7
:1069C000FAD003990D1801F10109A9450C9500F3BE
:1069D0008180069C039B0D98A59E04EB09077A1EF7
:1069E00022AC191804EBC20705980C9A049772ABF5
:1069F00006EB81051918561C039505910796039D12
:106A000055F8040F039500F0A1FF049C069FE4E9EC
:106A10000201002F049460DB09EB0A0322A800EBBB
:106A2000C30757E902230AF1FF3EDBE900010EF03C
:106A3000010800F0F1FF02460B460020002100F0A3
:106A400039FE0126083F56450D460446594638D0C2
:106A5000B8F1000F12D077E90223DBE9020100F060
:106A6000DBFF02460B462046294600F023FE0226A5
:106A700056450D4604460BF1080122D0884657E9D9
:106A80000223D8E9020100F0C7FF02460B46204668
:106A9000294600F00FFE57E9042304460D46D8E9C5
:106AA000040100F0B9FF02460B462046294600F0DB
:106AB00001FE0236103F564504460D4608F1100807
:106AC000DDD1059A079BE2E9024509F101099945E3
:106AD000059294D10C980390CDE500240025F0E7B1
:106AE000002A3FF4F7AEC2F1807243F8042C01246F
:106AF000F0E631D103980DF1380E411E5EF82120E9
:106B0000D515BFE6002132463B460020C3F6F071A2
:106B100000F0CEFD06460F46002C3FF410AF0021DA
:106B2000099A0020C3F6F07100F002FD02460B4600
:106B30003046394600F0BCFD06460F46FFE6039896
:106B40000DF1380E431E5EF8231021F07F4222F42F
:106B500000004EF82300EFE600230022C3F6E073A6
:106B600001F0E0F920B90025E9E60024002573E5ED
:106B7000039A0225002A08F101083FF78BAE002492
:106B8000C7E601201DE70EAA0695099D52F824309C
:106B9000CDF81C80183D0995002B40F0688302EB6E
:106BA00084060394294656F8040D013C1839002840
:106BB000F9D00394099100210020C3F6F071099ADD
:106BC00000F0B6FC039E002E04460D46C0F2CE80B7
:106BD000771C0497049A0DF5E47B0DF138090BEB53
:106BE000C70609EB8208CBEB0603083B58F8040DF7
:106BF000C3F3C00700F0AAFE22462B4600F00CFFAC
:106C0000002366E90201002220462946C3F670638C
:106C100000F002FF5E4504460D4643D0AFB158F880
:106C2000040D00F093FE22462B4600F0F5FE0023F3
:106C300066E90201002220462946C3F6706300F08F
:106C4000EBFE5E4504460D462CD0474657F8040C33
:106C500000F07CFE22462B4600F0DEFE002346E9D3
:106C600002010022C3F670632046294600F0D4FEDC
:106C700004460D4657F8080C00F068FE22462B46E5
:106C800000F0CAFE002346E90401002220462946FE
:106C9000C3F6706300F0C0FE103E083F5E45044638
:106CA0000D46D3D10399481E4FF000090590089A6C
:106CB000002AC0F28E82B9F1000FC0F28A82059ECE
:106CC000089B3E4FC9EB0608002400250026DB0781
:106CD0000BEBC80812D5F8E90223F7E9020100F02E
:106CE0009BFE02460B462046294600F0E3FC0D467B
:106CF00008990126B14204462CDA2DE0D8E9022396
:106D0000D7E9020100F088FE02460B4620462946DC
:106D100000F0D0FC044607F10800089F06F1010AC4
:106D200008F10802023657450D4600F1080702F146
:106D3000080811DBCA450FDCD2E90223D0E90201C1
:106D400000F06AFE02460B462046294600F0B2FCDF
:106D500004460D464E45D1DD4AAB03EBC901C1E9FE
:106D60000045049C09F10109A145A0D1A49C032C74
:106D70001DD8DFE814F0EF0175017501250000252D
:106D80002F460698002800F05A81059E0A9C7168DB
:106D9000F0683268B368226001F1004100F1004000
:106DA00007F100476160A360E06025616761079DAE
:106DB00005F007000DF51B7DBDE8F08FD8670108D1
:106DC000039E002E40F36582039E4AAD721C05EBC4
:106DD000C20353E9046753E902AB05954CAD049334
:106DE0005C1B52465B4630463946089500F062FC13
:106DF0008046894642464B463046394600F058FCAC
:106E000002460B465046594600F054FCDDF810B0DF
:106E10006BE90201083CAB45C4F3C0044BE90289AD
:106E200059D0E4B15BE9046742464B4639463046E7
:106E300000F040FC04460D46224639462B463046BB
:106E400000F036FC02460B464046494600F032FC54
:106E50006BE90201089FBB454BE902453BD0DA468E
:106E60007AE902895BE9046742464B463046394677
:106E700000F020FC04460D463046394622462B469B
:106E800000F016FC02460B464046494600F012FC54
:106E90004BE902015AE9048922462B464AE9024598
:106EA0004046494600F006FC06460F4632463B4641
:106EB0004046494600F0FCFB02460B462046294668
:106EC00000F0F8FBAAF1080B4AE902014BE902675E
:106ED000089EB345C3D1039901297FF750AF0498A9
:106EE000059F50E902AB50E9044510375B46C61BCD
:106EF000524620462946039700F0DCFB804689462F
:106F000042464B462046294600F0D2FB02460B463D
:106F10005046594600F0CEFBDDF810B06BE9020197
:106F2000083EBB45C6F3C0064BE9028959D0E6B11D
:106F30005BE9046742464B463046394600F0BAFBEF
:106F400004460D4622462B463046394600F0B0FB3B
:106F500002460B464046494600F0ACFB6BE9020195
:106F6000039A93454BE902453BD0DA467AE9028918
:106F70005BE9046742464B463046394600F09AFBCF
:106F800004460D463046394622462B4600F090FB1B
:106F900002460B464046494600F08CFB4BE9020195
:106FA0005AE9048922462B464AE9024540464946A9
:106FB00000F080FB06460F4632463B4640464946B7
:106FC00000F076FB0B4602462946204600F072FB95
:106FD000039BAAF1080B9B454AE902014BE90267B2
:106FE000C3D1049C039D0020671B014674E9022362
:106FF00000F060FB083FC7F3C0060F4603998C42C0
:1070000005463FF4BEAE36B12846394674E9022340
:1070100000F050FB0AE054E902232846394600F00C
:1070200049FB54E9042300F045FB103C039EB442A5
:1070300005460F46EFD1069800287FF4A6AE059CC2
:10704000059994ED007B91ED020B2A460A9C0A9D5E
:107050003B4685ED007B84ED020BC4E90423A6E6E4
:1070600003980028C0F21181039D4AAC691C04EB0F
:10707000C10600203546C4EB060C75E90223ACF1CD
:10708000080E0146CEF3C00800F014FBA5420246EC
:107090000F461BD0B8F1000F07D075E9022300F0AE
:1070A00009FBA54202460F4610D01046394655E965
:1070B000022300F0FFFA064655E90423304600F0AB
:1070C000F9FA103DA54202460F46EED1069D002D6D
:1070D00000F0828007F10040034619463B460A9FB4
:1070E0001046C7E90001D4E9000100F0E1FA039A73
:1070F000002A844624DD254604EBC2066046F5E9F5
:10710000022300F0D7FA341B083CB542C4F3C00494
:10711000844615D03CB16046F5E9022300F0CAFA76
:10712000B54284460CD06046D5E9022300F0C2FA8D
:10713000D5E9042300F0BEFA1035B5428446F2D1F9
:10714000069E0EB101F100410A9F62460B46C7E957
:1071500002232CE6039E002EC0F29480711C4AACE0
:1071600004EBC10300201D46C4EB0308014675E98A
:10717000022300F09FFAA8F10807A542C7F3C00850
:107180000E4607461BD0B8F1000F07D075E9022361
:1071900000F090FAA54207460E4610D055E90223AA
:1071A0003846314600F086FA0646304655E9042353
:1071B00000F080FA103DA54207460E46EED1069C2F
:1071C0000CB106F100460A9D3A463346C5E9002354
:1071D000EDE500240025BFE538467DE70695099DCD
:1071E000CDF81C806A423046394600F0A1F90023F0
:1071F0000022C4F2701304460D4600F093FE0028EE
:1072000037D000230022C3F670632046294600F0E1
:1072100003FC00F09BFE00F099FB00230022C4F267
:10722000701306460F4600F0F7FB02460B46204659
:10723000294600F03DFA00F089FE039C0DF1380C60
:1072400039464CF82400304600F080FE099D621C4F
:107250000EAB18350392099543F82200ABE40020E9
:107260000021FFF75EB900200021FFF76AB90394FF
:10727000A1E42946204600F069FE0EAB039943F8CD
:10728000210098E400273E4699E7002217464AACC1
:107290001CE700254AA82F46059072E50000000073
:1072A0002DE9F04F21F00046B6F1795F85B0044634
:1072B0000D460F469046994603DA00F047FE002837
:1072C0006ED022462B462046294600F0A5FB2246DA
:1072D0002B4606460F4600F09FFB41A3D3E900234F
:1072E00082468B463046394600F096FB3EA3D3E9F2
:1072F000002300F0DDF932463B4600F08DFB3CA355
:10730000D3E9002300F0D6F932463B4600F084FB77
:1073100039A3D3E9002300F0CBF932463B4600F015
:107320007BFB37A3D3E9002300F0C4F90E9BCDE922
:107330000001002B39D000230022C3F6E073404641
:10734000494600F069FBDDE90023CDE90201504622
:10735000594600F061FB02460B46DDE9020100F0F0
:10736000A7F932463B4600F057FB42464B4600F039
:107370009FF925A3D3E9002306460F4650465946F8
:1073800000F04AFB02460B463046394600F092F9BF
:1073900002460B462046294600F08AF904460D466F
:1073A0002046294605B0BDE8F08F02460B46304620
:1073B000394600F031FB14A3D3E9002300F078F93B
:1073C00052465B4600F028FB02460B462046294603
:1073D00000F070F904460D46E2E700BFAFF300800D
:1073E0007CD5CF5A3AD9E53DEB9C2B8AE6E55A3E4F
:1073F0007DFEB157E31DC73ED561C119A0012A3FEB
:10740000A6F810111111813F495555555555C53FE5
:1074100021F00041704700BF2DE9F843C1F30A583D
:10742000A8F2FF36132E02460B4604460D460F46C1
:1074300021DC002E45DB4FF6FF7CC0F20F0C4CFA2E
:1074400006F808EA010C5CEA000C10D034A3D3E97A
:10745000002300F02FF90022002300F06DFD20B181
:10746000002D3EDB25EA080700243B462246104655
:107470001946BDE8F883332E07DDB6F5806FF6D1E7
:1074800000F018F902460B46F1E7A8F2134C4FF052
:10749000FF3929FA0CF919EA000FE8D020A3D3E943
:1074A000002300F007F90022002300F045FD00282A
:1074B000DBD0002D1BDB24EA09042F463B46224685
:1074C000D5E717A3D3E9002300F0F4F80022002346
:1074D00000F032FD0028C8D0002D15DB002427461F
:1074E000C3E74FF4801141FA06F6AD19BAE7142E3E
:1074F00008D0C8F58668012308F1030803FA08F0EC
:107500000419D8D30135D6E725F0004222430023E1
:107510009A42CBF6F07318BF002418BF1F46A4E7A9
:107520009C7500883CE4377E002070470000000016
:10753000C1F30A532DE9F04104460D4606460F46B5
:1075400090467BBB21F0004353EA000C26D0002379
:107550000022C4F2503300F05FFA43F6B042CFF697
:10756000FF72904504460D4606460F463BDBC1F3CD
:107570000A53363B03EB080040F2FE7290421BDDDB
:1075800022462B4628A1D1E9000100F081F826A36C
:10759000D3E9002300F040FA04460D462046294670
:1075A000BDE8F08140F2FF72934224D003EB080063
:1075B00040F2FE729042E3DC002806DD21F0FF423B
:1075C00022F4E00545EA0055E8E710F1350F19DA35
:1075D0004CF25030804522462B46D3DC14A1D1E931
:1075E000000100F055F812A3D3E9002300F014FACB
:1075F00004460D46D2E702460B4600F05BF804460F
:107600000D46CBE721F0FF4525F4E001363041EA95
:1076100000531946002320460022C3F6904300F091
:10762000FBF904460D46B9E79C7500883CE4377EBB
:1076300059F3F8C21F6EA50108B902207047B0F1D6
:10764000004FFAD0A0F500026FF001439A4201D832
:107650000420704700F1FF419942F9D94FF6FE73BB
:10766000421EC0F27F039A4201D80320704700F106
:1076700000414A1E9A42F8D9B0F1FF4F05D010F5EB
:10768000000F14BF0020012070470120704700BF89
:1076900003F0004321F0004230B40D46044643EAB3
:1076A000020130BC704700BF81F0004102E000BF22
:1076B00083F0004330B54FEA41044FEA430594EAB2
:1076C000050F08BF90EA020F1FBF54EA000C55EAED
:1076D000020C7FEA645C7FEA655C00F0E2804FEABE
:1076E0005454D4EB5555B8BF6D420CDD2C4480EAA0
:1076F000020281EA030382EA000083EA010180EAD0
:10770000020281EA0303362D88BF30BD11F0004F1D
:107710004FEA01314FF4801C4CEA113102D0404253
:1077200061EB410113F0004F4FEA03334CEA13338E
:1077300002D0524263EB430394EA050F00F0A780A6
:10774000A4F10104D5F1200E0DDB02FA0EFC22FAA1
:1077500005F2801841F1000103FA0EF2801843FA95
:1077600005F359410EE0A5F120050EF1200E012A86
:1077700003FA0EFC28BF4CF0020C43FA05F3C018C4
:1077800051EBE37101F0004507D54FF0000EDCF13D
:10779000000C7EEB00006EEB0101B1F5801F1BD3E6
:1077A000B1F5001F0CD349085FEA30004FEA3C0CEA
:1077B00004F101044FEA445212F5800F80F09A80E0
:1077C000BCF1004F08BF5FEA500C50F1000041EBE4
:1077D000045141EA050130BD5FEA4C0C404141EBE8
:1077E000010111F4801FA4F10104E9D191F0000F0F
:1077F00004BF01460020B1FA81F308BF2033A3F192
:107800000B03B3F120020CDA0C3208DD02F1140C88
:10781000C2F10C0201FA0CF021FA02F10CE002F1C3
:107820001402D8BFC2F1200C01FA02F120FA0CFCBC
:10783000DCBF41EA0C019040E41AA2BF01EB045105
:10784000294330BD6FEA04041F3C1CDA0C340EDC03
:1078500004F11404C4F1200220FA04F001FA02F346
:1078600040EA030021FA04F345EA030130BDC4F104
:107870000C04C4F1200220FA02F001FA04F340EAF9
:107880000300294630BD21FA04F0294630BD94F0AA
:10789000000F83F4801306BF81F480110134013D91
:1078A0004EE77FEA645C18BF7FEA655C29D094EA02
:1078B000050F08BF90EA020F05D054EA000C04BF80
:1078C0001946104630BD91EA030F1EBF002100206B
:1078D00030BD5FEA545C05D14000494128BF41F00A
:1078E000004130BD14F580043CBF01F5801130BD6E
:1078F00001F0004545F0FE4141F470014FF00000F9
:1079000030BD7FEA645C1ABF194610467FEA655CA9
:107910001CBF0B46024650EA013406BF52EA03354B
:1079200091EA030F41F4002130BD00BF90F0000F39
:1079300004BF0021704730B54FF4806404F1320475
:107940004FF000054FF0000150E700BF90F0000F2E
:1079500004BF0021704730B54FF4806404F1320455
:1079600010F0004548BF40424FF000013EE700BF25
:1079700042004FEAE2014FEA31014FEA02701FBFB5
:1079800012F07F4393F07F4F81F06051704792F087
:10799000000F14BF93F07F4F704730B54FF4607401
:1079A00001F0004521F0004120E700BF50EA01024C
:1079B00008BF704730B54FF000050AE050EA0102F9
:1079C00008BF704730B511F0004502D5404261EB69
:1079D00041014FF4806404F132045FEA915C3FF4AA
:1079E000DCAE4FF003025FEADC0C18BF03325FEA43
:1079F000DC0C18BF033202EBDC02C2F1200300FAF8
:107A000003FC20FA02F001FA03FE40EA0E0021FA1C
:107A100002F11444C1E600BF70B54FF0FF0C4CF406
:107A2000E06C1CEA11541DBF1CEA135594EA0C0FBC
:107A300095EA0C0F00F0DEF82C4481EA030621EAF7
:107A40004C5123EA4C5350EA013518BF52EA033532
:107A500041F4801143F4801338D0A0FB02CE4FF0E4
:107A60000005E1FB02E506F00042E0FB03E54FF014
:107A70000006E1FB03569CF0000F18BF4EF0010E0C
:107A8000A4F1FF04B6F5007F64F5407404D25FEA08
:107A90004E0E6D4146EB060642EAC62141EA5551BB
:107AA0004FEAC52040EA5E504FEACE2EB4F1FD0CFD
:107AB00088BFBCF5E06F1ED8BEF1004F08BF5FEA7B
:107AC000500E50F1000041EB045170BD06F000462D
:107AD00046EA010140EA020081EA0301B4EB5C04DA
:107AE000C2BFD4EB0C0541EA045170BD41F48011D2
:107AF0004FF0000E013C00F3AB8014F1360FDEBFF7
:107B0000002001F0004170BDC4F10004203C35DAD2
:107B10000C341BDC04F11404C4F1200500FA05F355
:107B200020FA04F001FA05F240EA020001F00042F6
:107B300021F0004110EBD37021FA04F642EB06016C
:107B40005EEA430E08BF20EAD37070BDC4F10C0496
:107B5000C4F1200500FA04F320FA05F001FA04F25A
:107B600040EA020001F0004110EBD37041F1000146
:107B70005EEA430E08BF20EAD37070BDC4F1200551
:107B800000FA05F24EEA020E20FA04F301FA05F2B9
:107B900043EA020321FA04F001F0004121FA04F261
:107BA00020EA020000EBD3705EEA430E08BF20EA31
:107BB000D37070BD94F0000F0FD101F0004640006B
:107BC00041EB010111F4801F08BF013CF7D041EAED
:107BD000060195F0000F18BF704703F000465200F1
:107BE00043EB030313F4801F08BF013DF7D043EAC2
:107BF0000603704794EA0C0F0CEA135518BF95EA78
:107C00000C0F0CD050EA410618BF52EA4306D1D1FE
:107C100081EA030101F000414FF0000070BD50EA1D
:107C2000410606BF1046194652EA430619D094EAA7
:107C30000C0F02D150EA013613D195EA0C0F05D191
:107C400052EA03361CBF104619460AD181EA0301E5
:107C500001F0004141F0FE4141F470014FF000009D
:107C600070BD41F0FE4141F4780170BD70B54FF038
:107C7000FF0C4CF4E06C1CEA11541DBF1CEA1355B8
:107C800094EA0C0F95EA0C0F00F0A7F8A4EB05049A
:107C900081EA030E52EA03354FEA013100F0888091
:107CA0004FEA03334FF0805545EA131343EA12635A
:107CB0004FEA022245EA111545EA10654FEA00260F
:107CC0000EF000419D4208BF964244F1FD0404F5C8
:107CD000407402D25B084FEA3202B61A65EB030524
:107CE0005B084FEA32024FF480104FF4002CB6EBE1
:107CF000020E75EB030E22BFB61A754640EA0C0061
:107D00005B084FEA3202B6EB020E75EB030E22BFA0
:107D1000B61A754640EA5C005B084FEA3202B6EBE1
:107D2000020E75EB030E22BFB61A754640EA9C00A0
:107D30005B084FEA3202B6EB020E75EB030E22BF70
:107D4000B61A754640EADC0055EA060E18D04FEA2E
:107D5000051545EA16754FEA06164FEAC30343EACE
:107D600052734FEAC2025FEA1C1CC0D111F4801F9B
:107D70000BD141EA00014FF000004FF0004CB6E794
:107D800011F4801F04BF01430020B4F1FD0C88BF33
:107D9000BCF5E06F3FF6AFAEB5EB030C04BFB6EB3E
:107DA000020C5FEA500C50F1000041EB045170BD31
:107DB0000EF0004E4EEA113114EB5C04C2BFD4EB5E
:107DC0000C0541EA045170BD41F480114FF0000EE2
:107DD000013C90E645EA060E8DE60CEA135594EA5E
:107DE0000C0F08BF95EA0C0F3FF43BAF94EA0C0F61
:107DF0000AD150EA01347FF434AF95EA0C0F7FF4D6
:107E000025AF104619462CE795EA0C0F06D152EA29
:107E100003353FF4FDAE1046194622E750EA41060D
:107E200018BF52EA43067FF4C5AE50EA41047FF41E
:107E30000DAF52EA43057FF4EBAE12E74FF0FF3C83
:107E400006E000BF4FF0010C02E000BF4FF0010C54
:107E50004DF804CD4FEA410C7FEA6C5C4FEA430CCD
:107E600018BF7FEA6C5C1BD001B050EA410C0CBF1C
:107E700052EA430C91EA030F02BF90EA020F00207E
:107E8000704710F1000F91EA030F58BF994208BFE5
:107E900090422CBFD8176FEAE37040F001007047A2
:107EA0004FEA410C7FEA6C5C02D150EA013C07D1F9
:107EB0004FEA430C7FEA6C5CD6D152EA033CD3D044
:107EC0005DF8040B704700BF8446104662468C463E
:107ED0001946634600E000BF01B5FFF7B7FF002871
:107EE00048BF10F1000F01BD4DF808EDFFF7F4FF9A
:107EF0000CBF012000205DF808FB00BF4DF808ED25
:107F0000FFF7EAFF34BF012000205DF808FB00BF47
:107F10004DF808EDFFF7E0FF94BF012000205DF869
:107F200008FB00BF4DF808EDFFF7CEFF94BF01201E
:107F300000205DF808FB00BF4DF808EDFFF7C4FF17
:107F400034BF012000205DF808FB00BF4FEA41026A
:107F500012F5001215D211D56FF47873B3EB62529B
:107F600012D94FEAC12343F0004343EA505311F0C2
:107F7000004F23FA02F018BF404270474FF0000054
:107F8000704750EA013005D111F0004008BF6FF092
:107F9000004070474FF00000704700BF4A0011D208
:107FA00012F5001211D20DD56FF47873B3EB625253
:107FB0000ED44FEAC12343F0004343EA505323FA5F
:107FC00002F070474FF00000704750EA013002D1D4
:107FD0004FF0FF3070474FF0000070474FEA41020A
:107FE000B2F1E04324BFB3F5001CDCF1FE5C0DD917
:107FF00001F0004C4FEAC0024CEA5070B2F1004F61
:1080000040EB830008BF20F00100704711F0804F63
:1080100021D113F13872BCBF01F00040704741F428
:1080200080114FEA5252C2F11802C2F1200C10FA2C
:108030000CF320FA02F018BF40F001004FEAC12310
:108040004FEAD32303FA0CFC40EA0C0023FA02F3B4
:108050004FEA4303CCE77FEA625307D150EA01338A
:108060001EBF4FF0FE4040F44000704701F000405A
:1080700040F0FE4040F40000704700BF4FF0FF0C9E
:108080001CEAD0521EBF1CEAD15392EA0C0F93EAAD
:108090000C0F6FD01A4480EA010C400218BF5FEA4F
:1080A00041211ED04FF0006343EA501043EA5111C2
:1080B000A0FB01310CF00040B1F5000F3EBF4900BC
:1080C00041EAD3715B0040EA010062F17F02FD2AC0
:1080D0001DD8B3F1004F40EBC25008BF20F00100A3
:1080E000704790F0000F0CF0004C08BF49024CEABA
:1080F000502040EA51207F3AC2BFD2F1FF0340EA4C
:10810000C250704740F400004FF00003013A5DDCBC
:1081100012F1190FDCBF00F000407047C2F10002FD
:10812000410021FA02F1C2F1200200FA02FC5FEAEA
:10813000310040F1000053EA4C0308BF20EADC7034
:10814000704792F0000F00F0004C02BF400010F4A6
:10815000000F013AF9D040EA0C0093F0000F01F053
:10816000004C02BF490011F4000F013BF9D041EA75
:108170000C018FE70CEAD15392EA0C0F18BF93EA77
:108180000C0F0AD030F0004C18BF31F0004CD8D1A1
:1081900080EA010000F00040704790F0000F17BF28
:1081A00090F0004F084691F0000F91F0004F14D06E
:1081B00092EA0C0F01D142020FD193EA0C0F03D1C6
:1081C0004B0218BF084608D180EA010000F00040C9
:1081D00040F0FE4040F40000704740F0FE4040F4A4
:1081E000400070474FF0FF0C1CEAD0521EBF1CEA43
:1081F000D15392EA0C0F93EA0C0F69D0A2EB030261
:1082000080EA010C49024FEA402037D04FF08053FA
:1082100043EA111143EA10130CF000408B4238BFBF
:108220005B0042F17D024FF4000C8B4224BF5B1ACD
:1082300040EA0C00B3EB510F24BFA3EB510340EA1B
:108240005C00B3EB910F24BFA3EB910340EA9C00C9
:10825000B3EBD10F24BFA3EBD10340EADC001B0139
:1082600018BF5FEA1C1CE0D1FD2A3FF650AF8B42DD
:1082700040EBC25008BF20F0010070470CF0004CEA
:108280004CEA50207F32C2BFD2F1FF0340EAC25015
:10829000704740F400004FF00003013A37E792F0D6
:1082A000000F00F0004C02BF400010F4000F013A34
:1082B000F9D040EA0C0093F0000F01F0004C02BF2F
:1082C000490011F4000F013BF9D041EA0C0195E798
:1082D0000CEAD15392EA0C0F08D142027FF47DAF31
:1082E00093EA0C0F7FF470AF084676E793EA0C0F21
:1082F00004D14B023FF44CAF08466EE730F0004C1F
:1083000018BF31F0004CCAD130F000427FF45CAFAE
:1083100031F000437FF43CAF5FE700BF4FF0FF3C1C
:1083200006E000BF4FF0010C02E000BF4FF0010C6F
:108330004DF804CD4FEA40024FEA41037FEA226C38
:1083400018BF7FEA236C11D001B052EA530C18BF5A
:1083500090EA010F58BFB2EB030088BFC81738BFBF
:108360006FEAE17018BF40F0010070477FEA226CAD
:1083700002D15FEA402C05D17FEA236CE4D15FEAA9
:10838000412CE1D05DF8040B704700BF84460846DD
:108390006146FFE70FB5FFF7C9FF002848BF10F19E
:1083A000000F0FBD4DF808EDFFF7F4FF0CBF0120E3
:1083B00000205DF808FB00BF4DF808EDFFF7EAFF6D
:1083C00034BF012000205DF808FB00BF4DF808ED28
:1083D000FFF7E0FF94BF012000205DF808FB00BF1D
:1083E0004DF808EDFFF7D2FF94BF012000205DF8A3
:1083F00008FB00BF4DF808EDFFF7C8FF34BF0120B0
:1084000000205DF808FB00BF40F26873C2F2000371
:10841000186870470EB470B59DB021AC40F2687317
:1084200054F8042BC2F200036FF000454FF40271C0
:108430000646ADF814100495079518680296234671
:1084400002A94FF6FF750696ADF81650019400F09C
:1084500039F8029B00221A701DB0BDE8704003B0CD
:10846000704700BF20F0030110F00300C0F10000CE
:1084700051F8043B00F1040C4FEACC0C6FF0000201
:108480001CBF22FA0CF213434FF0010C4CEA0C2CE7
:108490004CEA0C4CA3EB0C0222EA030212EACC12C7
:1084A00004BF51F8043B0430F4D013F0FF0F1FBF9A
:1084B000013013F47F4F013013F47F0F18BF0130E8
:1084C000704700BF2DE9F04FC3B014460A911093D6
:1084D0000C9003F00DF800681390FFF7C3FF1590A0
:1084E0000A98838903F080010AB200200021CDE9B7
:1084F000160122B10A980369002B01F0C482002002
:1085000032ABDFF8FC9411900793259327902690C7
:10851000A246189019900F901E469AF80040002C21
:1085200000F09C81252C00F099810AF1010501E001
:10853000252904D02C46013521780029F8D1CAEB31
:1085400004057DB1269B279AC6F800A0591C501936
:10855000072975602790269100F3648108360F9AE9
:1085600050190F902378002B00F0648100224FF007
:10857000FF3194F8018009910D9204F1010A8DF800
:108580007320089220202B210AF1010AA8F1200370
:10859000582B00F2B982DFE813F0FB01B702B702F3
:1085A0000502B702B702B702B702B702B702B201BB
:1085B0004E02B7023E010C02B702C502CC02CC0249
:1085C000CC02CC02CC02CC02CC02CC02CC02B70250
:1085D000B702B702B702B702B702B702B702B702D3
:1085E000B70284008001B7028001B702B702B70268
:1085F000B7024702B702B7026D00B702B702B7026F
:10860000B702B7025900B702B702DD01B702B702DD
:10861000B702B702B702B702B702B702B702B70292
:108620003502880080018001800187028800B7023E
:10863000B702AB02B702530271008E02A402B70266
:108640006102B7025D00B702B702BD01089D45F0A7
:1086500010040894089B9D0600F18F810899CC06B0
:1086600041F19280109A1568171D2C46109700252D
:10867000012312E0089A42F010050895089F17F0B0
:10868000200340F0FF80089C14F0100001F06E8081
:10869000109F3A1D3C681092002500278DF87370DA
:1086A00017E0089D45F010030893089FBF0640F1AE
:1086B000D780109DEB1D23F00700D0E90023083080
:1086C000109014461D46002A73F10000C0F2338753
:1086D00001230999002903DB089F27F080000890F7
:1086E00054EA050240F0F183099A002A40F0ED8334
:1086F000002B40F05786089BD90741F10C8042AF10
:10870000302007F8410D079AD41B0E94099C0E984F
:108710009DF873301294A042B8BF204600220B90FF
:10872000149213B10B9B591C0B91089B13F0020080
:10873000099002D00B998C1C0B94089A12F0840BB0
:1087400040F028820D9D0B9BED1A002D40F32282F4
:10875000102D41F30682279A269BA44910243160EC
:108760001A9111195A1CA5F1110E072A7460CEF343
:1087700000132791269200F370850836103D102DC6
:1087800040F3FC818BB1013246F678031031C0F61C
:108790000103072A86E818002791269200F36C85CA
:1087A0000836103D102D40F3E9813346CDF86CB00A
:1087B0002E46BB460A9D0C9F13E00833013246F655
:1087C00078001031C0F60100103E072A83E811003E
:1087D0002791269200F3BE81103E0833102E40F3FD
:1087E000C881013246F678001031C0F60100072A30
:1087F00083E8110027912692DFDD3846294625AA15
:1088000003F0C2FFE8B92799269A32ABD6E70D9A52
:10881000109352420D92089B43F0040208929AF87A
:108820000080B1E60C980A9925AA03F0ADFF40B983
:1088300032AE94E6279B23B10C980A9925AA03F03F
:10884000A3FF0A9881890F9801F0400213B2002B10
:1088500018BF4FF0FF3043B0BDE8F08F544681E6BB
:108860000898C50600F15B8608994C0640F15786CA
:10887000109A109FB2F90040381DE51722462B468A
:10888000109020E7109BDD1D25F0070101F1080085
:108890001090D1E900450023FFE6109CE11D21F076
:1088A000070000F1080710974468D0F800B021468F
:1088B0005846CDE916012146584603F01FFF01280E
:1088C0002146584640F0388700220023FFF716FB68
:1088D000002841F037829DF87330002708991297DD
:1088E00003244348434F0B9421F080020E9400244C
:1088F000B8F1470FD8BF07460892149411E7109AB1
:10890000109B12680433002A0D9280DB9AF80080D5
:10891000109339E6384F1897089FB9061FD5109C59
:10892000E01D20F00703D3E9004503F10801109191
:108930000898C70740F1828454EA050200F07E845B
:10894000302240F002078DF874208DF8758008976A
:108950000223A2E6089F294DB9061895DFD4089C8A
:10896000E20600F1F1850898430640F1ED85109B81
:10897000191D1C8810910025DAE7109CE31D23F0D7
:10898000070101F108001090D1E90045012384E6B8
:108990009DF87330002B40F003878DF873009AF830
:1089A0000080F1E5089B43F0010208929AF80080EC
:1089B000EAE5544614F8018BB8F12A0F01F0C98298
:1089C000A8F130030022092B01F2068214F8018B72
:1089D00002EB820203EB4202A8F13003092BA2460C
:1089E000F4D942EAE2720992D0E500BF7868010842
:1089F00024680108286801084868010834680108EB
:108A000068680108109F10993C68012300200A1D26
:108A10008DF873000B9310928DF8A0400E9328AF41
:108A200000221292149280E6089A42F008030893FA
:108A30009AF80080A8E58DF873109AF80080A3E5F5
:108A4000089CA10640F1B08610990F9A10980B6807
:108A5000D417011D1A605C6010915EE5109D002422
:108A60008DF873402F680435002F01F0F480099AC7
:108A7000002A3846C1F251802146099A02F0ECFFE3
:108A8000002801F08F8109991294C01B88420E9032
:108A900040F3E38721EAE17009990B909DF8733068
:108AA00010950E9114943CE6089B43F04002089206
:108AB0009AF8008068E5109D10992868089B0F1DA2
:108AC000AA49109743F002024FF07808044630207C
:108AD0008DF87580002508928DF874001891022396
:108AE000DBE5089B43F0200208929AF800804BE5F2
:108AF0009AF80080B8F16C0F534600F00087089A8E
:108B000042F0100308933FE5B8F1000F3FF492AE36
:108B1000012700240B970E978DF8A0808DF87340E5
:108B200028AF7DE7089A42F0800308939AF8008006
:108B30002AE552460023A8F1300512F8018BA8F16E
:108B4000300403EB8303092C05EB43039246F2D96F
:108B50000D931BE53846294625AA03F015FE00288B
:108B60007FF46FAE103E102E32AB2799269A3FF756
:108B700038AE5F46DDF86CB035461E46501C1A9B79
:108B80004C19072886E828002794269000F30F84C4
:108B9000083600E0279C9DF8731069B1269B581C8D
:108BA000013401210DF173020728326071602794AE
:108BB000269000F3FE820836099B63B12698411C7B
:108BC000023402231DAA072932607360279426917C
:108BD00000F3FA820836BBF1800F00F02D82129D5F
:108BE0000E9AAD1A002D6FDD102D40F3FA852699EF
:108BF0005F48C6F800904FF0100B4A1CA5F1110C0D
:108C00005C44072AC6F804B0099027942692CCF356
:108C1000001300F3A9820836103D102D49DD63B121
:108C200001321034072A86E8000A2794269200F3BE
:108C3000A9820836103D102D3BDD314620464646C0
:108C40003C46DDF828800C9F0DE0083101321030E1
:108C5000103D072A81E8000A2692279017DC103D74
:108C60000831102D21DD01321030072A81E8000A79
:108C700027902692E9DD3846414625AA03F084FD77
:108C800000287FF4DEAD2798269A32A9DEE7384621
:108C9000414625AA03F078FD00287FF4D2AD103DAF
:108CA000102D32A92798269ADDDCB04627460E46BD
:108CB0000446501C099B6419072886E8280027945D
:108CC000269000F36B820836089BDA0500F12881B4
:108CD00026980E9A0E993760431CA418072B7160D2
:108CE0002794269300F3B0800836089A530740F182
:108CF000B9800D9D0B982D1A002D40F3B380102DD7
:108D000040F3CF87269BDFF86C8046F67807C0F6E5
:108D100001073760591C1027A5F1110BE419072929
:108D20007760CBF3001B2794269100F3C6830836A7
:108D3000103D102D40F3B680BBF1000F11D0013172
:108D400046F678001034C0F60100072986E8810055
:108D50002794269100F3D7830836103D102D40F359
:108D6000A1803246DDF830B00A9E18E0486801085C
:108D700068680108786801080832411C46F67800E6
:108D80001034C0F60100103D072982E881002691C9
:108D9000279477DC103D0832102D40F38280481C68
:108DA00046F678011034C0F60101072882E88200F7
:108DB00027942690E0DD5846314625AA03F0E4FCCE
:108DC00000287FF43EAD279C269832AAD5E7119D56
:108DD000012D40F37B84269B37605D1C013401210B
:108DE000072D71602794269500F37B840836159B28
:108DF00013980135E418072D86E809002794269575
:108E000000F37C840836DDE9160100220023FFF719
:108E10006BF8002840F0D782119A0137501E2418B1
:108E200001353760072D70602794269500F3868101
:108E3000083619980135241821AB072D336070606E
:108E4000279426957FF750AF0C980A9925AA03F02E
:108E50009BFC00287FF4F5AC089A279C530732AEA0
:108E60003FF547AF0F980B990D9A9142ACBF401850
:108E700080180F90002C40F06D810024269432AEB3
:108E8000FFF74BBB5846314625AA03F07DFC00286E
:108E90007FF4D7AC103D102D32AA279C26993FF7BE
:108EA0007EAF16464B1C2C19072BC6F80080756048
:108EB00027942693D6DD0C980A9925AA03F064FC22
:108EC00000287FF4BEAC279CCCE7012B00F0A881E2
:108ED000022B0DF1C70C00F0878107234FEAD40E57
:108EE00004EA03004EEA457BE90830305C460D4653
:108EF000C0B254EA050167468CF800000CF1FF3C53
:108F0000ECD1089AD4073B4605D5302803D030244D
:108F1000674603F8014C079CE21B0E92FFF7F6BB75
:108F2000B8F1650F7FF753AFDDE91601002200238A
:108F3000FEF7DAFF002800F0AC812698A849431C10
:108F400001340122072B316072602794269300F3CD
:108F50004D8408361E98119B984203DB0899CB0775
:108F60007FF5C3AE269B1598139A7060591C241880
:108F7000072932602794269100F379850836119DE0
:108F8000013D002D7FF7B1AE102D40F38882269869
:108F9000119AC6F800901027411CA2F1120EE41994
:108FA00007297760DFF83CB227942691CEF30018AA
:108FB00000F310860836103D102D40F37382B8F18F
:108FC000000F0ED0013110340729C6F800907760E9
:108FD0002794269100F30B860836103D102D40F3A0
:108FE00061822046DDF830800A9C10E00836591C6A
:108FF0001030103D0729C6F8009077602691279021
:1090000000F31F810836103D102D40F3E8834B1C00
:109010001030072BC6F80090776027902693E5DD87
:109020004046214625AA03F0AFFB00287FF409AC97
:109030002798269B32AEDAE70D9D0B982D1A002D4E
:109040007FF7CDAD102D40F3A8862698654AC6F867
:1090500000904FF0100B0130A5F111035C4407287C
:10906000C6F804B0099227942690C3F3001300F3C6
:1090700013830836103D102D48DD63B101301034E4
:10908000072886E8000A2794269000F31383083601
:10909000103D102D3ADD214632460C9C2E460346EB
:1090A0000A9D0DE00832431C1031103E072B82E868
:1090B000000A2693279117DC103E0832102E21DD7E
:1090C000581C1031072882E8000A27912690E9DD14
:1090D0002046294625AA03F057FB00287FF4B1ABB0
:1090E0002799269832AADEE72046294625AA03F0CA
:1090F0004BFB00287FF4A5AB103E102E32AA279917
:10910000269BDDDC35460C4616461846411C099B5D
:109110006419072986E828002794269100F3008324
:1091200008365CE52F4A09920135099BE419072DA1
:1091300086E88800279426957FF77AAE0C980A99DE
:1091400025AA03F021FB00287FF47BAB32AE279CDD
:10915000269D6EE60C980A9925AA03F015FB0028B7
:109160003FF48BAEFFF76DBB0C980A99069325AAC6
:1091700003F00AFB069B00287FF463AB32AE279C0A
:10918000269A49E50C980A9925AA03F0FDFA0028C9
:109190007FF457AB32AE279C269A4BE50C980A9980
:1091A00025AA03F0F1FA00287FF44BAB279C32AEDE
:1091B0008AE50C980A9925AA03F0E6FA00287FF4BC
:1091C00040AB279C32AEF7E40C980A9925AA03F02D
:1091D000DBFA00287FF435AB279C32AEFBE400BFFE
:1091E0006468010868680108DDF860E00B960F21EB
:1091F00004EA01060EEB060027092A0947EA05746E
:109200000378154654EA050267468CF800300CF1E5
:10921000FF3CEDD107990B9EC81B0E90FFF776BA65
:10922000002D08BF0A2C80F0548142AF303407F87B
:10923000414D079BD91B0E91FFF768BA0223FFF738
:109240002CBA4046214625AA03F09EFA00287FF456
:10925000F8AA32AE27982699D5E60C980A99069373
:1092600025AA03F091FA069B00287FF4EAAA32AE01
:109270002799269AFFF782BA0C980A9925AA03F033
:1092800083FA00287FF4DDAA32AE2799269AFFF7E9
:1092900088BA1E9D002D40F3B582119D1499119A34
:1092A0008D42A8BF0D46B818002D09900ADD269BF7
:1092B0003760591C6419072975602794269100F3BB
:1092C0007D840836149A25EAE575551B002D40F378
:1092D0004F81102D40F3748226999F4BC6F8009061
:1092E0004FF010080131A5F1110E44440729C6F8CA
:1092F00004800E9327942691CEF3001B00F3518433
:109300000836103D102D40F35E82BBF1000F0FD0E8
:10931000013110340729C6F80090C6F8048027945C
:10932000269100F371840836103D102D40F34B82D6
:109330002046DDF830B00A9C12E006F10802591C04
:109340001030103D0729C2F80090C2F80480269121
:1093500027901BDC02F10806103D102D40F3078416
:109360004B1C1030072BC6F80090C6F804802790DD
:109370002693E2DD5846214625AA03F005FA002887
:109380007FF45FAA2798269B32AAD8E75846214641
:1093900025AA03F0F9F900287FF453AA32AE2798E2
:1093A0002699D9E7099C32AF0E94FFF7AFB90C9814
:1093B0000A9925AA03F0E8F900287FF442AA279C1D
:1093C00032AEFFF7E8BB119F013F002F7FF731ADB1
:1093D000102F7FF7A7AE11985F4BC6F800904FF0A3
:1093E00010080135A0F1120B4444072DC6F8048083
:1093F000099327942695CBF3001B00F3BA83083614
:10940000103F102F7FF790AEBBF1000F0FD001354A
:109410001034072DC6F80090C6F8048027942695CE
:1094200000F3B3830836103F102F7FF77DAE21463F
:10943000DDF830B00A9C10E0083601351031103FDD
:10944000072DC6F80090C6F80480279126951ADCEF
:109450000836103F102F40F35D8301351031072D82
:10946000C6F80090C6F8048027912695E4DD58469A
:10947000214625AA03F088F900287FF4E2A927995C
:10948000269D32AED9E75846214625AA03F07CF93D
:1094900000287FF4D6A932AE2799269DD9E72699D0
:1094A000DFF8B4B0013164190729C6F800B075605F
:1094B000279426917FF718ACC6E40C980A9925AA40
:1094C00003F062F900287FF4BCA932AE279C2699EC
:1094D0002EE40DF1C70B204629460A22002303F093
:1094E00069FE30328BF80020204629460A220023EC
:1094F00003F060FE04460D4654EA05005F460BF19A
:10950000FF3BE8D107E50C980A9925AA03F03CF93E
:1095100000287FF496A932AE279C26991DE4109965
:109520000C68E51722462B460F1D002A73F1000038
:109530001097BFF6CDA82D22644265EB45058DF846
:1095400073200123FFF7C5B8109A1568171D2C4624
:1095500010970025FFF7ECB9686801080C980A9984
:1095600025AA03F011F900287FF46BA9279C32AEDD
:109570001E9B119A14989342074472DB0899C907FD
:109580006FD4099D1199ED1BC91AA942B8BF0D46A8
:10959000002D0ADD269A3760501C64190728756073
:1095A0002794269000F36F83083625EAE5754D1B56
:1095B000002D7FF79AAB102D7FF771AF269AC6F872
:1095C00000901027511CA5F11108E41907297760B4
:1095D000DFF848B327942691C8F3001800F34783B7
:1095E0000836103D102D7FF75DAFB8F1000F0ED09B
:1095F000013110340729C6F800907760279426912E
:1096000000F3A5830836103D102D7FF74BAF2046A1
:10961000DDF830800A9C0FE00836591C1030103DF0
:109620000729C6F8009077602691279028DC083635
:10963000103D102D40F3D3804B1C1030072BC6F883
:109640000090776027902693E6DD4046214625AAC4
:1096500003F09AF800287FF4F4A82798269B32AEEE
:10966000DBE726991398159A3060A41815984A1CC0
:10967000072A70602794269200F3D382083680E789
:109680004046214625AA03F07FF800287FF4D9A898
:1096900032AE27982699CBE70C980A99069325AA0B
:1096A00003F072F8069B00287FF4CBA832AE279C0B
:1096B0002698DFE40C980A9925AA03F065F800289B
:1096C0007FF4BFA832AE279C2698E1E40899CA0728
:1096D0003FF581AB269A37600134551C0120FFF716
:1096E000A1BB0C980A9925AA03F04EF800287FF434
:1096F000A8A8279C269D32AEFFF779BB0C980A9943
:1097000025AA03F041F800287FF49BA8279C269DFA
:1097100032AEFFF778BB099932AF0E91FEF7F6BF74
:109720000C980A9925AA03F02FF800287FF489A83D
:10973000279C32AEFFF753BA02F0E0FF002840F05A
:10974000F1800327734A0B97734F129008989DF886
:109750007330B8F1470FD8BF1746129A20F0800433
:10976000032108940E911492FEF7DBBF089B13F0BF
:10977000400300F0BB8103461098109D011D2C880A
:1097800010910025FEF789BF0898400640F1A58199
:109790001099081D0C88109001230025FEF77DBF4D
:1097A0009AF80080FEF7F0BE089BDA0640F1A68129
:1097B000109A0F981368141D10941860FEF7ADBE30
:1097C000564826990E904B1C0E986419072B86E874
:1097D0002100279426933FF7C1AE0836C8E6044619
:1097E00060E64E4B269A0993FFF763BA0C980A99E4
:1097F00025AA02F0C9FF00287FF423A8279C32AED7
:10980000FFF7A8BB269A464B501C013401210728BC
:10981000336071602794269000F3448108362DB997
:10982000119A1AB90898C0077FF55FAA2698139B6A
:10983000159933606218431C1599072B71602792A4
:10984000269300F3BC8208366D42002D40F37D81E3
:10985000102D40F3F28110240133A5F1110C1219DF
:10986000072BC6F800907460DFF8B0B027922693FB
:10987000CCF3001800F319830836103D102D40F387
:10988000DE81B8F1000F0ED001331032072BC6F87D
:10989000009074602792269300F313830836103DDE
:1098A000102D40F3CC813046DDF830802E460A9DE5
:1098B00010E0083001331032103E072BC0F8009042
:1098C00044602792269300F3FC800830103E102E4F
:1098D00040F39D8201331032072BC0F800904460A2
:1098E00027922693E5DD4046294625AA02F04CFF43
:1098F00000287EF4A6AF279A269B32A8DAE7089ABA
:1099000093F8018042F020020AF1010A0892FEF762
:109910003BBE00BF2C680108306801086868010878
:1099200064680108099D6B1C00F0C880B8F1670FDE
:1099300000F05782B8F1470F00F05382089B002CCB
:1099400043F480751A95C0F2598200201290B8F144
:10995000660F00F00882B8F1460F00F00482B8F1FB
:10996000650F00F05082B8F1450F00F04C82DDF831
:1099700024C002218DE802101FA820A91EAD03906B
:109980005A462346029504910C98CDF818C000F071
:109990007FFCB8F1670F0746DDF818C002D0B8F1B8
:1099A000470F03D1089AD00740F19782B8F1460FCC
:1099B00007EB0C0500F0EA815846214600220023FF
:1099C000FEF792FAE8B9209CA54240F2E7822346CE
:1099D000302103F8011BE243A818AB42209300F0AA
:1099E00001020DD022B10133AB426170209307D048
:1099F0001C4604F8011B5970631CAB422093F7D13D
:109A00001D46ED1BB8F1670F119500F05D81B8F1AF
:109A1000470F00F05981B8F1660F40F0BA821E9AE4
:109A2000002A40F38D82099B002B40F05882089C4D
:109A3000E30700F1548222EAE2710B910E92149234
:109A4000129C002C00F03A811A982D2100248DF8E8
:109A5000731008901294FEF765BE0E9B109523EAD2
:109A6000E3720B929DF873301494FEF75ABE0C9873
:109A70000A9925AA02F088FE00287EF4E2AE279C0F
:109A800032AEFFF77CBA40210C9801F037FD0A99FD
:109A900008600861002800F075820A9A4026566125
:109AA000FEF72DBD0C980A9925AA02F06DFE00283C
:109AB0007EF4C7AE1E9D279C32AEB0E606270997FE
:109AC0003CE74046294625AA02F05EFE00287EF4C7
:109AD000B8AE32A8279A269BF8E6109A1768131D8D
:109AE00010933C4600250123FEF7D7BD10990A6864
:109AF0000F1D144600251097FEF7CFBD089A530698
:109B000040F1D480109A0F991468101D1090218094
:109B1000FEF703BD0C46FFF707BBFEF7A3FC20EAE8
:109B2000E0710E9012940B919DF87330109514947F
:109B3000FEF7F7BD0C980A9925AA02F025FE002829
:109B40007EF47FAE279A269B32AE11993760541867
:109B50005A1C072A7160279426927FF7C5A8FFF741
:109B600073B9A3482799269A1A90FFF707B80446B5
:109B700029E60C980A9925AA02F006FE00287EF430
:109B800060AE32AE279C269D3AE40C980A9925AA2D
:109B900002F0FAFD00287EF454AE32AE279C269DDA
:109BA00041E40C980A9925AA02F0EEFD00287EF403
:109BB00048AE32AE279C2699FFF7A3BB0C980A99B2
:109BC00025AA02F0E1FD00287EF43BAE279C32AED0
:109BD000FFF778BB0C980A9925AA02F0D5FD00285A
:109BE0007EF42FAE32AE279C2699FFF7E4B90C988D
:109BF0000A9925AA02F0C8FD00287EF422AE32AEF2
:109C0000279C2699FFF7E9B90C980A9925AA02F032
:109C1000BBFD00287EF415AE32AE279C2699FFF7D7
:109C200083BB0C980A9925AA02F0AEFD00287EF4A9
:109C300008AE1E9B279C32AEA3E4DFF8BCB1013313
:109C40005219072BC6F800B07560279226933FF78C
:109C500071AF083679E7099F1095062F28BF0627B0
:109C600027EAE7740E970B94624FFEF7D9BE0C9863
:109C70000A9925AA02F088FD00287EF4E2AD32AEF2
:109C8000279C2699ADE40C980A9925AA02F07CFD40
:109C900000287EF4D6AD1E9E119B279C991B32AEE8
:109CA00083E42699DFF84881FFF7FCB810980F9BF2
:109CB0000168041D10940B60FEF72FBC1A9A9DF8E2
:109CC00073300892FEF72DBD1E9AD11C104602DBA0
:109CD000099B934228DAA8F10208431E002B1E9329
:109CE0008DF88480C0F21C812B228DF88520092BF1
:109CF00000F39E80303330218DF886108DF8873048
:109D000022AC21AA1198119BA11A4418012B199178
:109D10000E9440F30A810E9B5A1C22EAE271002045
:109D20000E920B9114908BE6119CA24272DB089C60
:109D3000E00700F1ED8022EAE2710B910E924FF004
:109D400067087CE62D238DF87330FEF7C6BD0C98AE
:109D50000A9925AA02F018FD00287EF472AD32AEF1
:109D6000279C26994FE4099D032700971EA81FA949
:109D700020AF23460195029004975A4603910C9810
:109D800000F086FA099B0746C5189C463A78302AA7
:109D900000F0AD801E982D180EE6174926980991FF
:109DA000FFF7B4B9099B099A129023EAE3740B9464
:109DB0009DF8733010950E921490FEF7B2BC0C987B
:109DC0000A9925AA02F0E0FC00287EF43AAD1E9D17
:109DD000279A269B32AE37E50022A2460992FEF76B
:109DE000D5BB0998002808BF01200990A6E500BF4F
:109DF000786801085C680108686801082D2104F191
:109E000000441291A3E5099F07F1010CB1E5354625
:109E1000064614E7002A1199D4BFC2F102000120BE
:109E2000401820EAE0730E900B934FF0670806E6A7
:109E300046F267640DF19201C6F2666484FB032565
:109E4000D817C0EBA50000EB80050A46A3EB45033D
:109E500003F130011170511E09280346EEDC303346
:109E60000DF19305D8B28D4202F8010C40F29380B7
:109E7000AC1AE4070DF1850113460DD513468DF894
:109E800086000DF1860113F8010B05E013F8011BA4
:109E9000617013F8010B611C4C1CAB424870F5D18A
:109EA00042ABC2EB4304F63C2BE70C980A9925AA77
:109EB00002F06AFC00287EF4C4AC32AE279A269BDE
:109EC000DBE40C980A9925AA02F05EFC00287EF4D7
:109ED000B8AC32AE279A269BE1E4209D91E5099823
:109EE000431CD41824EAE4710E940B91A7E558465C
:109EF000214600220023CDF818C0FDF7F5FFDDF85C
:109F000018C000287FF446AFCCF101001E9042E754
:109F1000501C20EAE0730E900B934FF067088EE51B
:109F20002D245B428DF88540E1E6089A12F001018C
:109F30007FF4F1AE0E98149120EAE0740B947FE563
:109F40000999C1B90898C40715D401230B930E933E
:109F500075E5109B9AF801801A68109B0992099A7E
:109F60000433002A1093A246BEF60EAB4FF0FF3327
:109F70000993FEF709BB099CA11C21EAE1700E912F
:109F80000B905CE50C9A0C2111604FF0FF30FEF74E
:109F900062BC1E98A1E60DF18604B2E6254630E5C6
:109FA0002DE9F04F03690C699C4283B0064600F32B
:109FB0006B81E01C82008F18B5187B6868685A1C9A
:109FC000B0FBF2F501F114030193013C043706F1F3
:109FD0001408002D00F0BE804A69D8F80030DDF882
:109FE000049090B24FEA124C05FB00F005FB0CF216
:109FF00002EB104C1FFA8CFE9AB280B2121ACEEB12
:10A00000134303EB224E92B2C9EB070006F118038B
:10A0100042EA0E4901F11802974243F8049CC0F34A
:10A0200080004FEA1C4C4FEA2E4E70D328B31068C4
:10A030001B6882B2000C05FB02CC05FB00F000EBB4
:10A040001C401EFA83F21FFA8CFC1FFA80FECCEB38
:10A050000202CEEB134303EB224E1FFA82FC06F101
:10A060001C0301F11C024CEA0E4C974243F804CC4D
:10A070004FEA2E4E4FEA104C49D31046D3F80090C9
:10A0800050F804BB1FFA8BFA4FEA1B4B05FB0ACCB6
:10A0900005FB0BFA0AEB1C4B1FFA8BFA1EFA89FE22
:10A0A0001FFA8CFCCCEB0E0ECAEB194C0CEB2E4AB3
:10A0B00099461FFA8EFE4EEA0A4C49F804CB5268C4
:10A0C0005B681FFA82FE05FB0EFE4FEA124C0EEB98
:10A0D0001B4B05FB0CF202EB1B4C9AB21FFA8CFED9
:10A0E00002EB2A421FFA8BFBCBEB0202CEEB1343AF
:10A0F00003EB224E92B24B4642EA0E49021D9742B2
:10A1000043F8049B4FEA1C4C4FEA2E4EB5D2201D5B
:10A1100006EB80035A68EAB9181D984519D250F821
:10A12000042CB2B9043BC8EB0300C21C50070DD588
:10A13000013C98450DD21A68043B3AB109E0186811
:10A14000043B30B91A68013C043B12B9013C984504
:10A15000F5D33461304602F03DF90028C0F2838027
:10A16000019AD8F8003052F8040B1FFA83F981B233
:10A17000000CC1EB0901C0EB1343DDF8049003EBC5
:10A180002140434689B241EA0041C9EB070C013541
:10A190000014974243F8041BCCF380014BD3B9B1B0
:10A1A00052F804EB19681FFA8EF91FFA81FAC9EB0D
:10A1B0000A094FEA1E4C4844CCEB114101EB204107
:10A1C00080B240EA014043F8040B0814974232D3AE
:10A1D00082461146D3F800E051F8040B1FFA8EFBBB
:10A1E0001FFA80F94FEA104CC9EB0B0B0BEB0A007E
:10A1F000CCEB1E4A0AEB20499E4680B240EA094059
:10A200004EF8040B50685B6882B21FFA83FC000CA6
:10A21000C2EB0C0202EB2942C0EB134303EB2240DA
:10A2200092B242EA004A73460A1D974243F804ABD1
:10A230004FEA204ACDD2211D06EB8103586890B920
:10A240001A1D98450ED252F8041C59B9043BC8EBAC
:10A250000300C21C520713D5013C984502D218686E
:10A26000043B68B13461284603B0BDE8F08F1A683A
:10A27000043B002AF6D11968013C043B0029F1D1C6
:10A28000013C9845F3D3EDE70020EDE70000000026
:10A290002DE9F04F016C9FB081462B9C92469B4666
:10A2A00051B1436C012202FA03F24B608A6001F063
:10A2B0003FFD0020C9F84000BBF1000839DB002158
:10A2C000216000242246C7F6F074C7F6F07208EA4F
:10A2D0000400904216D00022002350465946FDF754
:10A2E00003FE00282BD02A9D2C9C01202860002CE6
:10A2F00000F0CF80A2494B1E2160059305981FB046
:10A30000BDE8F08F2A9C42F20F722260BAF1000F72
:10A3100000F0A6809B4D05952C9C002CEED0059D51
:10A32000EB78002B00F00B82284608302C9C206034
:10A33000E4E728F0004801232360C346C1E71DAECF
:10A340001CAF52460096019748465B4602F076F9EC
:10A35000C8F30A520C90002A40F08C801C9F1D9973
:10A360006FF482637E189E42C0F234834FF60E452E
:10A37000CFF6FF75A91B06F2124208FA01F32AFA7A
:10A3800002F01843FDF7D2FA0124013EA1F1F87161
:10A390000D9400230022C3F6F873FDF789F972A328
:10A3A000D3E90023FDF738FB71A3D3E90023FDF7C0
:10A3B00081F9044630460D46FDF7C8FA6EA3D3E98D
:10A3C0000023FDF729FB02460B4620462946FDF7F0
:10A3D00071F904460D46FDF7B9FD294609900022A2
:10A3E00020460023FDF78AFD002840F0C682099828
:10A3F000162800F2BF82644C04EBC005D5E90001C9
:10A4000052465B46FDF798FD002800F0EB82099963
:10A4100000204B1E09931290BE1B013E00F1C48226
:10A4200000240A960E9409990029C0F2B4820A9D6C
:10A4300011916B1800210A931091289809282BD8A4
:10A44000052841F34C80021F28920025289CA31E5A
:10A45000032B23D8DFE813F043052F0549034005FC
:10A4600048484A49C8F31308B8F1000F18BF01461D
:10A47000059151E72BF07F4727F4700444F07F5596
:10A48000A2F2FF360022504645F440111C9F0D9267
:10A490007FE73F4D059531E7002528950024C9F851
:10A4A00044404846214601F01DFC4FF0FF33059023
:10A4B000C9F8400001200B93139329940F901D9924
:10A4C0000029C0F23F81099A0E2A00F33B812E4DEC
:10A4D000299B05EBC20090ED007B002B8DED067BE8
:10A4E000C0F20085DDE9062350465946FDF7BEFB64
:10A4F000FDF72CFD0646FDF729FADDE90623FDF7F9
:10A500008BFA02460B4650465946FDF7D1F80B9B95
:10A51000DDF8148006F13002012B04460D4608F8E0
:10A52000012B00F0918000230022C4F22403FDF7E8
:10A5300073FA0022002304460D46FDF7D5FC0028DF
:10A5400040F0C080059F059E0B98023706EB000B7C
:10A55000C7EB0B01C90700F1C780CDF820B0DDE9DA
:10A5600006AB4BE0AFF3008061436F63A787D23F38
:10A57000B3C8608B288AC63FFB799F501344D33FF2
:10A580006568010894680108B068010888680108D6
:10A5900064680108FDF740FA0022002304460D46D6
:10A5A000FDF7A2FC52465B46002840F08B80204617
:10A5B0002946FDF75BFBFDF7C9FC0646FDF7C6F92A
:10A5C00052465B46FDF728FA02460B4620462946CE
:10A5D000FDF76EF8303600230022C4F2240307F89A
:10A5E000016CFDF719FA00220023B84604460D4617
:10A5F00007F10107FDF778FC002863D152465B465E
:10A6000020462946FDF732FBFDF7A0FC0646FDF784
:10A610009DF952465B46FDF7FFF902460B46204680
:10A620002946FDF745F8DDF820C0002306F1300883
:10A630000022674507F8018C0446B8460D46C4F26F
:10A64000240307F10107A5D122462B4620462946BF
:10A65000FDF730F804460D462246DDE906012B469B
:10A66000FDF74CFC40B9DDE9060122462B46FDF71B
:10A670003BFC38B3F40725D518F801BC059AD34341
:10A6800008EB0300C00700F104851446BBF1390F45
:10A6900008F1FF3112D18C4200F03E8511F801BC67
:10A6A000BBF1390F884601F1FF3107D111F801BC28
:10A6B0008846BBF1390F08F1FF31ECD00BF10105F1
:10A6C000EAB20A7048460C9901F032FB099D2C9CB5
:10A6D0006B1C2A9D002288F800202B60002C3FF480
:10A6E0000DAEC4F8008009E6DDE9062320462946C0
:10A6F000FDF7BCFAFDF72AFC0646FDF727F9DDE970
:10A700000623FDF789F902460B4620462946FCF749
:10A71000CFFF303600230022C4F2240307F8016C77
:10A72000FDF77AF9B846059F0022002304460D463E
:10A730000337FDF7D9FB00283FF40FAFC2E7059AB6
:10A74000D01CF3E50F9F002F00F03381289C012CD3
:10A7500040F3F8830B98109A411E8A42C0F2E784B6
:10A76000551A0B980028C0F237860E9C0B9F0E9B43
:10A77000DDF828E0DA190EEB0708484601210E92B1
:10A78000CDF8288001F0A6FB0D907CB10A98002836
:10A790000CDDDDF838C00746A742A8BF2746C7EB47
:10A7A0000C0EC11BCDF838E0E41B0A91109B002B66
:10A7B0001ADD0F9A002A00F0A784002D10DD0D99F4
:10A7C0002A46484601F0F8FC0D900D990C9A48462F
:10A7D00001F08AFB0C990646484601F0A9FA0C964E
:10A7E0001098421B40F0A8830121484601F072FBFB
:10A7F000119D002D074605DD394648462A4601F0E1
:10A80000DBFC07462899012940F356810025119861
:10A81000002840F0168401210A98091811F01F033E
:10A8200000F0CC80C3F12002042A40F35B86DDF8FF
:10A8300038E00A9AC3F11C000EEB00081118CDF89D
:10A84000388024180A910E9B002B05DD48460C9990
:10A850000E9A01F0FBFC0C900A9A002A04DD39469E
:10A86000484601F0F3FC07461298002840F0CE83DA
:10A870000B98002840F3EF830F99002940F0B48033
:10A880000B9C0F9DE20740F19F83A2460C9EDDF8D2
:10A89000148010E001F056FA39460646FFF780FBB7
:10A8A000303008F80400314648460A22002301F0FF
:10A8B00049FA651C064639463046FFF771FB6C1CA9
:10A8C00000F1300B0A220023A2453146484608F821
:10A8D00005B0DFDC0C96DDF814800B9A0025012A08
:10A8E000ACBF904408F1010801220C99484601F0E0
:10A8F000ADFC39460C9001F06DFD002840F3498411
:10A9000018F8012C0599C84308EB0003DB0707D5AD
:10A91000392A08F1FF3418D114F8012C0599A04602
:10A92000392A08F1FF3410D1A14200F0688314F8ED
:10A93000012C392AA04604F1FF3406D114F8012C69
:10A94000A046392A08F1FF34EED001322270484681
:10A95000394601F0EDF90D9A002A3FF4B3AE002D0F
:10A9600000F0E482954200F0E1824846294601F079
:10A97000DFF9DBE2012212924EE50998FCF7E6FFCF
:10A9800022462B46FDF7B0FA00287FF430AD099936
:10A990004B1E09932BE50E9D099B0024E81A5A4291
:10A9A0000E901092119448E5764200220E960A927B
:10A9B00039E50F9B109D0E9C0D93E6E61C200E9929
:10A9C000DDF828800B1808EB000C0E932418CDF846
:10A9D00028C038E74FF6EE30CFF6FF70841B0AFA36
:10A9E00004F0CFE4129017E5002C05DD48460D99E0
:10A9F000224601F02BFC0D90002D40F002840D9EAC
:10AA0000059D0B99059A6B180AF001000D9DDDF864
:10AA100030A00A93541C0B9039465046FFF7C0FAF9
:10AA200029468046504601F0D5FC394632468346D9
:10AA3000484601F0FDFCC368611E0246089108F11A
:10AA4000300C002B00F0878248461146CDF80CC030
:10AA500001F06EF9DDF80CC00120BBF1000FC0F26F
:10AA6000788305D1289A1AB90B99002900F07183CF
:10AA7000002800F3DE830A9804F801CC8442A04643
:10AA800000F0E68351460A220023484601F05AF9B5
:10AA9000B542824600F08E8229460A2200234846AB
:10AAA00001F050F9314605460A224846002301F0DC
:10AAB00049F901340646AFE7BAF1000F7FF4A6AEBC
:10AAC000CBF313025B46002A40F094840025C7F6BE
:10AAD000F0751D40002D3FF49AAE0E980A9B411C64
:10AAE0005A1C0E910A92012591E601210F91299B92
:10AAF000002B40F329831C4613930B930021172C42
:10AB0000C9F844100AD9012204235B0003F11400A0
:10AB100011460132A042F8D9C9F84410484601F064
:10AB2000E1F80E2C0590C9F840003FF6C8AC002DA6
:10AB30003FF4C5AC099F002FCDE914AB40F33D8332
:10AB4000994807F00F0600EBC6013E11D1E9004518
:10AB5000F10640F1F582954F50465946D7E9082352
:10AB6000FDF784F806F00F0682468B46032786B170
:10AB7000DFF8388220462946F20704D5D8E90023B9
:10AB8000FCF74AFF0137761008F10808F4D10446B3
:10AB90000D465046594622462B46FDF767F8824639
:10ABA0008B46129B53B10023504659460022C3F6F0
:10ABB000F073FDF7A3F9002840F024843846FCF731
:10ABC000C5FE52465B46FCF727FF00230022C4F275
:10ABD0001C03FCF76FFD04460B98A1F1507500288B
:10ABE00000F07582099E1B960B9E0F99002900F0BC
:10ABF00038836D4A002102EBC60353E9022300208B
:10AC0000C3F6E071FDF732F82B462246FCF750FD03
:10AC1000CDE9180159465046FDF798F90546FCF76D
:10AC200095FE02460B4650465946FCF741FD30352D
:10AC3000DDF81480CDE916015FFA85FB08F801BB49
:10AC4000DDE91801DDE91623FDF776F9002840F06B
:10AC50001D840021DDE916230020C3F6F071FCF706
:10AC600027FD02460B46DDE91801FDF765F90028CE
:10AC700040F03184012E40F39C8205996FEA080769
:10AC80008E19BC19002304F001050022C4F224032C
:10AC9000DDE918011A961895FCF7BEFE0023002284
:10ACA000C4F2240304460D46DDE91601FCF7B4FEA8
:10ACB0000F460646FDF74AF98346FCF747FE024673
:10ACC0000B4630463946FCF7F3FCC2460BF1300226
:10ACD0005FFA82FB0AF801BB22462B4606460F4666
:10ACE000D046FDF70BF9002840F0E2800021324603
:10ACF0003B460020C3F6F071FCF7DAFC22462B46F7
:10AD0000FDF7FCF8002840F0C783DDF868E0F24565
:10AD100000F04F821898002841D000230022C4F28E
:10AD2000240320462946FCF777FE00230022C4F2C4
:10AD3000240304460D4630463946FCF76DFE0F46A7
:10AD40000646FDF703F98046FCF700FE02460B4677
:10AD500030463946FCF7ACFC08F130035FFA83FB60
:10AD60000AF801BB22462B4606460F46D046FDF7A1
:10AD7000C5F8002840F09C80002132463B46002068
:10AD8000C3F6F071FCF794FC22462B46FDF7B6F8AB
:10AD9000002840F081831A998A4500F00A82CDF894
:10ADA0005890DDF8689050E0B068010878690108B3
:10ADB00000210020C3F6F071FCF77AFC22462B46F6
:10ADC000FDF79CF800230022C4F22403002840F081
:10ADD000618320462946FCF71FFE00230022C4F2AF
:10ADE000240304460D4630463946FCF715FE0F464F
:10ADF0000646FDF7ABF88046FCF7A8FD02460B4679
:10AE000030463946FCF754FC08F130035FFA83FB07
:10AE10000AF801BB22462B4606460F46FDF76EF8A0
:10AE2000D04632463B46002840D100210020C3F6E0
:10AE3000F071FCF73DFC22462B46FDF75FF8002839
:10AE400040F02883CA4500F0B281002320462946FD
:10AE50000022C4F22403FCF7DFFD00230022C4F229
:10AE6000240304460D4630463946FCF7D5FD0F460F
:10AE70000646FDF76BF88346FCF768FD02460B4675
:10AE800030463946FCF714FCD0460BF130025FFA2D
:10AE900082FB08F801BB22462B4606460F46FDF70B
:10AEA0002DF8C24632463B46002881D0DDF8589046
:10AEB0001B99099106E400200F90DDF8A4E00998A1
:10AEC0000EEB0002541C002C13920B943FF716AEAD
:10AED0000021C9F8441021E601210F91EDE700227D
:10AEE0000F9204E60B9900293FF7FCAA40F0EE828E
:10AEF00000230022C4F21403DDE90601FCF78CFDF7
:10AF000052465B46FDF70EF80B9F0D97002800F0A8
:10AF1000B7802998DDF81480C14309914846394625
:10AF200000F006FF0D9C002C3FF4CCAB48460D9979
:10AF300000F0FEFEFFF7C6BB48460C9901F03CF955
:10AF40000C9051E40D9A002A00F04D8201F2334733
:10AF5000109D0E9C0BE411465046CDF80CC0049297
:10AF600001F038FA049A034611464846049300F06B
:10AF7000DFFE0498DDF80CC000287FF46EAD289940
:10AF800000297FF46AAD0B9B002B7FF466ADBCF10A
:10AF9000390FCDF830A0DA46E34600F0F280BAF17E
:10AFA000000F01DD08F1310BDDF820800D9608F867
:10AFB00001BBCCE4294648460A22002300F0C2FE29
:10AFC00001340546064627E50C983946FEF7E8FFAA
:10AFD00000F1300B0B98059B0125A84283F800B0C7
:10AFE0007FF779AC48460C990F9B0A2200F0AAFE25
:10AFF000DDF82CA00C900646DDF814805BE409987F
:10B00000059C431C312109932170A0E40C9839461A
:10B0100001F0E0F90028BFF62BAC0A2248460C9953
:10B02000002300F08FFEDDF824C00F9A0C900CF185
:10B03000FF3ECDF824E0002A40F03D8213990B91A9
:10B0400016E43B6907EB8302106900F0F7FEC0F1DC
:10B050002001FFF7E1BB289A022A7FF70DAC0028F8
:10B060007FF457AF394605220B9B484600F06AFE35
:10B07000074639460C9801F0ADF900287FF749AF33
:10B08000099ADDF814803125531C08F8015B0993F7
:10B0900044E7BBF1390F08F1FF317FF40FAB11F832
:10B0A00001BC059C8846FFF7F1BA3846FCF74EFC18
:10B0B00002460B4650465946FCF7AEFC00230022E0
:10B0C000C4F21C03FCF7F6FA0446A1F15075002304
:10B0D0000022C4F2140350465946FCF7E9FA22460E
:10B0E0002B4682468B46FCF727FF0746002840F098
:10B0F000B580224605F1004350465946FCF7FEFE56
:10B10000002856D00D9704E748460C99109A01F094
:10B1100053F80C90FFF768BB059C099B3021217008
:10B120002146581C312209900A70FFF7CBBA109FB4
:10B13000119B1091CD1B5C1911940025FFF711BBD9
:10B14000DDE914AB022712E5012413940B94299432
:10B15000BEE60028E346CDF830A064467FF724AF72
:10B1600001220C99484601F071F839460C9001F023
:10B1700031F9002840F39881392C08F1310B7FF424
:10B1800013AFDDF820800D96392208F8012BFFF768
:10B19000B9BB03D11BF0010F7FF4B2AB4346984615
:10B1A000013B18F8012C302AF9D0FFF7D0BBDDF8AD
:10B1B0005890DDE914ABFFF782B9099D6C42002C71
:10B1C00000F01B81B64B04F00F0103EBC102D2E982
:10B1D0000023DDE91401FCF71FFC241182468B4695
:10B1E00000F07681AF4D0227E30704D5D5E90023AF
:10B1F000FCF712FC013708356410F5D182468B4606
:10B20000CFE40D994846496800F06CFD0D9D2B690F
:10B2100004462946981C82000C3104F10C0000F011
:10B22000BBFC48462146012201F010F80646FFF714
:10B23000E7BBBCF1390FE346CDF830A0A1D0DDF873
:10B2400020800D960CF1010E08F801EBFFF77FBB93
:10B25000E346CDF830A00D96FFF746BB00270D97CB
:10B260000EE78F4B06F1FF3803EBC80022462B4652
:10B27000D0E90001CDF86880FCF7CEFBCDE91601DE
:10B2800059465046FCF762FE0446FCF75FFB024657
:10B290000B4650465946FCF70BFADDF81480303463
:10B2A000012E82468B4608F8014B00F08180059FF5
:10B2B00000237D1E05EB060A0022C4F22403CDF80C
:10B2C0000CA0FCF7A9FBFE4306EB0A040F4606465A
:10B2D000FCF73CFE04F001050446FCF737FB024690
:10B2E0000B4630463946FCF7E3F9DDF814C030343C
:10B2F0008CF80140DDF80CC0E04582468B4647469D
:10B3000054D0F5B100230022C4F22403CDF80CC0C0
:10B31000FCF782FB8B468246FCF718FE0546FCF7DD
:10B3200015FB474602460B46504659463035FCF75A
:10B33000BFF907F8015FDDF80CC0674582468B4610
:10B3400034D050465946664600230022C4F22403F6
:10B35000FCF762FB0D460446FCF7F8FD8246FCF75D
:10B36000F5FA02460B4620462946FCF7A1F90AF1F8
:10B37000300400230022C4F2240307F8014FFCF735
:10B380004BFB0D460446FCF7E1FD8346FCF7DEFA75
:10B3900002460B4620462946FCF78AF90BF130029B
:10B3A00007F8012FB742CFD182468B461A998844BD
:10B3B00000230022C3F6E073DDE91601FCF77AF9F9
:10B3C00052465B46FCF79AFD002848D01B9C18F8B3
:10B3D00001BC0994FFF752B9DDF838C00027C0EB73
:10B3E0000C04FFF7C4B91C99109D0E9CC1F13607DF
:10B3F000FFF7BDB95546FFF70ABADDE914AB0227DE
:10B40000FFF7CFBB0B9D002D3FF44FAE139A002AE0
:10B410007FF7CFAE00230022C4F2240350465946E2
:10B42000FCF7FAFA8246781C8B46FCF78FFA024644
:10B430000B4650465946FCF7EFFA00230022C4F2AF
:10B440001C03FCF737F9DDF824C0139E0CF1FF3E16
:10B450000446CDF86CE0A1F15075FFF7C6BB0021A2
:10B46000DDE916230020C3F6E071FCF721F952460E
:10B470005B46FCF761FD00283FF49BAE43469846CF
:10B4800003F1FF3318F8010C3028F8D01B9C099405
:10B49000FFF718B9DDF858901B980990FFF7EEB840
:10B4A000B0680108786901087FF47EAD1BF0010FD8
:10B4B0003FF47AAD60E6002348460D990A2200F079
:10B4C00041FC139B0D900B93FFF7D2B9002719E6AF
:10B4D0000227FFF766BB1B9A0992FFF7CFB8012539
:10B4E000FEF7B4BF3FF4AFA9C3F13C00FFF767BA62
:10B4F00040F26C70C2F20000704700BF2DE9F04FBF
:10B5000001F10B05162D83B0064627D935F0070546
:10B5100027D4A94225D8304600F0E0FBB5F5FC7FE2
:10B5200023D2BA4F4FEAD50C07EBCC02D468944231
:10B5300000F0DE816368E268A16823F0030023184D
:10B54000CA605868916040F001025A60304600F0CD
:10B55000C7FB0834204603B0BDE8F08F1025A94290
:10B56000D9D90C2434600024F4E75FEA552C00F0AC
:10B570008B80BCF1040F00F255814FEA951707F15B
:10B58000380E4FEA4E01A14F07EB8101CC68A14272
:10B5900005D10CE0002A7CDAE468A14207D0636898
:10B5A00023F00300421B0F2AF4DD0EF1FF3E0EF1E3
:10B5B000010C964B3C6903F1080E744500F075814F
:10B5C000616821F003014A1B0F2A00F35B81002A06
:10B5D000C3F814E0C3F810E069DAB1F5007F80F039
:10B5E0002F81CA0803EBC2014FF00109921009FA3A
:10B5F00002F95A688868E16049EA0209A060C3F864
:10B6000004908C60C46001204FEAAC0400FA04F09E
:10B61000484556D819EA000F07D12CF0030C40001A
:10B6200019EA000F0CF1040CF9D007EBCC094C46D9
:10B63000E046E3689C4207D13AE1002A80F2628149
:10B64000DB689C4200F03481596821F003014A1BF9
:10B650000F2AF2DD1C465919D86854F808CF8A50D1
:10B6600045F0010542F00102CCF80C00C0F808C01A
:10B670005D6079613961C1F80CE0C1F808E04A60A9
:10B68000304600F02DFB65E74FEAD50E4FEA4E013C
:10B6900079E72218E3685068A16840F00100506023
:10B6A000CB609960304600F01BFB083452E761180C
:10B6B00030464B6843F001024A6000F011FB083449
:10B6C00048E7BC68606820F00309A94504D3C5EBCE
:10B6D00009030F2B00F38D804D4A4E4B11681868FB
:10B6E000013104EB090B05EB000300F05A8103F56F
:10B6F00080500F3020F47F6121F00F0C61463046FE
:10B700008DE8041001F02EF8B0F1FF3F80469DE86F
:10B71000041000F05281834500F20F81DFF800A190
:10B72000DAF80030C3456344CAF8003000F04A81BB
:10B730001268013200F05781CBEB080B5B44CAF86A
:10B74000003018F0070100F00B81C1F10800C1F5CD
:10B750008053804403F1080208EB0C010805030D37
:10B76000C3EB020B3046594600F0FCFF431C00F0CF
:10B770004681C8EB00020BEB020141F00100DAF850
:10B780000030C7F808805B44BC42CAF80030C8F8F3
:10B79000040015D0B9F10F0F40F2F2806168A9F1F1
:10B7A0000C0222F00702A01801F0010C42EA0C0E74
:10B7B00005210F2AC4F804E04160816000F217817E
:10B7C000154ABC681068834288BF1360134A116829
:10B7D0008B4288BF1360636823F00300A842C5EB67
:10B7E000000301D30F2B04DC304600F079FA00246B
:10B7F000B0E6621943F0010145F00105656030468D
:10B800005160BA6000F06CFA0834A3E6A407002087
:10B81000B00B0020D40B0020D00B0020CC0B00205C
:10B82000D80B0020BCF1140F7BD9BCF1540F00F2EF
:10B830008D804FEA153404F16E0E4FEA4E01A2E6F8
:10B84000480A042872D9142800F2AE8000F15B097E
:10B850004FEA490207EB8200DFF8F08183688342F8
:10B8600000F081805A6822F00302914202D29B6864
:10B870009842F7D1DA68D7F80490E260A360DC6000
:10B880009460C0E6611942F0010045F00105656071
:10B89000596119614860C1F80CE0C1F808E08A50AC
:10B8A000304600F01DFA083454E6D3F80490AAE6B6
:10B8B00008F10108083418F0030F7FF4BAAE4946C6
:10B8C0001CF0030FA1F108040CF1FF3C00F0B08064
:10B8D0000968A142F4D07C684000A0423FF6F1AE76
:10B8E00000283FF4EEAE044200F0A780C4469CE678
:10B8F00004F108036469A34208BF0CF1020C3FF491
:10B9000058AE17E659181C464868DB6854F8082FEB
:10B9100040F001004860D3609A60304600F0E0F9E2
:10B9200018E60CF15B0E4FEA4E012CE64FEA911837
:10B9300008F138094FEA49028CE7BC423FF4EEAE09
:10B94000424CA468626822F0030047E7BCF5AA7F76
:10B950001CD84FEAD53202F1770E4FEA4E0112E6BB
:10B960004FF48052F8E6D8F804004FEAA90201210A
:10B9700001FA02F242EA0009C8F804901A467CE78C
:10B980000122C8F804204446002027E740F254531F
:10B990009C4524D84FEA954000F17C0E4FEA4E01B9
:10B9A000F1E503F1100CA9E654282CD84FEA113226
:10B9B00002F16E094FEA49024CE7BC68616821F068
:10B9C00003000BE74FEA0B50010D00297FF4B0AEE6
:10B9D000B8680CEB090141F001044460F0E6FC2179
:10B9E0004FF07E0ECFE51A48C0F80080A9E604F1BA
:10B9F0000801184C304600F0C3FF2368E0E6012040
:10BA00004FF0000BBBE6B0F5AA7F06D84FEAD13362
:10BA100003F177094FEA49021CE740F25453984278
:10BA20000FD84FEA914000F17C094FEA490211E733
:10BA30007C6824EA00047C604EE7400008F10408BA
:10BA400051E7FC224FF07E0904E700BFA407002065
:10BA5000B00B0020D80B00208307F0B4C9B200F06F
:10BA60009680531E002A00F0948002788A420BD000
:10BA7000421CD8071AD512F0030F10461CD01478B8
:10BA8000013B01328C4211D1F0BC7047002B7CD0BD
:10BA90001278013B8A42F7D014F0030F204604F1DC
:10BAA000010209D02478013B8C42EDD012F0030F43
:10BAB000104602F10104E9D1032B3FD9046841EAA1
:10BAC000012545EA054585EA0407A7F1013222EA86
:10BAD00007021E1F041D12F0803FC6F380072DD100
:10BAE000032E334629D967B120460434066885EA17
:10BAF0000602A2F1013626EA020212F0803F19D0B6
:10BB00001CE0261D2046246885EA0402A2F10134C7
:10BB100024EA020212F0803F10D1346885EA040260
:10BB2000A2F1013424EA0202043B341D12F0803FEA
:10BB3000304603D1043B032BE3D820465D1E23B3DC
:10BB400003788B42A0D0431C0022E80714D5184686
:10BB50000122047801338C4296D09542184603F1B5
:10BB6000010402F102020ED01B788B428CD0631CC0
:10BB7000204624788C4287D09542184603F1010470
:10BB800002F10202F0D100207EE718467CE713465E
:10BB900092E7104678E700BF0F2A2DE9F00340F244
:10BBA000958041EA00039B0740F092800C68046096
:10BBB0004D6845608E68A2F110038660CC681D4612
:10BBC0000F2DC460C3F3001601F1100400F110033F
:10BBD00022D966B126681E6066685E60A6689E60AF
:10BBE000E668103DDE60103410330F2D14D926683E
:10BBF0001E6066685E60A6689E60E668DE60266914
:10BC00001E6166695E61A6699E61E669203DDE612E
:10BC1000203420330F2DEAD8A2F1100323F00F04B3
:10BC200002F00F031034032B00EB0408214451D918
:10BC3000A3F104090B464FEA990901EB890C53F86B
:10BC4000046BC1EB0C0544460CF1040C634544F84D
:10BC5000046BC5F3800512D02DB153F8045B634526
:10BC600044F8045B0BD01E46254656F8047B45F885
:10BC7000047B5F68331D67602C1D6345F3D109F1B8
:10BC800001039C00091902F003024444DAB123467F
:10BC90000D7803F8015BA218E4431419934204F0F1
:10BCA000010410D02CB111F8014F03F8014B93425D
:10BCB00009D04D781C4604F8015B8D785D70631CDB
:10BCC00002319342F5D1BDE8F00370470446DDE749
:10BCD0000446DCE744461A46D8E700BF704700BF79
:10BCE000704700BFC36C70B505460C464BB153F8A6
:10BCF000240080B1016843F8241000230361C3606D
:10BD000070BD0421212200F0BFFD0346E864002835
:10BD1000EDD1002070BD012101FA04F6721D284604
:10BD2000920000F0B1FD0028F3D044608660E4E7A3
:10BD300031B1C36C4A6853F82200086043F82210FE
:10BD4000704700BF2DE9F0410E46496937698CB252
:10BD50000D0C02FB043302FB05F101EB134506F168
:10BD600018049BB203EB054344F8043C0123791EFD
:10BD70002D0C9F42804601F0010039DD98B1246806
:10BD8000A3B2210C02FB035502FB01F1ABB201EBA4
:10BD9000154003EB004106F11C040223050C9F42F1
:10BDA00044F8041C24DD206881B2000C02FB015120
:10BDB00002FB00F0254600EB114089B201EB004187
:10BDC00045F8041B64681FFA84FC210C02FB0CFC80
:10BDD0000CEB104002FB01F101EB10412C46023349
:10BDE00085B205EB01400D0C9F4244F8040BDADCF0
:10BDF0003DB1B268974207DA06EB87020137556119
:10BE000037613046BDE8F08173684046591CFFF742
:10BE100069FF31698A1C044606F10C0100F10C002F
:10BE20009200FFF7B9FE7068D8F84C3053F8201034
:10BE3000316043F820602646DEE700BF020C03466F
:10BE400016D10304102013F07F4F01D108301B02DC
:10BE500013F0704F01D104301B0113F0404F01D19A
:10BE600002309B00002B02DB5B0003D420207047D4
:10BE70000020E8E7013070470368024613F007002E
:10BE800007D0D9071FD498071FD498081060022044
:10BE9000704799B209B91B0C102013F0FF0F01D1A4
:10BEA00008301B0A190701D104301B09990701D179
:10BEB00002309B08D90704D45B0801D120207047C9
:10BEC000013013607047002070475908116001204D
:10BED000704700BF10B50C460121FFF703FF012298
:10BEE0004461026110BD00BF2DE9F04F0C69176974
:10BEF000BC4285B00E46904604DA224646463C4691
:10BF000088461746B3687168E2199A42C8BF013182
:10BF10000192FFF7E7FE0199039000EB81031433D0
:10BF20001430984202931AD20299039BC2438A1892
:10BF300002991833002599420560C2F380000ED99A
:10BF400028B11D60039B029A1C339A4207D90298BC
:10BF5000194641F8045B5D600B1D9842F8D808EB68
:10BF60008703143306EB840408F1140714349F424A
:10BF7000009306F1140C80F0F8800398183057F8FD
:10BF8000043B9AB2002A6ED0614650F8045C51F826
:10BF9000046BABB21FFA86F82D0C360C02FB08338B
:10BFA00002FB065606EB13466FEA0C059BB243EA0A
:10BFB00006436519360C8C4240F8043CC5F38005F5
:10BFC00003464DD9CDB1DCF8045003681FFA85F95A
:10BFD0001FFA83F82D0C1B0C02FB0988464402FB58
:10BFE000053505EB16450346B6B246EA054604316B
:10BFF00043F8046B2E0C8C4232D90D46D3F800E086
:10C0000055F8049B1FFA8EFA1FFA89FB02FB0BAA54
:10C010004FEA19494FEA1E48564402FB098E0EEBBF
:10C0200016499846B6B246EA094648F8046B4E6887
:10C030005B681FFA86FA99B2360C1B0C02FB0A11D8
:10C0400001EB194102FB063606EB114689B2434665
:10C0500041EA0648291D360C8C4243F8048BCCD8A3
:10C060001E6057F8043C1A0C7AD050F8046CBCF8E7
:10C070000050310C02FB0515B3B243EA0546E14618
:10C08000034640F8046C59F8041B53F8046B090C80
:10C090001FFA86FA02FB01A16FEA0C0E04EB0E08F0
:10C0A00001EB15414C45C8F3800A05464FEA11489B
:10C0B00055D9BAF1000F1BD0BCF80450360C02FB66
:10C0C000056505EB080E89B241EA0E4643F8046C9B
:10C0D00059F8041B1D4653F8046B090C1FFA86FA25
:10C0E00002FB01A101EB1E414C454FEA114836D934
:10C0F000B9F800B0350C02FB0B5AC24489B21D4698
:10C100004E4641EA0A4143F8041C56F804EB55F840
:10C11000041BD9F804801FFA81FB4FEA1E49090C61
:10C1200002FB09BE1FFA88F80EEB1A4902FB081E33
:10C130000EEB19481FFA89F1B14641EA084645F865
:10C14000046C59F8041B5E68090CB3B202FB01339E
:10C1500003EB18412B1D4C454FEA1148C8D8296004
:10C16000009A0430BA423FF60AAF019900291ADD5D
:10C17000029B53F8040C043BA8B901994A1ED0074E
:10C1800017D553F8040D019268B9019A08E053F8E5
:10C19000041C043B31B953F8040C013A043B08B9C0
:10C1A000013AF4D1019201990398016105B0BDE80B
:10C1B000F08F0A46F4E700BF12F003032DE9F041C7
:10C1C000144680460F462BD1A4101BD0D8F84860E7
:10C1D0002EB92EE0641015D03568B5B12E46E307B0
:10C1E000F8D5394632464046FFF77EFEB7B17A6849
:10C1F000D8F84C3053F822106410396043F822709C
:10C200000746E9D13846BDE8F0813146324640461E
:10C21000FFF76AFE306005600646E0E70746D9E7AB
:10C220005D1E094A002352F82520FFF78BFD0746C3
:10C23000CAE7404640F27121FFF74CFE0646C8F8B7
:10C24000480000203060CAE7A46801082DE9F04FDB
:10C2500017460A698B687E1183B0B41801940134C3
:10C260009C420D468046496803DD5B0001319C42DB
:10C27000FBDC4046FFF736FD002E00F114011FDD08
:10C280000123721E4FF0000CB342C1F800C002EA55
:10C29000030100F1180210D031B10223B342C2F8F9
:10C2A00000C000F11C0208D01146023341F804CB53
:10C2B000C2F804C00A1DB342F6D100EB8301143169
:10C2C0002E6905EB8606143617F01F0705F1140ECC
:10C2D00000975BD0DEF8002002FA07F205F11803A0
:10C2E00041F8042B6FEA0E0953F8042C06EB090AF7
:10C2F000C7F1200E9E42CAF3800A22FA0EF931D904
:10C30000BAF1000F0FD01F68009B07FA03F749EA44
:10C31000070205F11C0341F8042B53F8047C9E42EC
:10C3200027FA0EF91ED91A68DDF800B00F4602FA96
:10C330000BFC49EA0C0947F8049B1A46D3F804A001
:10C3400052F8043B0AFA0BFC23FA0EFB4BEA0C0AE8
:10C350001346C1F804A053F8049B391D9E4229FAE4
:10C360000EF9E0D8C1F80090B9F1000F01D0019C9E
:10C370000234D8F84C306A6853F82210013C04614A
:10C38000296043F8225003B0BDE8F08F6FEA0E0336
:10C39000DEF8007005F11802F318964241F8047BAC
:10C3A000C3F38003E5D933B1136805F11C0296424B
:10C3B00041F8043BDDD994460F465CF8043B47F84E
:10C3C000043B53680CF104024B60391D9642F2D8CD
:10C3D000CFE700BFF0B40B6905460069C01A24D14D
:10C3E0001A1D94002B191E1D0919143556F8044CFA
:10C3F0000A68EF43BE199442C6F3800610D19D42ED
:10C4000013D23EB153F8044D51F8042D944207D194
:10C410009D420AD253F8044D51F8042D9442F1D0B4
:10C42000A24294BF01204FF0FF30F0BC704700BF24
:10C430002DE9F84F0F460546114638469346FFF75B
:10C44000C9FF041E00F0F180C0F2EA8000242846F3
:10C450007968FFF747FCDBF814607A69DBF8105065
:10C46000C4601FFA82FC4FEA164AB4B2C4EB0C0651
:10C470003B690BEB8505CAEB12420BF1140102EB91
:10C48000264A05F11408C943B4B20BF1180608EBAB
:10C49000010244EA0A4407EB830900F11805B0459C
:10C4A000C2F38001446109F1140907F1180C4FEA45
:10C4B0002A4A2A4652D9D9B1DCF8002036681AFA3D
:10C4C00082FE310CB4B2C4EB0E06C1EB124C0CEB85
:10C4D000264AB2B242EA0A440BF11C062C60B0456F
:10C4E00000F11C0507F11C0C4FEA2A4A2A4635D9EF
:10C4F0006246374652F8041B57F8044B1AFA81FE7D
:10C500001FFA84FB240CCBEB0E0AC4EB114101EBA8
:10C510002A441FFA8AFE29464EEA044B41F804BB1E
:10C52000DCF804C076681FFA8CFA0AEB24441FFA80
:10C5300086FB4FEA1646CBEB0404C6EB1C4E0EEB13
:10C54000244AA6B246EA0A443E1D6C600D1DB04561
:10C5500002F1040C4FEA2A4A2A46C9D8E14555D9C6
:10C5600062466FEA0C0452F8041B1AFA81FE4FEA85
:10C57000114808EB2E481FFA8EFA294609EB0406EB
:10C5800091454AEA084441F8044BC6F380064FEA55
:10C59000284833D986B152F8044B18FA84FE260C89
:10C5A00006EB2E461FFA8EF848EA0644914541F8FC
:10C5B000044B4FEA264821D917460E4657F8044B3C
:10C5C00018FA84FE240C04EB2E441FFA8EF848EA75
:10C5D000044E46F804EB52681FFA82F808EB244434
:10C5E0004FEA124202EB244EA4B244EA0E443A1D32
:10C5F0004C60311D91454FEA2E48DDD86FEA0C01A1
:10C6000001EB090222F003010A1DAA18043A24B919
:10C6100052F8041D013B0029FAD00361BDE8F88FF0
:10C620003B4601245F469B4611E728462146FFF71B
:10C6300059FB012202614461BDE8F88F2DE9F04306
:10C6400083B001211D4614460A9FFFF74BFBC5F33B
:10C650000A5625F07F438046A94623F470000EB1A8
:10C6600040F480100190002C24D002AA684642F8C1
:10C67000084DFFF701FC019B002831D1009CC8F850
:10C680001440002B0CBF01240224C8F81830C8F84D
:10C690001040DEB908EB8402A0F2324310693B601F
:10C6A000FFF7CCFB0B99C0EB44100860404603B089
:10C6B000BDE8F08301A8FFF7DFFB01990124C8F86A
:10C6C0001410C8F810402030002EE3D0A6F23349F1
:10C6D0000B9B09EB0002C0F135003A601860E5E7FA
:10C6E000C0F12001009A03FA01F444EA020123FA9E
:10C6F00000F3C8F814100193C3E700BF0B4661B103
:10C70000B1F1004F09D04FF6FF72A3F58011C7F6C3
:10C71000DF72914205D8042070470028F3D102202F
:10C72000704703F1FF4101F5E0019142F3D94FF663
:10C73000FF72C0F20F02934201D80320704703F149
:10C7400000419142F9D90022C7F6F072934204D019
:10C7500013F5801F01D000207047D0F1010038BFD1
:10C760000020704738B5074C002305460846236073
:10C77000F8F7D8FB431C00D038BD21680029FBD056
:10C78000296038BD184600202DE9F04F94681768DD
:10C7900083B0924681460D46002C6ED04FF0000BC0
:10C7A00008688E685C46002C47D0B442B04649D336
:10C7B000AB8913F4906F30D06E69296906EB46029D
:10C7C000C1EB000802EBD276601C76104044864232
:10C7D00003F4806332461BB23CBF064632464846ED
:10C7E000002B32D01146FEF789FE002836D0296989
:10C7F00001904246FFF7D0F9AA8922F4906040F0F8
:10C800008001A9810199C8EB060301EB08006E6164
:10C81000296128602646AB60A0465946424600F092
:10C8200079F9DAF80810AA682868961B40440C1BAE
:10C83000AE602860CAF80840FCB1D7F800B07C6848
:10C840000837B0E72646A046E7E700F0C5FA0146FC
:10C850000028D8D14846296900F092F8AA89002119
:10C8600042F040000C23C9F80030A8814FF0FF309F
:10C87000CAF80810CAF8041002E0CAF804402046BA
:10C8800003B0BDE8F08F00BF10B501FB02F1FEF769
:10C8900035FE044668B150F8042C22F003010A1F4B
:10C8A000242A18D8132A06D8034600201860586096
:10C8B0009860204610BD00231B2A036043600FD9F7
:10C8C000242A8360C36005BF0361436100F1100344
:10C8D00000F11803E9E7002100F0E8F9204610BD57
:10C8E00000F10803E1E700BFF8B5224D0F4604460A
:10C8F000FFF7F4F9AB685E6826F0030606F6EF7002
:10C90000C11B0A0B571E3F03B7F5805F07DB0021F1
:10C910002046FFF727FFAB689919884204D02046CC
:10C92000FFF7DEF90020F8BD79422046FFF71AFF35
:10C9300001300DD0104BA8681A68F61B46F00106AE
:10C94000D71B466020461F60FFF7CAF90120F8BDDB
:10C9500000212046FFF706FFAB68C21A0F2ADEDD72
:10C9600006490968401A044942F0010208605A6009
:10C97000D5E700BFA4070020D80B0020B00B002093
:10C980002DE9F0410D460646002955D0FFF7A6F9DE
:10C9900055F8041CDFF86CC1A5F1080421F001036F
:10C9A000E218DCF808005768904227F0030765D0CA
:10C9B00011F00101576032D00021D0194068C00742
:10C9C00006D4DB19906800294AD0D268C260906012
:10C9D00043F001006060E350E1B9B3F5007F2DD36F
:10C9E0005A0A042A66D89809383042000CEB820EA5
:10C9F0004449DEF80820724562D0506820F00301F7
:10CA00008B4202D292689645F7D1D068E060A2606E
:10CA1000D46084603046BDE8F041FFF761B955F855
:10CA2000085C641B0CF10808A06840452B443FD00B
:10CA3000E568C560A860C0E7BDE8F081DD080CEBE3
:10CA4000C502DCF804009168E260AB10012505FA2C
:10CA500003F31843A160CCF804009460CC60D9E7DC
:10CA6000294DA842B1D143F00102CCF81440CCF8D2
:10CA70001040E060A0606260E350CBE7FF18CB0796
:10CA800007D455F8081C641A7F18E368A068C360CF
:10CA900098601E4ACCF80840116847F001038F42A5
:10CAA0006360B7D31A4A30461168FFF71DFFB1E73C
:10CAB000012182E7142A0CD802F15B00420095E7BD
:10CAC0004B688010012505FA00F003434B601046C7
:10CAD0009CE7542A03D8180B6E30420086E7B2F563
:10CAE000AA7F03D8D80B773042007FE740F2545139
:10CAF0008A4203D8980C7C30420077E7FC227E20E3
:10CB000074E700BFA4070020AC070020AC0B002096
:10CB1000D40B002088422DE9F00326D98C18A042BE
:10CB200023D28318551EEAB1224605F0010412F8FB
:10CB3000011D03F8011D691EA5B13CB112F8014D9C
:10CB40000139B1F1FF3F03F8014D0BD012F8014D4F
:10CB500003F8014D023912F8014DB1F1FF3F03F81E
:10CB6000014DF3D1BDE8F00370470F2A40F29680E3
:10CB700041EA00039B0740F093800C6804604D6815
:10CB800045608E68A2F110038660CC681D460F2DAB
:10CB9000C460C3F3001601F1100400F1100322D9A0
:10CBA00066B126681E6066685E60A6689E60E6687C
:10CBB000103DDE60103410330F2D14D926681E602E
:10CBC00066685E60A6689E60E668DE6026691E6133
:10CBD00066695E61A6699E61E669203DDE6120347A
:10CBE00020330F2DEAD8A2F1100323F00F0402F036
:10CBF0000F031034032B00EB0408214452D9A3F196
:10CC000004090B464FEA990901EB890C53F8046BB0
:10CC1000C1EB0C0544460CF1040C634544F8046B6D
:10CC2000C5F3800512D02DB153F8045B634544F879
:10CC3000045B0BD01E46254656F8047B45F8047B62
:10CC40005F68331D67602C1D6345F3D109F1010353
:10CC50009C00091902F003024444002A82D02346B2
:10CC60000D7803F8015BA218E4431419934204F011
:10CC700001043FF477AF34B111F8014F03F8014BD1
:10CC800093423FF46FAF4D781C4604F8015B8D78FA
:10CC90005D70631C02319342F5D163E70446DCE723
:10CCA0000446DCE744461A46D7E700BFF0B48407E1
:10CCB000034600F08E80541E002A00F08880E507AD
:10CCC000CEB211D41A46671E02F8016B1346154600
:10CCD00092070FD0002C7AD003F8016B9A073C46DC
:10CCE0001D4607D0013CEDE7034603F8016B9A07A8
:10CCF0001D46F7D1032C52D9CEB246EA06270F2C97
:10CD000047EA07432DD9A4F1100217460F2FC2F3AB
:10CD100000162B606B60AB60EB6005F1100216D95A
:10CD20003EB1103F136053609360D36010320F2FF9
:10CD30000DD9203F02F11006136053609360D36059
:10CD4000136153619361D36120320F2FF1D8A4F1A5
:10CD5000100222F00F0204F00F041032032C1544CD
:10CD60001DD9271F3E462A46032E42F8043BC7F32F
:10CD700080070DD927B1043E032E42F8043B07D9A2
:10CD80001746083E47F8043B53603A1D032EF7D878
:10CD9000231F23F00302131D04F00304ED18B4B1A4
:10CDA0002B46C9B203F8011B2C19ED436219A342AB
:10CDB00002F001050BD01DB103F8011BA34206D000
:10CDC0001A4602F8011B5970531CA342F8D1F0BC5B
:10CDD0007047054614468DE72DE9F04F0C4683B0A9
:10CDE00081461746002900F0C580FEF777FF07F15E
:10CDF0000B0554F8043C162DA4F1080A23F0030691
:10CE00004FD810210D46AF4250D88E4253DADFF88A
:10CE1000A0C3DCF808000AEB0602904200F0B080E4
:10CE2000D2F804E02EF001089044D8F8048018F0FD
:10CE3000010F59D04FF0000E7246DB0776D454F83C
:10CE4000083CC3EB0A0BDBF8043023F003039B1907
:10CE50000193002A67D082420EEB030800F0F180B4
:10CE6000884560DBD16890685F46C1608860DBF808
:10CE70000C3057F8081F321F242ACB60996000F24B
:10CE80002A81132A40F2B9802368CBF80830616800
:10CE90001B2ACBF80C1000F234810BF1100008347F
:10CEA000ACE025F00705002D2946ACDA0C27C9F8BF
:10CEB0000070002714E0B046C5EB08070F2F1ED8FE
:10CEC00003F001030AEB080143EA0800CAF8040072
:10CED0004A6842F001074F604846FEF701FF2746C7
:10CEE000384603B0BDE8F08F2EF0030E0EEB0608B7
:10CEF0008845A2DBD7689268D760BA60DCE70AEBA6
:10CF0000050103F00103C8191D4347F00102CAF8E7
:10CF100004504A60476847F00103436008314846BF
:10CF2000FFF72EFDD8E7019B8B4234DA394648469D
:10CF3000FEF7E4FA0746C8B154F8043C23F00102B6
:10CF4000A0F108015244914200F0BE80321F242A11
:10CF500073D8132A46D82346196801605A6842607C
:10CF60009B68836048462146FFF70AFD4846FEF766
:10CF7000B7FEB5E7114603B0BDE8F04FFEF7BEBA05
:10CF8000426822F0030E0EEB060205F1100842453E
:10CF90003FDA024651E75F46DBF80C0057F8081FFE
:10CFA000321F242AC860816000F2A080132A40F258
:10CFB0009B802068CBF8080061681B2ACBF80C1016
:10CFC00000F2B4800BF1100308342068DDF804800F
:10CFD000186062685A60A4689C60DBF804303C46C4
:10CFE000DA4669E72168016060681B2A786060D8CA
:10CFF00007F1080004F10803AEE738462368036030
:10D0000062684260A4688460DBF804303C46DA461B
:10D0100052E70AEB0507501B40F001027A6054F812
:10D02000041CCCF8087001F001031D4344F8045CB3
:10D030004846FEF755FE274652E72146FFF76AFDB0
:10D0400090E705F110008045FFF66DAF5F46DBF815
:10D050000C0057F8081F321F242AC860816000F2B4
:10D060008780132A78D92068CBF8080061681B2ACA
:10D07000CBF80C1000F285800BF110030834206807
:10D08000186062685A60A16899600BEB0503C5EBF4
:10D09000080040F001025A60DBF80410CCF80830B8
:10D0A00001F001031D43CBF804504846FEF718FE7B
:10D0B00016E7A368BB60E168242AF9602DD007F168
:10D0C000100004F1100347E750F8047C27F0030C2C
:10D0D0000CEB0608F0E621463846FFF71BFD3C4600
:10D0E000DBF80430DA46E7E63B466EE72146384691
:10D0F000FFF710FD3C46DBF80430DDF80480DA462B
:10D10000DAE6A068CBF81000E368242ACBF81430E4
:10D1100018D00BF11800103470E722693A61636986
:10D1200007F118007B6104F1180315E7A368CBF839
:10D130001030E068242ACBF814000FD00BF118034C
:10D14000103442E72269CBF8182061690BF1200006
:10D15000CBF81C10183451E73B4690E72269CBF816
:10D16000182061690BF12003CBF81C1018342CE750
:10D1700038462146CDF800C0FFF7CCFCDDF800C0F2
:10D1800083E7A368CBF81030E068242ACBF81400BA
:10D1900003D00BF11803103471E72269CBF8182083
:10D1A00061690BF12003CBF81C10183467E700BF4E
:10D1B000A40700204BB942B9002908BF002802D0BB
:10D1C0004FF0FF31084600F037B882B0EC462DE949
:10D1D000005000F01BF8DDF804E002B00CBC704712
:10D1E000F8B5164604460D461F4600F027F806FB24
:10D1F00001F300FB0737A6FB0023FB18A21A65EB1F
:10D200000303069CC4E90023F8BD00BFF8B5164629
:10D2100004460D461F4600F06FF900FB07F7A0FB20
:10D22000062306FB0177FB18A21A65EB0303069C95
:10D23000C4E90023F8BD00BF704700BF00292DE9F5
:10D24000F00F1D46C0F29D800024002DC0F2948096
:10D2500080460F4694461E46E3BB8A4255D9B2FA31
:10D2600082F747B1C7F1200520FA05F601FA07F168
:10D27000BA403143B840170CB1FBF7F6030C1FFA64
:10D2800082FC07FB16110CFB06F543EA01439D42A5
:10D2900008D9711E9B1880F013819D4240F21081C5
:10D2A000023E9B18591BB1FBF7F507FB151380B223
:10D2B0000CFB05FC40EA03418C4507D96B1E8A181C
:10D2C00080F00081944540F2FD80023D45EA064130
:10D2D000002503E08B420CD9002529460A462B463F
:10D2E00014B1524263EB430310461946BDE8F00FF8
:10D2F0007047B3FA83F5002D40F087808B4201D34D
:10D300008242EAD800250121E8E712B90126B6FBDE
:10D31000F2F2B2FA82F6002E39D18E1A130C1FFAED
:10D3200082FC0125B6FBF3F703FB17614FEA1049B6
:10D330000CFB07F849EA0146B04506D9791EB61834
:10D3400002D2B04500F2D3800F46C8EB0606B6FB0A
:10D35000F3F103FB116380B20CFB01FC40EA0343D1
:10D360009C4506D94E1E9A1802D2944500F2C280FE
:10D37000314641EA0741B1E7E443524263EB4303DC
:10D3800066E7404261EB41014FF0FF345DE7B24098
:10D39000C6F1200921FA09F720FA09F5130C01FA60
:10D3A00006F1B7FBF3F845EA01091FFA82FC03FB1B
:10D3B00018774FEA19410CFB08F541EA0747B040DE
:10D3C000BD420AD9BF1808F1FF3680F08E80BD42F9
:10D3D00040F28B80A8F10208BF18791BB1FBF3F56E
:10D3E00003FB15171FFA89F90CFB05F649EA0741FB
:10D3F0008E4206D96F1E891871D28E426FD9023DB6
:10D4000089188E1B45EA08458CE7C5F1200122FAF0
:10D4100001F306FA05F61E4327FA01F24FEA164910
:10D4200007FA05F720FA01F1B2FBF9F80F433B0CBC
:10D430001FFA86FA09FB18220AFB08FB43EA02429C
:10D4400093450CFA05FC08D9921908F1FF314AD22C
:10D45000934548D9A8F102089219CBEB0203B3FB1C
:10D46000F9F109FB1132BFB20AFB01FA47EA0243A4
:10D470009A4506D94A1E9B1933D29A4531D90239A9
:10D480009B1941EA08410F0C1FFA8CF808FB07F6BC
:10D490008AB24FEA1C4C08FB02F80CFB026202EB5A
:10D4A00018420CFB07FC964288BF0CF5803CCAEB87
:10D4B00003030CEB124C63450ED305D000250DE79A
:10D4C0000E46EFE61D4601E71FFA88F800FA05F060
:10D4D00008EB0245A842F1D201390025FEE63D469F
:10D4E0008FE71146CDE78846B7E7B04675E7023FBC
:10D4F000B6182AE702393CE72DE9F007144605463D
:10D500000E46002B3DD18A4249D9B2FA82F747B183
:10D51000C7F1200120FA01F206FA07F6BC401643D3
:10D52000BD40220CB6FBF2F02F0CA1B202FB10663C
:10D5300001FB00F347EA0646B34208D9471E3619F5
:10D5400080F0F880B34240F2F58002383619F61ABE
:10D55000B6FBF2F302FB1362ADB201FB03F145EA45
:10D560000242914207D95E1E121980F0E580914275
:10D5700040F2E280023B43EA00400021BDE8F007B0
:10D5800070478B4243D8B3FA83F4002C42D18B42CC
:10D5900002D3824200F2DF8000210120EEE712B9BF
:10D5A0000127B7FBF2F4B4FA84F2002A40F0888035
:10D5B0000A1B230CA7B20121B2FBF3F603FB1622D0
:10D5C0004FEA154C07FB06F04CEA0242904207D99D
:10D5D000121906F1FF3C02D2904200F2CE8066465C
:10D5E000121AB2FBF3F003FB1023ADB207FB00F7F6
:10D5F00045EA03439F4207D9421E1B1980F09E80D3
:10D600009F4240F29B80023840EA0640B6E7002184
:10D610000846B3E7C4F1200622FA06F503FA04F33C
:10D620002B434FEA134C21FA06F501FA04F120FAD4
:10D6300006F6B5FBFCF746EA010A1FFA83F80CFB75
:10D6400017554FEA1A4108FB07F941EA0545A94574
:10D6500002FA04F203D97E1EED187FD33746C9EBD8
:10D660000501B1FBFCF60CFB16151FFA8AFA08FB44
:10D6700006F84AEA0541884503D9751EC91873D3CF
:10D680002E4646EA0746370C1FFA82FC0CFB07F5CC
:10D69000120CB3B20CFB03FC02FB035303EB1C4361
:10D6A00002FB07F29D4288BF02F58032C8EB010100
:10D6B00002EB134291424BD342D0304600215DE74A
:10D6C0009440C2F1200521FA05F6230C20FA05F753
:10D6D00001FA02F1B6FBF3FC39430D0CA7B203FBD0
:10D6E0001C6645EA064607FB0CF8B04500FA02F551
:10D6F00008D936190CF1FF303DD2B0453BD9ACF119
:10D70000020C3619C8EB0602B2FBF3F003FB10263D
:10D710008AB242EA064207FB00F1914206D9461E50
:10D72000121926D2914224D902381219521A40EA0B
:10D730000C4141E738460AE733461CE7104663E7E9
:10D740001FFA8CFC00FA04F00CEB03439842B4D2AD
:10D75000701E002112E7214620460FE7A9457FF6FB
:10D760007DAF023FED187AE7884589D9023EC91896
:10D7700087E73046DAE78446C4E7023E12192FE70E
:10D7800000018000800140004001C000C001200075
:10D790002001A000A00160006001E000E001100095
:10D7A00010019000900150005001D000D0013000D5
:10D7B0003001B000B00170007001F000F00108000D
:10D7C00008018800880148004801C800C8012800F5
:10D7D0002801A800A80168006801E800E801180015
:10D7E00018019800980158005801D800D801380055
:10D7F0003801B800B80178007801F800F801040099
:10D8000004018400840144004401C400C4012400D4
:10D810002401A400A40164006401E400E4011400F4
:10D8200014019400940154005401D400D401340034
:10D830003401B400B40174007401F400F4010C006C
:10D840000C018C008C014C004C01CC00CC012C0054
:10D850002C01AC00AC016C006C01EC00EC011C0074
:10D860001C019C009C015C005C01DC00DC013C00B4
:10D870003C01BC00BC017C007C01FC00FC010200FE
:10D8800002018200820142004201C200C201220064
:10D890002201A200A20162006201E200E201120084
:10D8A00012019200920152005201D200D2013200C4
:10D8B0003201B200B20172007201F200F2010A00FC
:10D8C0000A018A008A014A004A01CA00CA012A00E4
:10D8D0002A01AA00AA016A006A01EA00EA011A0004
:10D8E0001A019A009A015A005A01DA00DA013A0044
:10D8F0003A01BA00BA017A007A01FA00FA01060088
:10D9000006018600860146004601C600C6012600C3
:10D910002601A600A60166006601E600E6011600E3
:10D9200016019600960156005601D600D601360023
:10D930003601B600B60176007601F600F6010E005B
:10D940000E018E008E014E004E01CE00CE012E0043
:10D950002E01AE00AE016E006E01EE00EE011E0063
:10D960001E019E009E015E005E01DE00DE013E00A3
:10D970003E01BE00BE017E007E01FE00FE010100F0
:10D98000037F137D317B5E799877E07534749472F0
:10D99000FF70766FF66D826C166BB5695C680C670C
:10D9A000C46584644C631C62F360D05FB55EA05DA7
:10D9B000915C885B855A885990589E57B056C855D7
:10D9C000E45405542B5355528351B650EC4F264F17
:10D9D000644EA64DEC4C344C814BD04A234A7849D6
:10D9E000D1482D488C47ED465146B84521458D44D8
:10D9F000FC436C43DF425542CC414641C24040406B
:10DA00003FF0037F2074137D39E7317B949F5E796B
:10DA100029FD98772869E0754D5534744B3B947215
:10DA2000409CFF703100766F93F5F66DE310826CC9
:10DA30003AEC166BF626B5695F655C685D500C675D
:10DA40002D95C46519E584643EF54C634F7E1C62D8
:10DA5000613CF360B3EED05F8557B55EEB3BA05DF4
:10DA6000A163915CE698885B5AA8855ADF60885963
:10DA70007393905818139E57B8B4B0560B4FC855AF
:10DA800080BAE45424D105548F6E2B53D06F555275
:10DA90005AB38351F318B650A281EC4FA2CF264F50
:10DAA0004EE6644E1DAAA64D8B00EC4C10D0344CB3
:10DAB0001600814BEF78D04AC423234A96EA78496E
:10DAC00027B8D148FE772D4857168C471D80ED4664
:10DAD000E5A25146E26CB845E1CC214544B28D4403
:10DAE000FA0CFC4378CD6C43B4E4DF422644554243
:10DAF000B6DDCC41C6A346412389C24002814040E5
:10DB00000010002000400080080000000800000015
:10DB100008000000080000000100000001000000F3
:10DB200001000000000000000000000006000000EE
:10DB3000417564696F20537065637472756D20411F
:10DB40006E616C797A6572006F6E2053544D33327A
:10DB500046343037564700002D204453502F464658
:10DB600054204C6962726172790000002D2050448B
:10DB70004D204C69627261727900000050726573C9
:10DB80007320627574746F6E20746F20636F6E748F
:10DB9000696E75652E2E2E0044656D6F202D206FE9
:10DBA0006E652073696E6520776176650000000000
:10DBB00044656D6F202D2074776F2073696E65202A
:10DBC000776176657300000044656D6F202D2074C9
:10DBD000687265652073696E65207761766573008C
:10DBE00044656D6F202D20666F75722073696E65B8
:10DBF0002077617665730000463D253464205B31F3
:10DC00005D00000046313D253464205B315D2C20F1
:10DC100046323D253464205B315D000046333D25AE
:10DC20003464205B315D000046333D253464205B65
:10DC3000315D2C2046343D253464205B315D00008D
:10DC4000417564696F20537065637472756D00006F
:10DC5000463D25322E32665B6B487A5D20202000DF
:10DC6000252E3266000000005B6B487A5D000000E4
:10DC70000000003F000000BFF036FF3EB1FFFFBED6
:10DC8000E16DFE3EC4FEFFBED3A4FD3E39FDFFBEE6
:10DC9000C6DBFC3E11FBFFBEBB12FC3E4AF8FFBEDA
:10DCA000B249FB3EE6F4FFBEAD80FA3EE3F0FFBEB4
:10DCB000ABB7F93E43ECFFBEACEEF83E05E7FFBE66
:10DCC000B225F83E29E1FFBEBD5CF73EAFDAFFBEEC
:10DCD000CD93F63E97D3FFBEE3CAF53EE2CBFFBE3F
:10DCE0000002F53E8FC3FFBE2339F43E9EBAFFBE4D
:10DCF0004D70F33E0FB1FFBE7FA7F23EE3A6FFBE1D
:10DD0000B9DEF13E189CFFBEFD15F13EB190FFBE9D
:10DD1000494DF03EAB84FFBE9F84EF3E0878FFBEC6
:10DD2000FFBBEE3EC76AFFBE6AF3ED3EE95CFFBE95
:10DD3000DF2AED3E6D4EFFBE6162EC3E543FFFBEFA
:10DD4000EF99EB3E9D2FFFBE89D1EA3E491FFFBEF2
:10DD50003009EA3E580EFFBEE540E93EC9FCFEBE72
:10DD6000A878E83E9DEAFEBE79B0E73ED4D7FEBE75
:10DD700059E8E63E6DC4FEBE4920E63E69B0FEBEEF
:10DD80004958E53EC99BFEBE5990E43E8B86FEBED7
:10DD90007AC8E33EB070FEBEAD00E33E385AFEBE28
:10DDA000F138E23E2343FEBE4871E13E722BFEBED7
:10DDB000B2A9E03E2413FEBE2FE2DF3E38FAFDBEDC
:10DDC000BF1ADF3EB1E0FDBE6553DE3E8CC6FDBE30
:10DDD0001E8CDD3ECCABFDBEEDC4DC3E6E90FDBEC8
:10DDE000D2FDDB3E7474FDBECD36DB3EDE57FDBE9C
:10DDF000DF6FDA3EAC3AFDBE08A9D93EDD1CFDBEA0
:10DE000049E2D83E73FEFCBEA11BD83E6CDFFCBECF
:10DE10001355D73EC9BFFCBE9D8ED63E8A9FFCBE21
:10DE200041C8D53EB07EFCBEFF01D53E3A5DFCBE8A
:10DE3000D73BD43E283BFCBECB75D33E7A18FCBE04
:10DE4000DAAFD23E31F5FBBE05EAD13E4DD1FBBE85
:10DE50004C24D13ECDACFBBEB15ED03EB287FBBE02
:10DE60003299CF3EFC61FBBED2D3CE3EAB3BFBBE74
:10DE7000900ECE3EBE14FBBE6C49CD3E37EDFABED1
:10DE80006884CC3E16C5FABE84BFCB3E599CFABE10
:10DE9000C0FACA3E0273FABE1C36CA3E1049FABE28
:10DEA0009A71C93E841EFABE3AADC83E5EF3F9BE11
:10DEB000FBE8C73E9DC7F9BEDF24C73E439BF9BEC2
:10DEC000E760C63E4E6EF9BE119DC53EC040F9BE2C
:10DED00060D9C43E9812F9BED415C43ED6E3F8BE4C
:10DEE0006C52C33E7BB4F8BE298FC23E8684F8BE16
:10DEF0000DCCC13EF853F8BE1709C13ED122F8BE81
:10DF00004846C03E10F1F7BEA083BF3EB7BEF7BE85
:10DF100020C1BE3EC58BF7BEC8FEBD3E3A58F7BE17
:10DF2000993CBD3E1724F7BE937ABC3E5BEFF6BE2C
:10DF3000B6B8BB3E07BAF6BE04F7BA3E1B84F6BEBF
:10DF40007D35BA3E974DF6BE2074B93E7A16F6BEC0
:10DF5000EFB2B83EC6DEF5BEEAF1B73E7BA6F5BE2F
:10DF60001131B73E976DF5BE6670B63E1D34F5BEF5
:10DF7000E7AFB53E0BFAF4BE97EFB43E62BFF4BE16
:10DF8000752FB43E2284F4BE816FB33E4B48F4BE7D
:10DF9000BDAFB23EDD0BF4BE28F0B13ED9CEF3BE2C
:10DFA000C430B13E3F91F3BE9071B03E0E53F3BE0C
:10DFB0008EB2AF3E4714F3BEBDF3AE3EEBD4F2BE1D
:10DFC0001D35AE3EF894F2BEB176AD3E7054F2BE51
:10DFD00077B8AC3E5213F2BE71FAAB3E9FD1F1BEA0
:10DFE0009E3CAB3E578FF1BE007FAA3E7A4CF1BEFD
:10DFF00096C1A93E0809F1BE6204A93E01C5F0BE62
:10E000006347A83E6680F0BE9B8AA73E373BF0BEC2
:10E0100009CEA63E73F5EFBEAE11A63E1BAFEFBE16
:10E020008A55A53E3068EFBE9E99A43EB020EFBE53
:10E03000EBDDA33E9ED8EEBE7122A33EF88FEEBE6E
:10E040003067A23EBE46EEBE28ACA13EF2FCEDBE5D
:10E050005BF1A03E93B2EDBEC936A03EA167EDBE16
:10E06000717C9F3E1D1CEDBE55C29E3E07D0ECBE8E
:10E0700075089E3E5E83ECBED24E9D3E2436ECBEBD
:10E080006B959C3E58E8EBBE42DC9B3EFB99EBBE99
:10E0900056239B3E0C4BEBBEA96A9A3E8CFBEABE14
:10E0A0003AB2993E7BABEABE0BFA983ED95AEABE29
:10E0B0001B42983EA709EABE6B8A973EE4B7E9BEC9
:10E0C000FBD2963E9165E9BECD1B963EAE12E9BEEF
:10E0D000DF64953E3CBFE8BE34AE943E396BE8BE8B
:10E0E000CAF7933EA816E8BEA441933E87C1E7BE97
:10E0F000C08B923ED86BE7BE20D6913E9915E7BE05
:10E10000C320913ECCBEE6BEAC6B903E7167E6BECE
:10E11000D9B68F3E880FE6BE4B028F3E10B7E5BEE4
:10E12000034E8E3E0B5EE5BE019A8D3E7904E5BE40
:10E1300046E68C3E59AAE4BED1328C3EAC4FE4BEDA
:10E14000A47F8B3E73F4E3BEBFCC8A3EAC98E3BEA3
:10E15000231A8A3E5A3CE3BECF67893E7BDFE2BE8C
:10E16000C4B5883E1082E2BE0204883E1A24E2BE94
:10E170008B52873E98C5E1BE5EA1863E8A66E1BEAF
:10E180007CF0853EF206E1BEE63F853ECFA6E0BECE
:10E190009B8F843E2146E0BE9CDF833EE9E4DFBEE8
:10E1A000EA2F833E2783DFBE8480823EDB20DFBEF2
:10E1B0006DD1813E05BEDEBEA322813EA65ADEBEE3
:10E1C0002774803EBEF6DDBEF38B7F3E4D92DDBEF2
:10E1D00038307E3E532DDDBE1BD57C3ED1C7DCBE24
:10E1E0009E7A7B3EC761DCBEC1207A3E34FBDBBE3B
:10E1F00086C7783E1A94DBBEEE6E773E792CDBBE86
:10E20000F916763E50C4DABEA8BF743EA05BDABEF3
:10E21000FB68733E6AF2D9BEF412723EAD88D9BE75
:10E2200094BD703E6A1ED9BEDB686F3EA1B3D8BEF6
:10E23000CB146E3E5348D8BE63C16C3E7FDCD7BE64
:10E24000A56E6B3E2670D7BE921C6A3E4803D7BEB1
:10E250002ACB683EE595D6BE6E7A673EFE27D6BECF
:10E260005F2A663E93B9D5BEFFDA643EA44AD5BEA6
:10E270004C8C633E31DBD4BE4A3E623E3B6BD4BE27
:10E28000F7F0603EC3FAD3BE56A45F3EC789D3BE43
:10E2900066585E3E4918D3BE2A0D5D3E49A6D2BEE1
:10E2A000A0C25B3EC633D2BECB785A3EC2C0D1BEFE
:10E2B000AB2F593E3D4DD1BE41E7573E37D9D0BE79
:10E2C0008E9F563EAF64D0BE9158553EA8EFCFBE4C
:10E2D0004E12543E1F7ACFBEC3CC523E1704CFBE5F
:10E2E000F287513E908DCEBEDB43503E8916CEBEA6
:10E2F00080004F3E029FCDBEE1BD4D3EFD26CDBE0E
:10E30000FF7B4C3E79AECCBEDB3A4B3E7835CCBE83
:10E3100075FA493EF8BBCBBECEBA483EFA41CBBEF9
:10E32000E87B473E7FC7CABEC23D463E874CCABE59
:10E330005D00453E12D1C9BEBBC3433E2155C9BE97
:10E34000DC87423EB3D8C8BEC14C413ECA5BC8BEA2
:10E350006B12403E65DEC7BEDAD83E3E8560C7BE62
:10E360000FA03D3E2AE2C6BE0A683C3E5463C6BECC
:10E37000CE303B3E03E4C5BE59FA393E3964C5BED2
:10E38000AEC4383EF5E3C4BECD8F373E3763C4BE5E
:10E39000B65B363E00E2C3BE6B28353E5160C3BE5D
:10E3A000ECF5333E29DEC2BE39C4323E895BC2BEC3
:10E3B0005493313E70D8C1BE3E63303EE154C1BE7D
:10E3C000F6332F3EDAD0C0BE7E052E3E5C4CC0BE7A
:10E3D000D7D72C3E67C7BFBE01AB2B3EFC41BFBEAB
:10E3E000FC7E2A3E1BBCBEBECB53293EC535BEBEFD
:10E3F0006D29283EF9AEBDBEE3FF263EB827BDBE5F
:10E400002DD7253E03A0BCBE4EAF243ED917BCBEBF
:10E410004488233E3B8FBBBE1262223E2906BBBE10
:10E42000B73C213EA47CBABE3418203EACF2B9BE43
:10E430008BF41E3E4268B9BEBBD11D3E65DDB8BE41
:10E44000C6AF1C3E1652B8BEAC8E1B3E55C6B7BEFC
:10E450006E6E1A3E233AB7BE0C4F193E7FADB6BE64
:10E460008830183E6C20B6BEE112173EE792B5BE6A
:10E470001AF6153EF304B5BE31DA143E8F76B4BEFB
:10E4800029BF133EBCE7B3BE01A5123E7A58B3BE06
:10E49000BB8B113EC9C8B2BE5673103EAA38B2BE7D
:10E4A000D55B0F3E1DA8B1BE37450E3E2217B1BE4B
:10E4B0007D2F0D3EBB85B0BEA71A0C3EE6F3AFBE66
:10E4C000B7060B3EA561AFBEADF3093EF7CEAEBEBB
:10E4D0008AE1083EDE3BAEBE4ED0073E59A8ADBE37
:10E4E000FBBF063E6914ADBE90B0053E0F80ACBECA
:10E4F0000EA2043E4AEBABBE7694033E1B56ABBE67
:10E50000C987023E82C0AABE087C013E802AAABEFC
:10E510003271003E1594A9BE91CEFE3D41FDA8BECC
:10E520009ABCFC3D0566A8BE7EACFA3D61CEA7BE96
:10E530003F9EF83D5636A7BEDE91F63DE39DA6BE52
:10E540005D87F43D0A05A6BEBC7EF23DCB6BA5BE41
:10E55000FE77F03D25D2A4BE2373EE3D1A38A4BE4B
:10E560002D70EC3DA99DA3BE1C6FEA3DD302A3BE56
:10E57000F36FE83D9967A2BEB172E63DFBCBA1BE49
:10E580005A77E43DF92FA1BEED7DE23D9393A0BE05
:10E590006C86E03DCBF69FBED890DE3D9F599FBE76
:10E5A000329DDC3D12BC9EBE7CABDA3D221E9EBE7F
:10E5B000B7BBD83DD17F9DBEE4CDD63D1FE19CBE0B
:10E5C00003E2D43D0C429CBE18F8D23D99A29BBEFA
:10E5D0002110D13DC6029BBE222ACF3D93629ABE36
:10E5E0001A46CD3D00C299BE0B64CB3D0F2199BEAA
:10E5F000F783C93DC07F98BEDEA5C73D12DE97BE3A
:10E60000C1C9C53D073C97BEA2EFC33D9F9996BEC9
:10E610008217C23DD9F695BE6241C03DB75395BE43
:10E62000436DBE3D39B094BE269BBC3D5F0C94BE8D
:10E630000CCBBA3D2A6893BEF7FCB83D9AC392BE94
:10E64000E730B73DB01E92BEDE66B53D6B7991BE38
:10E65000DD9EB33DCDD390BEE4D8B13DD52D90BE67
:10E66000F614B03D84878FBE1253AE3DDBE08EBE04
:10E670003B93AC3DDA398EBE71D5AA3D81928DBEF9
:10E68000B519A93DD0EA8CBE0860A73DC9428CBE31
:10E690006CA8A53D6B9A8BBEE2F2A33DB7F18ABE92
:10E6A000693FA23DAD488ABE058EA03D4E9F89BE02
:10E6B000B5DE9E3D9BF588BE7B319D3D924B88BE6D
:10E6C00057869B3D36A187BE4BDD993D86F686BEBB
:10E6D0005836983D824B86BE7F91963D2CA085BED4
:10E6E000C0EE943D84F484BE1D4E933D894884BEA3
:10E6F00097AF913D3D9C83BE2F13903D9FEF82BE0F
:10E70000E6788E3DB14282BEBCE08C3D739581BE01
:10E71000B34A8B3DE4E780BECCB6893D063A80BE65
:10E720000725883DB2177FBE6795863DBBBA7DBE83
:10E73000EA07853D275D7CBE947C833DF7FE7ABE6B
:10E7400064F3813D2DA079BE5B6C803DC84078BEEE
:10E75000F6CE7D3DCBE076BE89C97A3D358075BE6B
:10E7600070C8773D071F74BEAECB743D43BD72BE0B
:10E7700044D3713DEA5A71BE34DF6E3DFBF76FBE84
:10E7800080EF6B3D79946EBE2A04693D63306DBEA7
:10E79000331D663DBBCB6BBE9E3A633D81666ABE50
:10E7A0006B5C603DB70069BE9E825D3D5D9A67BE51
:10E7B00038AD5A3D753366BE3ADC573DFECB64BE7C
:10E7C000A60F553DFA6363BE7D47523D6AFB61BEAD
:10E7D000C3834F3D4F9260BE78C44C3DA9285FBEB5
:10E7E0009E094A3D79BE5DBE3653473DC1535CBE6E
:10E7F00043A1443D80E85ABEC6F3413DB97C59BEB1
:10E80000C04A3F3D6B1058BE34A63C3D99A356BE4E
:10E8100023063A3D413655BE8E6A373D67C853BE22
:10E8200078D3343D095A52BEE140323D2AEB50BE06
:10E83000CCB22F3DCA7B4FBE39292D3DEA0B4EBECF
:10E840002BA42A3D8B9B4CBEA323283DAE2A4BBE56
:10E85000A3A7253D53B949BE2C30233D7C4748BE74
:10E860003FBD203D29D546BEDF4E1E3D5C6245BE04
:10E870000CE51B3D15EF43BEC97F193D557B42BEDC
:10E88000161F173D1E0741BEF5C2143D6F923FBED5
:10E89000676B123D4A1D3EBE6F18103DAFA73CBED0
:10E8A0000DCA0D3DA0313BBE43800B3D1EBB39BEA2
:10E8B000123B093D2A4438BE7CFA063DC3CC36BE25
:10E8C00082BE043DEC5435BE2587023DA5DC33BE37
:10E8D0006754003DEF6332BE934CFC3CCBEA30BE44
:10E8E0009BF9F73C3A712FBEE8AFF33C3CF72DBEE5
:10E8F0007E6FEF3CD47C2CBE5E38EB3C01022BBE1D
:10E900008C0AE73CC48629BE0AE6E23C1F0B28BEFF
:10E91000DACADE3C128F26BE00B9DA3C9F1225BE51
:10E920007EB0D63CC59523BE55B1D23C871822BED9
:10E930008ABBCE3CE59A20BE1DCFCA3CDF1C1FBE61
:10E9400012ECC63C789E1DBE6B12C33CAF1F1CBEB2
:10E950002A42BF3C86A01ABE527BBB3CFE2019BE99
:10E96000E5BDB73C17A117BEE509B43CD22016BEE1
:10E97000555FB03C31A014BE36BEAC3C351F13BE53
:10E980008C26A93CDD9D11BE5798A53C2C1C10BEC1
:10E990009C13A23C229A0EBE5A989E3CC0170DBEF4
:10E9A00096269B3C07950BBE51BE973CF7110ABEBD
:10E9B0008C5F943C938E08BE4B0A913CDA0A07BEEA
:10E9C0008FBE8D3CCE8605BE5A7C8A3C700204BE4A
:10E9D000AE43873CC07D02BE8D14843CC0F800BEAF
:10E9E000FAEE803CE1E6FEBDEBA57B3CA4DBFBBD83
:10E9F0000481753CCCCFF8BD436F6F3C5AC3F5BD65
:10EA0000AC70693C51B6F2BD4285633CB2A8EFBD23
:10EA100009AD5D3C7F9AECBD04E8573CBA8BE9BD7B
:10EA20003736523C667CE6BDA6974C3C836CE3BD12
:10EA3000540C473C135CE0BD4494413C1A4BDDBD93
:10EA40007A2F3C3C9739DABDF9DD363C8F27D7BDAC
:10EA5000C59F313C0115D4BDE0742C3CF101D1BD02
:10EA60004F5D273C60EECDBD1359223C4FDACABD45
:10EA700030681D3CC2C5C7BDA98A183CB9B0C4BD29
:10EA800082C0133C379BC1BDBD090F3C3E85BEBD56
:10EA90005C660A3CCF6EBBBD64D6053CEC57B8BD86
:10EAA000D659013C9840B5BD6BE1F93BD428B2BDC5
:10EAB0000B36F13BA210AFBD90B1E83B04F8ABBD03
:10EAC0000154E03BFCDEA8BD611DD83B8CC5A5BD53
:10EAD000B60DD03BB6ABA2BD0625C83B7B919FBD12
:10EAE0005563C03BDE769CBDA7C8B83BE05B99BDD3
:10EAF0000255B13B834096BD6A08AA3BCA2493BD28
:10EB0000E3E2A23BB70890BD73E49B3B4AEC8CBDAB
:10EB10001D0D953B86CF89BDE55C8E3B6EB286BDF3
:10EB2000D0D3873B029583BDE271813B457780BDA1
:10EB30003C6E763B73B27ABD12476A3BC07574BDBA
:10EB40004C6E5E3B76386EBDF2E3523B9AFA67BD7F
:10EB50000AA8473B2EBC61BD9DBA3C3B377D5BBDDF
:10EB6000AF1B323BB93D55BD49CB273BB7FD4EBD31
:10EB700071C91D3B36BD48BD2C16143B397C42BDC6
:10EB800080B10A3BC33A3CBD749B013BDAF835BD0A
:10EB90001AA8F13A80B62FBDA1B6E03ABA7329BDE2
:10EBA0008762D03A8C3023BDD6ABC03AF9EC1CBD9D
:10EBB0009892B13A05A916BDD616A33AB46410BD11
:10EBC0009A38953A0A200ABDECF7873A0ADB03BD6A
:10EBD000A7A9763A742BFBBCB29E5E3A38A0EEBC75
:10EBE00007CF473A6914E2BCB53A323A0E88D5BC31
:10EBF000C8E11D3A30FBC8BC4EC40A3AD56DBCBC56
:10EC0000A5C4F13907E0AFBCBF77D039CB51A3BC65
:10EC100000A2B1392CC396BC7B4395392F348ABCF2
:10EC200084B87639BA497BBCC7D847397A2A62BCDE
:10EC3000DFE71D39B00A49BCC8CBF13869EA2FBCFF
:10EC4000DAA5B138B6C916BC3BBC76384B51FBBB14
:10EC500064E91D38900EC9BBD1A6B13758CB96BB1D
:10EC6000C6E91D37880F49BBDEE91D36C60FC9BA94
:10EC700000000000E845D2A8DEE91D36C60FC93AFB
:10EC8000C6E91D37880F493BD1A6B13758CB963B13
:10EC900064E91D38900EC93B3BBC76384B51FB3BB9
:10ECA000DAA5B138B6C9163CC8CBF13869EA2F3CB1
:10ECB000DFE71D39B00A493CC7D847397A2A623C98
:10ECC00084B87639BA497B3C7B4395392F348A3CEA
:10ECD00000A2B1392CC3963CBF77D039CB51A33CAD
:10ECE000A5C4F13907E0AF3C4EC40A3AD56DBC3C2F
:10ECF000C8E11D3A30FBC83CB53A323A0E88D53CE3
:10ED000007CF473A6914E23CB29E5E3A38A0EE3C27
:10ED1000A7A9763A742BFB3CECF7873A0ADB033D54
:10ED20009A38953A0A200A3DD616A33AB464103DA3
:10ED30009892B13A05A9163DD6ABC03AF9EC1C3D04
:10ED40008762D03A8C30233DA1B6E03ABA73293DB0
:10ED50001AA8F13A80B62F3D749B013BDAF8353D95
:10ED600080B10A3BC33A3C3D2C16143B397C423DF2
:10ED700071C91D3B36BD483D49CB273BB7FD4E3DD4
:10ED8000AF1B323BB93D553D9DBA3C3B377D5B3DAA
:10ED90000AA8473B2EBC613DF2E3523B9AFA673D1D
:10EDA0004C6E5E3B76386E3D12476A3BC075743DD3
:10EDB0003C6E763B73B27A3DE271813B4577803D94
:10EDC000D0D3873B0295833DE55C8E3B6EB2863D9A
:10EDD0001D0D953B86CF893D73E49B3B4AEC8C3DF2
:10EDE000E3E2A23BB708903D6A08AA3BCA24933DE0
:10EDF0000255B13B8340963DA7C8B83BE05B993DC7
:10EE00005563C03BDE769C3D0625C83B7B919F3D0C
:10EE1000B60DD03BB6ABA23D611DD83B8CC5A53D20
:10EE20000154E03BFCDEA83D90B1E83B04F8AB3D6B
:10EE30000B36F13BA210AF3D6BE1F93BD428B23D5C
:10EE4000D659013C9840B53D64D6053CEC57B83DD9
:10EE50005C660A3CCF6EBB3DBD090F3C3E85BE3DA6
:10EE600082C0133C379BC13DA98A183CB9B0C43D50
:10EE700030681D3CC2C5C73D1359223C4FDACA3D1C
:10EE80004F5D273C60EECD3DE0742C3CF101D13D5F
:10EE9000C59F313C0115D43DF9DD363C8F27D73D68
:10EEA0007A2F3C3C9739DA3D4494413C1A4BDD3D86
:10EEB000540C473C135CE03DA6974C3C836CE33D0F
:10EEC0003736523C667CE63D04E8573CBA8BE93D58
:10EED00009AD5D3C7F9AEC3D4285633CB2A8EF3DB5
:10EEE000AC70693C51B6F23D436F6F3C5AC3F53D7F
:10EEF0000481753CCCCFF83DEBA57B3CA4DBFB3D0E
:10EF0000FAEE803CE1E6FE3D8D14843CC0F8003E04
:10EF1000AE43873CC07D023E5A7C8A3C7002043E70
:10EF20008FBE8D3CCE86053E4B0A913CDA0A073EE9
:10EF30008C5F943C938E083E51BE973CF7110A3E7D
:10EF400096269B3C07950B3E5A989E3CC0170D3E5B
:10EF50009C13A23C229A0E3E5798A53C2C1C103EB6
:10EF60008C26A93CDD9D113E36BEAC3C351F133EC0
:10EF7000555FB03C31A0143EE509B43CD220163EAA
:10EF8000E5BDB73C17A1173E527BBB3CFE20193EA6
:10EF90002A42BF3C86A01A3E6B12C33CAF1F1C3EE8
:10EFA00012ECC63C789E1D3E1DCFCA3CDF1C1F3EA6
:10EFB0008ABBCE3CE59A203E55B1D23C8718223E12
:10EFC0007EB0D63CC595233E00B9DA3C9F12253E63
:10EFD000DACADE3C128F263E0AE6E23C1F0B283ED0
:10EFE0008C0AE73CC486293E5E38EB3C01022B3E8E
:10EFF0007E6FEF3CD47C2C3EE8AFF33C3CF72D3EDB
:10F000009BF9F73C3A712F3E934CFC3CCBEA303EE7
:10F010006754003DEF63323E2587023DA5DC333E59
:10F0200082BE043DEC54353E7CFA063DC3CC363EF0
:10F03000123B093D2A44383E43800B3D1EBB393EFE
:10F040000DCA0D3DA0313B3E6F18103DAFA73C3EB1
:10F05000676B123D4A1D3E3EF5C2143D6F923F3E26
:10F06000161F173D1E07413EC97F193D557B423E85
:10F070000CE51B3D15EF433EDF4E1E3D5C62453EF9
:10F080003FBD203D29D5463E2C30233D7C47483EA0
:10F09000A3A7253D53B9493EA323283DAE2A4B3EA5
:10F0A0002BA42A3D8B9B4C3E39292D3DEA0B4E3E2D
:10F0B000CCB22F3DCA7B4F3EE140323D2AEB503E61
:10F0C00078D3343D095A523E8E6A373D67C8533E65
:10F0D00023063A3D4136553E34A63C3D99A3563E63
:10F0E000C04A3F3D6B10583EC6F3413DB97C593E86
:10F0F00043A1443D80E85A3E3653473DC1535C3EF0
:10F100009E094A3D79BE5D3E78C44C3DA9285F3ECC
:10F11000C3834F3D4F92603E7D47523D6AFB613E47
:10F12000A60F553DFA63633E3ADC573DFECB643E85
:10F1300038AD5A3D7533663E9E825D3D5D9A673EB1
:10F140006B5C603DB700693E9E3A633D81666A3EF6
:10F15000331D663DBBCB6B3E2A04693D63306D3E7B
:10F1600080EF6B3D79946E3E34DF6E3DFBF76F3E72
:10F1700044D3713DEA5A713EAECB743D43BD723EFD
:10F1800070C8773D071F743E89C97A3D3580753E4A
:10F19000F6CE7D3DCBE0763E5B6C803DC840783E50
:10F1A00064F3813D2DA0793E947C833DF7FE7A3E49
:10F1B000EA07853D275D7C3E6795863DBBBA7D3E6F
:10F1C0000725883DB2177F3ECCB6893D063A803E82
:10F1D000B34A8B3DE4E7803EBCE08C3D7395813EB5
:10F1E000E6788E3DB142823E2F13903D9FEF823EE6
:10F1F00097AF913D3D9C833E1D4E933D8948843E93
:10F20000C0EE943D84F4843E7F91963D2CA0853ED3
:10F210005836983D824B863E4BDD993D86F6863EBC
:10F2200057869B3D36A1873E7B319D3D924B883E64
:10F23000B5DE9E3D9BF5883E058EA03D4E9F893EE6
:10F24000693FA23DAD488A3EE2F2A33DB7F18A3E56
:10F250006CA8A53D6B9A8B3E0860A73DC9428C3EC9
:10F26000B519A93DD0EA8C3E71D5AA3D81928D3E5B
:10F270003B93AC3DDA398E3E1253AE3DDBE08E3E21
:10F28000F614B03D84878F3EE4D8B13DD52D903E35
:10F29000DD9EB33DCDD3903EDE66B53D6B79913EAC
:10F2A000E730B73DB01E923EF7FCB83D9AC3923EA0
:10F2B0000CCBBA3D2A68933E269BBC3D5F0C943E26
:10F2C000436DBE3D39B0943E6241C03DB753953E5B
:10F2D0008217C23DD9F6953EA2EFC33D9F99963E57
:10F2E000C1C9C53D073C973EDEA5C73D12DE973E2E
:10F2F000F783C93DC07F983E0B64CB3D0F21993EFB
:10F300001A46CD3D00C2993E222ACF3D93629A3ED5
:10F310002110D13DC6029B3E18F8D23D99A29B3EDA
:10F3200003E2D43D0C429C3EE4CDD63D1FE19C3E21
:10F33000B7BBD83DD17F9D3E7CABDA3D221E9E3EC1
:10F34000329DDC3D12BC9E3ED890DE3D9F599F3ED3
:10F350006C86E03DCBF69F3EED7DE23D9393A03E73
:10F360005A77E43DF92FA13EB172E63DFBCBA13EB9
:10F37000F36FE83D9967A23E1C6FEA3DD302A33EBE
:10F380002D70EC3DA99DA33E2373EE3D1A38A43E9B
:10F39000FE77F03D25D2A43EBC7EF23DCB6BA53E70
:10F3A0005D87F43D0A05A63EDE91F63DE39DA63E4F
:10F3B0003F9EF83D5636A73E7EACFA3D61CEA73E55
:10F3C0009ABCFC3D0566A83E91CEFE3D41FDA83E9F
:10F3D0003271003E1594A93E087C013E802AAA3E67
:10F3E000C987023E82C0AA3E7694033E1B56AB3EBE
:10F3F0000EA2043E4AEBAB3E90B0053E0F80AC3E01
:10F40000FBBF063E6914AD3E4ED0073E59A8AD3E47
:10F410008AE1083EDE3BAE3EADF3093EF7CEAE3E9E
:10F42000B7060B3EA561AF3EA71A0C3EE6F3AF3E12
:10F430007D2F0D3EBB85B03E37450E3E2217B13EB7
:10F44000D55B0F3E1DA8B13E5673103EAA38B23EA2
:10F45000BB8B113EC9C8B23E01A5123E7A58B33EDD
:10F4600029BF133EBCE7B33E31DA143E8F76B43E7B
:10F470001AF6153EF304B53EE112173EE792B53E8B
:10F480008830183E6C20B63E0C4F193E7FADB63E1C
:10F490006E6E1A3E233AB73EAC8E1B3E55C6B73E43
:10F4A000C6AF1C3E1652B83EBBD11D3E65DDB83E10
:10F4B0008BF41E3E4268B93E3418203EACF2B93E91
:10F4C000B73C213EA47CBA3E1262223E2906BB3ED6
:10F4D0004488233E3B8FBB3E4EAF243ED917BC3EF3
:10F4E0002DD7253E03A0BC3EE3FF263EB827BD3EF8
:10F4F0006D29283EF9AEBD3ECB53293EC535BE3EF3
:10F50000FC7E2A3E1BBCBE3E01AB2B3EFC41BF3EF7
:10F51000D7D72C3E67C7BF3E7E052E3E5C4CC03E13
:10F52000F6332F3EDAD0C03E3E63303EE154C13E5A
:10F530005493313E70D8C13E39C4323E895BC23EDD
:10F54000ECF5333E29DEC23E6B28353E5160C33EAA
:10F55000B65B363E00E2C33ECD8F373E3763C43ED6
:10F56000AEC4383EF5E3C43E59FA393E3964C53E6F
:10F57000CE303B3E03E4C53E0A683C3E5463C63E83
:10F580000FA03D3E2AE2C63EDAD83E3E8560C73E29
:10F590006B12403E65DEC73EC14C413ECA5BC83E71
:10F5A000DC87423EB3D8C83EBBC3433E2155C93E6B
:10F5B0005D00453E12D1C93EC23D463E874CCA3E23
:10F5C000E87B473E7FC7CA3ECEBA483EFA41CB3EB3
:10F5D00075FA493EF8BBCB3EDB3A4B3E7835CC3E24
:10F5E000FF7B4C3E79AECC3EE1BD4D3EFD26CD3E8F
:10F5F00080004F3E029FCD3EDB43503E8916CE3EFB
:10F60000F287513E908DCE3EC3CC523E1704CF3E82
:10F610004E12543E1F7ACF3E9158553EA8EFCF3E32
:10F620008E9F563EAF64D03E41E7573E37D9D03E1D
:10F63000AB2F593E3D4DD13ECB785A3EC2C0D13E54
:10F64000A0C25B3EC633D23E2A0D5D3E49A6D23EE5
:10F6500066585E3E4918D33E56A45F3EC789D33EE6
:10F66000F7F0603EC3FAD33E4A3E623E3B6BD43E67
:10F670004C8C633E31DBD43EFFDA643EA44AD53E77
:10F680005F2A663E93B9D53E6E7A673EFE27D63E28
:10F690002ACB683EE595D63E921C6A3E4803D73E8B
:10F6A000A56E6B3E2670D73E63C16C3E7FDCD73EB5
:10F6B000CB146E3E5348D83EDB686F3EA1B3D83EB4
:10F6C00094BD703E6A1ED93EF412723EAD88D93E9A
:10F6D000FB68733E6AF2D93EA8BF743EA05BDA3E77
:10F6E000F916763E50C4DA3EEE6E773E792CDB3E5C
:10F6F00086C7783E1A94DB3EC1207A3E34FBDB3E5F
:10F700009E7A7B3EC761DC3E1BD57C3ED1C7DC3E8A
:10F7100038307E3E532DDD3EF38B7F3E4D92DD3EF5
:10F720002774803EBEF6DD3EA322813EA65ADE3E11
:10F730006DD1813E05BEDE3E8480823EDB20DF3E11
:10F74000EA2F833E2783DF3E9CDF833EE9E4DF3EF2
:10F750009B8F843E2146E03EE63F853ECFA6E03EBD
:10F760007CF0853EF206E13E5EA1863E8A66E13E81
:10F770008B52873E98C5E13E0204883E1A24E23E41
:10F78000C4B5883E1082E23ECF67893E7BDFE23E11
:10F79000231A8A3E5A3CE33EBFCC8A3EAC98E33EF5
:10F7A000A47F8B3E73F4E33ED1328C3EAC4FE43EFB
:10F7B00046E68C3E59AAE43E019A8D3E7904E53E28
:10F7C000034E8E3E0B5EE53E4B028F3E10B7E53E8C
:10F7D000D9B68F3E880FE63EAC6B903E7167E63E31
:10F7E000C320913ECCBEE63E20D6913E9915E73E21
:10F7F000C08B923ED86BE73EA441933E87C1E73E63
:10F80000CAF7933EA816E83E34AE943E396BE83E04
:10F81000DF64953E3CBFE83ECD1B963EAE12E93E0E
:10F82000FBD2963E9165E93E6B8A973EE4B7E93E8E
:10F830001B42983EA709EA3E0BFA983ED95AEA3E87
:10F840003AB2993E7BABEA3EA96A9A3E8CFBEA3E0D
:10F8500056239B3E0C4BEB3E42DC9B3EFB99EB3E22
:10F860006B959C3E58E8EB3ED24E9D3E2436EC3ED6
:10F8700075089E3E5E83EC3E55C29E3E07D0EC3E30
:10F88000717C9F3E1D1CED3EC936A03EA167ED3E3A
:10F890005BF1A03E93B2ED3E28ACA13EF2FCED3E02
:10F8A0003067A23EBE46EE3E7122A33EF88FEE3E8A
:10F8B000EBDDA33E9ED8EE3E9E99A43EB020EF3EE7
:10F8C0008A55A53E3068EF3EAE11A63E1BAFEF3E17
:10F8D00009CEA63E73F5EF3E9B8AA73E373BF03E2E
:10F8E0006347A83E6680F03E6204A93E01C5F03E33
:10F8F00096C1A93E0809F13E007FAA3E7A4CF13E2E
:10F900009E3CAB3E578FF13E71FAAB3E9FD1F13E2C
:10F9100077B8AC3E5213F23EB176AD3E7054F23E33
:10F920001D35AE3EF894F23EBDF3AE3EEBD4F23E52
:10F930008EB2AF3E4714F33E9071B03E0E53F33E8D
:10F94000C430B13E3F91F33E28F0B13ED9CEF33EF4
:10F95000BDAFB23EDD0BF43E816FB33E4B48F43E8B
:10F96000752FB43E2284F43E97EFB43E62BFF43E5E
:10F97000E7AFB53E0BFAF43E6670B63E1D34F53E79
:10F980001131B73E976DF53EEAF1B73E7BA6F53EE5
:10F99000EFB2B83EC6DEF53E2074B93E7A16F63EAA
:10F9A0007D35BA3E974DF63E04F7BA3E1B84F63ECF
:10F9B000B6B8BB3E07BAF63E937ABC3E5BEFF63E66
:10F9C000993CBD3E1724F73EC8FEBD3E3A58F73E6F
:10F9D00020C1BE3EC58BF73EA083BF3EB7BEF73EFB
:10F9E0004846C03E10F1F73E1709C13ED122F83E0D
:10F9F0000DCCC13EF853F83E298FC23E8684F83EB6
:10FA00006C52C33E7BB4F83ED415C43ED6E3F83EF8
:10FA100060D9C43E9812F93E119DC53EC040F93EE2
:10FA2000E760C63E4E6EF93EDF24C73E439BF93E7B
:10FA3000FBE8C73E9DC7F93E3AADC83E5EF3F93ECE
:10FA40009A71C93E841EFA3E1C36CA3E1049FA3EDF
:10FA5000C0FACA3E0273FA3E84BFCB3E599CFA3EBE
:10FA60006884CC3E16C5FA3E6C49CD3E37EDFA3E71
:10FA7000900ECE3EBE14FB3ED2D3CE3EAB3BFB3E01
:10FA80003299CF3EFC61FB3EB15ED03EB287FB3E79
:10FA90004C24D13ECDACFB3E05EAD13E4DD1FB3EE0
:10FAA000DAAFD23E31F5FB3ECB75D33E7A18FC3E41
:10FAB000D73BD43E283BFC3EFF01D53E3A5DFC3EA1
:10FAC00041C8D53EB07EFC3E9D8ED63E8A9FFC3E10
:10FAD0001355D73EC9BFFC3EA11BD83E6CDFFC3E90
:10FAE00049E2D83E73FEFC3E08A9D93EDD1CFD3E2E
:10FAF000DF6FDA3EAC3AFD3ECD36DB3EDE57FD3EF3
:10FB0000D2FDDB3E7474FD3EEDC4DC3E6E90FD3EE6
:10FB10001E8CDD3ECCABFD3E6553DE3E8CC6FD3E0D
:10FB2000BF1ADF3EB1E0FD3E2FE2DF3E38FAFD3E78
:10FB3000B2A9E03E2413FE3E4871E13E722BFE3E28
:10FB4000F138E23E2343FE3EAD00E33E385AFE3E2E
:10FB50007AC8E33EB070FE3E5990E43E8B86FE3E8E
:10FB60004958E53EC99BFE3E4920E63E69B0FE3E4F
:10FB700059E8E63E6DC4FE3E79B0E73ED4D7FE3E7E
:10FB8000A878E83E9DEAFE3EE540E93EC9FCFE3E1F
:10FB90003009EA3E580EFF3E89D1EA3E491FFF3E3A
:10FBA000EF99EB3E9D2FFF3E6162EC3E543FFF3EDE
:10FBB000DF2AED3E6D4EFF3E6AF3ED3EE95CFF3E0F
:10FBC000FFBBEE3EC76AFF3E9F84EF3E0878FF3ED4
:10FBD000494DF03EAB84FF3EFD15F13EB190FF3E36
:10FBE000B9DEF13E189CFF3E7FA7F23EE3A6FF3E42
:10FBF0004D70F33E0FB1FF3E2339F43E9EBAFF3EF7
:10FC00000002F53E8FC3FF3EE3CAF53EE2CBFF3E66
:10FC1000CD93F63E97D3FF3EBD5CF73EAFDAFF3E95
:10FC2000B225F83E29E1FF3EACEEF83E05E7FF3E87
:10FC3000ABB7F93E43ECFF3EAD80FA3EE3F0FF3E4A
:10FC4000B249FB3EE6F4FF3EBB12FC3E4AF8FF3EE3
:10FC5000C6DBFC3E11FBFF3ED3A4FD3E39FDFF3E5B
:10FC6000E16DFE3EC4FEFF3EF036FF3EB1FFFF3EBB
:10FC70000000003F0000003F8864003FB1FFFF3EEE
:10FC800010C9003FC4FEFF3E972D013F39FDFF3EE6
:10FC90001D92013F11FBFF3EA3F6013F4AF8FF3ED4
:10FCA000275B023FE6F4FF3EAABF023FE3F0FF3EC0
:10FCB0002B24033F43ECFF3EAA88033F05E7FF3EAA
:10FCC00027ED033F29E1FF3EA151043FAFDAFF3E9C
:10FCD00019B6043F97D3FF3E8E1A053FE2CBFF3E95
:10FCE000007F053F8FC3FF3E6FE3053F9EBAFF3E97
:10FCF000D947063F0FB1FF3E40AC063FE3A6FF3EAB
:10FD0000A310073F189CFF3E0275073FB190FF3ECE
:10FD10005CD9073FAB84FF3EB13D083F0878FF3E0A
:10FD200001A2083FC76AFF3E4B06093FE95CFF3E60
:10FD3000906A093F6D4EFF3ED0CE093F543FFF3ED3
:10FD400009330A3F9D2FFF3E3C970A3F491FFF3E64
:10FD500068FB0A3F580EFF3E8E5F0B3FC9FCFE3E1C
:10FD6000ACC30B3F9DEAFE3EC4270C3FD4D7FE3EFA
:10FD7000D38B0C3F6DC4FE3EDBEF0C3F69B0FE3E03
:10FD8000DC530D3FC99BFE3ED3B70D3F8B86FE3E35
:10FD9000C31B0E3FB070FE3EAA7F0E3F385AFE3E98
:10FDA00087E30E3F2343FE3E5C470F3F722BFE3E30
:10FDB00027AB0F3F2413FE3EE90E103F38FAFD3EFD
:10FDC000A072103FB1E0FD3E4ED6103F8CC6FD3E06
:10FDD000F139113FCCABFD3E899D113F6E90FD3E48
:10FDE0001701123F7474FD3E9964123FDE57FD3EC9
:10FDF00010C8123FAC3AFD3E7C2B133FDD1CFD3E8C
:10FE0000DC8E133F73FEFC3E2FF2133F6CDFFC3E93
:10FE10007755143FC9BFFC3EB1B8143F8A9FFC3EE2
:10FE2000E01B153FB07EFC3E017F153F3A5DFC3E76
:10FE300014E2153F283BFC3E1B45163F7A18FC3E5A
:10FE400013A8163F31F5FB3EFE0A173F4DD1FB3E8E
:10FE5000DA6D173FCDACFB3EA8D0173FB287FB3E13
:10FE60006733183FFC61FB3E1796183FAB3BFB3EE8
:10FE7000B8F8183FBE14FB3E4A5B193F37EDFA3E17
:10FE8000CCBD193F16C5FA3E3E201A3F599CFA3E9A
:10FE9000A0821A3F0273FA3EF2E41A3F1049FA3E7A
:10FEA00033471B3F841EFA3E63A91B3F5EF3F93EB6
:10FEB000820B1C3F9DC7F93E906D1C3F439BF93E52
:10FEC0008DCF1C3F4E6EF93E77311D3FC040F93E4D
:10FED00050931D3F9812F93E16F51D3FD6E3F83EAC
:10FEE000CA561E3F7BB4F83E6BB81E3F8684F83E70
:10FEF000F9191F3FF853F83E757B1F3FD122F83E9A
:10FF0000DCDC1F3F10F1F73E303E203FB7BEF73E2E
:10FF1000709F203FC58BF73E9C00213F3A58F73E2B
:10FF2000B461213F1724F73EB7C2213F5BEFF63E95
:10FF3000A523223F07BAF63E7E84223F1B84F63E6D
:10FF400042E5223F974DF63EF045233F7A16F63EB6
:10FF500088A6233FC6DEF53E0B07243F7BA6F53E71
:10FF60007767243F976DF53ECDC7243F1D34F53E9E
:10FF70000C28253F0BFAF43E3588253F62BFF43E3E
:10FF800046E8253F2284F43E3F48263F4B48F43E56
:10FF900022A8263FDD0BF43EEC07273FD9CEF33EE7
:10FFA0009E67273F3F91F33E38C7273F0E53F33EEE
:10FFB000B926283F4714F33E2286283FEBD4F23E71
:10FFC00071E5283FF894F23EA844293F7054F23E70
:10FFD000C5A3293F5213F23EC8022A3F9FD1F13EEA
:10FFE000B1612A3F578FF13E80C02A3F7A4CF13EE3
:10FFF000351F2B3F0809F13ECF7D2B3F01C5F03E59
:020000040801F1
:100000004EDC2B3F6680F03EB33A2C3F373BF03E50
:10001000FC982C3F73F5EF3E29F72C3F1BAFEF3ECA
:100020003B552D3F3068EF3E31B32D3FB020EF3EC2
:100030000A112E3F9ED8EE3EC86E2E3FF88FEE3E40
:1000400068CC2E3FBE46EE3EEC292F3FF2FCED3E43
:1000500052872F3F93B2ED3E9CE42F3FA167ED3EC8
:10006000C741303F1D1CED3ED59E303F07D0EC3ED2
:10007000C5FB303F5E83EC3E9758313F2436EC3E63
:100080004AB5313F58E8EB3EDF11323FFB99EB3E7A
:10009000556E323F0C4BEB3EABCA323F8CFBEA3E17
:1000A000E326333F7BABEA3EFB82333FD95AEA3E3D
:1000B000F3DE333FA709EA3ECB3A343FE4B7E93EEB
:1000C0008296343F9165E93E1AF2343FAE12E93E22
:1000D000904D353F3CBFE83EE6A8353F396BE83EE2
:1000E0001B04363FA816E83E2E5F363F87C1E73E29
:1000F00020BA363FD86BE73EF014373F9915E73EFC
:100100009E6F373FCCBEE63E2ACA373F7167E63E58
:100110009424383F880FE63EDB7E383F10B7E53E3B
:10012000FFD8383F0B5EE53E0033393F7904E53EAA
:10013000DD8C393F59AAE43E97E6393FAC4FE43EA7
:100140002E403A3F73F4E33EA0993A3FAC98E33E29
:10015000EFF23A3F5A3CE33E194C3B3F7BDFE23E35
:100160001EA53B3F1082E23EFFFD3B3F1A24E23ECC
:10017000BA563C3F98C5E13E51AF3C3F8A66E13EEE
:10018000C2073D3FF206E13E0D603D3FCFA6E03E97
:1001900033B83D3F2146E03E32103E3FE9E4DF3ECA
:1001A0000B683E3F2783DF3EBEBF3E3FDB20DF3E86
:1001B0004A173F3F05BEDE3EAF6E3F3FA65ADE3ECA
:1001C000EDC53F3FBEF6DD3E031D403F4D92DD3E97
:1001D000F273403F532DDD3EB9CA403FD1C7DC3EEC
:1001E0005921413FC761DC3ED077413F34FBDB3EC4
:1001F0001ECE413F1A94DB3E4524423F792CDB3E24
:10020000427A423F50C4DA3E16D0423FA05BDA3E0B
:10021000C125433F6AF2D93E437B433FAD88D93E77
:100220009BD0433F6A1ED93EC925443FA1B3D83E67
:10023000CD7A443F5348D83EA7CF443F7FDCD73EDA
:100240005724453F2670D73EDC78453F4803D73ECC
:1002500036CD453FE595D63E6421463FFE27D63E46
:100260006875463F93B9D53E40C9463FA44AD53E3E
:10027000ED1C473F31DBD43E6E70473F3B6BD43EB5
:10028000C2C3473FC3FAD33EEB16483FC789D33EAC
:10029000E669483F4918D33EB6BC483F49A6D23E1E
:1002A000580F493FC633D23ECD61493FC2C0D13E0F
:1002B00015B4493F3D4DD13E30064A3F37D9D03E77
:1002C0001D584A3FAF64D03EDCA94A3FA8EFCF3E5D
:1002D0006DFB4A3F1F7ACF3ECF4C4B3F1704CF3EBA
:1002E000049E4B3F908DCE3E09EF4B3F8916CE3E8C
:1002F000E03F4C3F029FCD3E88904C3FFD26CD3ED7
:1003000000E14C3F79AECC3E49314D3F7835CC3E93
:1003100063814D3FF8BBCB3E4CD14D3FFA41CB3EC4
:1003200006214E3F7FC7CA3E90704E3F874CCA3E63
:10033000E9BF4E3F12D1C93E110F4F3F2155C93E73
:10034000095E4F3FB3D8C83ED0AC4F3FCA5BC83EF2
:1003500065FB4F3F65DEC73ECA49503F8560C73EDB
:10036000FC97503F2AE2C63EFDE5503F5463C63E2F
:10037000CD33513F03E4C53E6A81513F3964C53EE8
:10038000D4CE513FF5E3C43E0D1C523F3763C43E0B
:100390001269523F00E2C33EE5B5523F5160C33E91
:1003A0008502533F29DEC23EF24E533F895BC23E77
:1003B0002B9B533F70D8C13E31E7533FE154C13EC0
:1003C0000233543FDAD0C03EA07E543F5C4CC03E66
:1003D0000ACA543F67C7BF3E4015553FFC41BF3E68
:1003E0004160553F1BBCBE3E0DAB553FC535BE3EC3
:1003F000A5F5553FF9AEBD3E0740563FB827BD3E77
:10040000358A563F03A0BC3E2DD4563FD917BC3E7B
:10041000EF1D573F3B8FBB3E7C67573F2906BB3ED6
:10042000D2B0573FA47CBA3EF3F9573FACF2B93E85
:10043000DD42583F4268B93E918B583F65DDB83E7A
:100440000FD4583F1652B83E551C593F55C6B73EBB
:100450006564593F233AB73E3DAC593F7FADB63E48
:10046000DEF3593F6C20B63E483B5A3FE792B53E1B
:100470007A825A3FF304B53E74C95A3F8F76B43E30
:1004800036105B3FBCE7B33EC0565B3F7A58B33E85
:10049000119D5B3FC9C8B23E2AE35B3FAA38B23E1A
:1004A0000B295C3F1DA8B13EB26E5C3F2217B13EE6
:1004B00021B45C3FBB85B03E56F95C3FE6F3AF3EEE
:1004C000523E5D3FA561AF3E15835D3FF7CEAE3E28
:1004D0009DC75D3FDE3BAE3EEC0B5E3F59A8AD3E97
:1004E00001505E3F6914AD3EDC935E3F0F80AC3E31
:1004F0007DD75E3F4AEBAB3EE21A5F3F1B56AB3EF9
:100500000E5E5F3F82C0AA3EFEA05F3F802AAA3EE9
:10051000B4E35F3F1594A93E2E26603F41FDA83EFF
:100520006D68603F0566A83E70AA603F61CEA73E39
:1005300038EC603F5636A73EC42D613FE39DA63E92
:10054000146F613F0A05A63E28B0613FCB6BA53E04
:1005500000F1613F25D2A43E9C31623F1A38A43E8F
:10056000FA71623FA99DA33E1CB2623FD302A33E33
:1005700002F2623F9967A23EAA31633FFBCBA13EE4
:100580001571633FF92FA13E42B0633F9393A03EA4
:1005900033EF633FCBF69F3EE52D643F9F599F3E6F
:1005A0005A6C643F12BC9E3E90AA643F221E9E3E3F
:1005B00089E8643FD17F9D3E4426653F1FE19C3E14
:1005C000C063653F0C429C3EFDA0653F99A29B3EE7
:1005D000FCDD653FC6029B3EBC1A663F93629A3EB5
:1005E0003D57663F00C2993E7F93663F0F21993E7B
:1005F00081CF663FC07F983E440B673F12DE973E37
:10060000C846673F073C973E0C82673F9F99963EDE
:1006100010BD673FD9F6953ED4F7673FB753953E77
:100620005832683F39B0943E9B6C683F5F0C943EF3
:100630009FA6683F2A68933E61E0683F9AC3923E56
:10064000E319693FB01E923E2453693F6B79913E96
:10065000248C693FCDD3903EE3C4693FD52D903EB5
:1006600061FD693F84878F3E9E356A3FDBE08E3EA9
:10067000996D6A3FDA398E3E52A56A3F81928D3E6E
:10068000C9DC6A3FD0EA8C3EFF136B3FC9428C3E07
:10069000F24A6B3F6B9A8B3EA4816B3FB7F18A3E67
:1006A00013B86B3FAD488A3E3FEE6B3F4E9F893E8D
:1006B00029246C3F9BF5883ED1596C3F924B883E74
:1006C000358F6C3F36A1873E57C46C3F86F6863E19
:1006D00035F96C3F824B863ED02D6D3F2CA0853E78
:1006E00028626D3F84F4843E3C966D3F8948843E89
:1006F0000DCA6D3F3D9C833E9AFD6D3F9FEF823E4C
:10070000E3306E3FB142823EE8636E3F7395813EB7
:10071000AA966E3FE4E7803E27C96E3F063A803EC8
:100720005FFB6E3FB2177F3E532D6F3FBBBA7D3EDE
:10073000035F6F3F275D7C3E6E906F3FF7FE7A3E12
:1007400094C16F3F2DA0793E75F26F3FC840783E4F
:100750001123703FCBE0763E6753703F3580753E86
:100760007983703F071F743E45B3703F43BD723EAF
:10077000CCE2703FEA5A713E0D12713FFBF76F3EBB
:100780000841713F79946E3EBD6F713F63306D3E9D
:100790002D9E713FBBCB6B3E56CC713F81666A3E4E
:1007A00039FA713FB700693ED627723F5D9A673EBE
:1007B0002D55723F7533663E3C82723FFECB643EE0
:1007C00006AF723FFA63633E88DB723F6AFB613EAD
:1007D000C407733F4F92603EB933733FA9285F3E11
:1007E000665F733F79BE5D3ECD8A733FC1535C3E09
:1007F000ECB5733F80E85A3EC4E0733FB97C593E84
:10080000540B743F6B10583E9D35743F99A3563E70
:100810009E5F743F4136553E5789743F67C8533ECB
:10082000C9B2743F095A523EF2DB743F2AEB503E84
:10083000D304753FCA7B4F3E6C2D753FEA0B4E3E8D
:10084000BD55753F8B9B4C3EC67D753FAE2A4B3EDA
:1008500086A5753F53B9493EFDCC753F7C47483E60
:100860002CF4753F29D5463E121B763F5C62453E0F
:10087000AF41763F15EF433E0368763F557B423EDE
:100880000F8E763F1E07413ED1B3763F6F923F3EBB
:100890004AD9763F4A1D3E3E79FE763FAFA73C3EA1
:1008A0005F23773FA0313B3EFC47773F1EBB393E7D
:1008B0004F6C773F2A44383E5890773FC3CC363E42
:1008C00018B4773FEC54353E8ED7773FA5DC333EE6
:1008D000BAFA773FEF63323E9B1D783FCBEA303E5A
:1008E0003340783F3A712F3E8162783F3CF72D3E8E
:1008F0008484783FD47C2C3E3DA6783F01022B3E79
:10090000ACC7783FC486293ED0E8783F1F0B283E0D
:10091000A909793F128F263E382A793F9F12253E3A
:100920007C4A793FC595233E756A793F8718223EF8
:10093000248A793FE59A203E87A9793FDF1C1F3E34
:100940009FC8793F789E1D3E6DE7793FAF1F1C3EE3
:10095000EF057A3F86A01A3E25247A3FFE20193EF5
:1009600011427A3F17A1173EB15F7A3FD220163E5F
:10097000057D7A3F31A0143E0E9A7A3F351F133E13
:10098000CCB67A3FDD9D113E3DD37A3F2C1C103E04
:1009900063EF7A3F229A0E3E3D0B7B3FC0170D3E20
:1009A000CB267B3F07950B3E0D427B3FF7110A3E5E
:1009B000045D7B3F938E083EAE777B3FDA0A073EAD
:1009C0000C927B3FCE86053E1DAC7B3F7002043E01
:1009D000E3C57B3FC07D023E5CDF7B3FC0F8003E4D
:1009E00088F87B3FE1E6FE3D68117C3FA4DBFB3DE0
:1009F000FC297C3FCCCFF83D43427C3F5AC3F53DB8
:100A00003D5A7C3F51B6F23DEB717C3FB2A8EF3DC1
:100A10004C897C3F7F9AEC3D60A07C3FBA8BE93DDE
:100A200027B77C3F667CE63DA1CD7C3F836CE33DF0
:100A3000CFE37C3F135CE03DAFF97C3F1A4BDD3DDB
:100A4000420F7D3F9739DA3D88247D3F8F27D73D80
:100A500081397D3F0115D43D2C4E7D3FF101D13DC3
:100A60008B627D3F60EECD3D9C767D3F4FDACA3D87
:100A70005F8A7D3FC2C5C73DD59D7D3FB9B0C43DAE
:100A8000FEB07D3F379BC13DD9C37D3F3E85BE3D16
:100A900067D67D3FCF6EBB3DA6E87D3FEC57B83DA6
:100AA00099FA7D3F9840B53D3D0C7E3FD428B23D3C
:100AB000941D7E3FA210AF3D9D2E7E3F04F8AB3DBE
:100AC000583F7E3FFCDEA83DC54F7E3F8CC5A53D0F
:100AD000E55F7E3FB6ABA23DB66F7E3F7B919F3D0B
:100AE000397F7E3FDE769C3D6F8E7E3FE05B993D99
:100AF000569D7E3F8340963DEFAB7E3FCA24933D9B
:100B00003ABA7E3FB708903D37C87E3F4AEC8C3DED
:100B1000E6D57E3F86CF893D46E37E3F6EB2863D79
:100B200058F07E3F0295833D1CFD7E3F4577803D1A
:100B300092097F3F73B27A3DB9157F3FC075743D0E
:100B400092217F3F76386E3D1C2D7F3F9AFA673D9C
:100B500058387F3F2EBC613D45437F3F377D5B3D2D
:100B6000E44D7F3FB93D553D35587F3FB7FD4E3D84
:100B700037627F3F36BD483DEA6B7F3F397C423D5F
:100B80004E757F3FC33A3C3D657E7F3FDAF8353D89
:100B90002C877F3F80B62F3DA58F7F3FBA73293DBD
:100BA000CF977F3F8C30233DAA9F7F3FF9EC1C3DC0
:100BB00037A77F3F05A9163D75AE7F3FB464103D52
:100BC00064B57F3F0A200A3D04BC7F3F0ADB033D3A
:100BD00056C27F3F742BFB3C58C87F3F38A0EE3C89
:100BE0000CCE7F3F6914E23C71D37F3F0E88D53C29
:100BF00088D87F3F30FBC83C4FDD7F3FD56DBC3C84
:100C0000C7E17F3F07E0AF3CF1E57F3FCB51A33C1D
:100C1000CCE97F3F2CC3963C58ED7F3F2F348A3C74
:100C200094F07F3FBA497B3C82F37F3F7A2A623C53
:100C300022F67F3FB00A493C72F87F3F69EA2F3CB9
:100C400073FA7F3FB6C9163C25FC7F3F4B51FB3BF7
:100C500088FD7F3F900EC93B9DFE7F3F58CB963B62
:100C600062FF7F3F880F493BD9FF7F3FC60FC93ADC
:100C70000000803FE845D228D9FF7F3FC60FC9BAA0
:100C800062FF7F3F880F49BB9DFE7F3F58CB96BBDD
:100C900088FD7F3F900EC9BB25FC7F3F4B51FBBBBE
:100CA00073FA7F3FB6C916BC72F87F3F69EA2FBC62
:100CB00022F67F3FB00A49BC82F37F3F7A2A62BCAA
:100CC00094F07F3FBA497BBC58ED7F3F2F348ABCFC
:100CD000CCE97F3F2CC396BCF1E57F3FCB51A3BC51
:100CE000C7E17F3F07E0AFBC4FDD7F3FD56DBCBCA8
:100CF00088D87F3F30FBC8BC71D37F3F0E88D5BCFE
:100D00000CCE7F3F6914E2BC58C87F3F38A0EEBCD0
:100D100056C27F3F742BFBBC04BC7F3F0ADB03BD84
:100D200064B57F3F0A200ABD75AE7F3FB46410BD35
:100D300037A77F3F05A916BDAA9F7F3FF9EC1CBDD1
:100D4000CF977F3F8C3023BDA58F7F3FBA7329BDDE
:100D50002C877F3F80B62FBD657E7F3FDAF835BD9B
:100D60004E757F3FC33A3CBDEA6B7F3F397C42BD45
:100D700037627F3F36BD48BD35587F3FB7FD4EBD1A
:100D8000E44D7F3FB93D55BD45437F3F377D5BBD5A
:100D900058387F3F2EBC61BD1C2D7F3F9AFA67BD3E
:100DA00092217F3F76386EBDB9157F3FC07574BD07
:100DB00092097F3F73B27ABD1CFD7E3F457780BDAF
:100DC00058F07E3F029583BD46E37E3F6EB286BDFE
:100DD000E6D57E3F86CF89BD37C87E3F4AEC8CBDC5
:100DE0003ABA7E3FB70890BDEFAB7E3FCA2493BDB1
:100DF000569D7E3F834096BD6F8E7E3FE05B99BDE2
:100E0000397F7E3FDE769CBDB66F7E3F7B919FBD76
:100E1000E55F7E3FB6ABA2BDC54F7E3F8CC5A5BD8D
:100E2000583F7E3FFCDEA8BD9D2E7E3F04F8ABBD43
:100E3000941D7E3FA210AFBD3D0C7E3FD428B2BDB5
:100E400099FA7D3F9840B5BDA6E87D3FEC57B8BD07
:100E500067D67D3FCF6EBBBDD9C37D3F3E85BEBD4E
:100E6000FEB07D3F379BC1BDD59D7D3FB9B0C4BDB0
:100E70005F8A7D3FC2C5C7BD9C767D3F4FDACABD44
:100E80008B627D3F60EECDBD2C4E7D3FF101D1BD2B
:100E900081397D3F0115D4BD88247D3F8F27D7BD83
:100EA000420F7D3F9739DABDAFF97C3F1A4BDDBD6C
:100EB000CFE37C3F135CE0BDA1CD7C3F836CE3BD01
:100EC00027B77C3F667CE6BD60A07C3FBA8BE9BD5E
:100ED0004C897C3F7F9AECBDEB717C3FB2A8EFBDA3
:100EE0003D5A7C3F51B6F2BD43427C3F5AC3F5BDEB
:100EF000FC297C3FCCCFF8BD68117C3FA4DBFBBD57
:100F000088F87B3FE1E6FEBD5CDF7B3FC0F800BEBA
:100F1000E3C57B3FC07D02BE1DAC7B3F700204BEBB
:100F20000C927B3FCE8605BEAE777B3FDA0A07BECA
:100F3000045D7B3F938E08BE0D427B3FF7110ABED6
:100F4000CB267B3F07950BBE3D0B7B3FC0170DBEED
:100F500063EF7A3F229A0EBE3DD37A3F2C1C10BE1F
:100F6000CCB67A3FDD9D11BE0E9A7A3F351F13BE77
:100F7000057D7A3F31A014BEB15F7A3FD22016BE04
:100F800011427A3F17A117BE25247A3FFE2019BED1
:100F9000EF057A3F86A01ABE6DE7793FAF1F1CBEF2
:100FA0009FC8793F789E1DBE87A9793FDF1C1FBE71
:100FB000248A793FE59A20BE756A793F871822BE58
:100FC0007C4A793FC59523BE382A793F9F1225BEBA
:100FD000A909793F128F26BED0E8783F1F0B28BEA3
:100FE000ACC7783FC48629BE3DA6783F01022BBE20
:100FF0008484783FD47C2CBE8162783F3CF72DBE40
:101000003340783F3A712FBE9B1D783FCBEA30BE0C
:10101000BAFA773FEF6332BE8ED7773FA5DC33BE97
:1010200018B4773FEC5435BE5890773FC3CC36BEEA
:101030004F6C773F2A4438BEFC47773F1EBB39BE12
:101040005F23773FA0313BBE79FE763FAFA73CBE22
:101050004AD9763F4A1D3EBED1B3763F6F923FBE1E
:101060000F8E763F1E0741BE0368763F557B42BE1A
:10107000AF41763F15EF43BE121B763F5C6245BE23
:101080002CF4753F29D546BEFDCC753F7C4748BE44
:1010900086A5753F53B949BEC67D753FAE2A4BBE86
:1010A000BD55753F8B9B4CBE6C2D753FEA0B4EBEFC
:1010B000D304753FCA7B4FBEF2DB743F2AEB50BEB0
:1010C000C9B2743F095A52BE5789743F67C853BEAC
:1010D0009E5F743F413655BE9D35743F99A356BE01
:1010E000540B743F6B1058BEC4E0733FB97C59BEBB
:1010F000ECB5733F80E85ABECD8A733FC1535CBEE6
:10110000665F733F79BE5DBEB933733FA9285FBE8A
:10111000C407733F4F9260BE88DB723F6AFB61BEBB
:1011200006AF723FFA6363BE3C82723FFECB64BE81
:101130002D55723F753366BED627723F5D9A67BEE6
:1011400039FA713FB70069BE56CC713F81666ABEFD
:101150002D9E713FBBCB6BBEBD6F713F63306DBECB
:101160000841713F79946EBE0D12713FFBF76FBE5F
:10117000CCE2703FEA5A71BE45B3703F43BD72BEC8
:101180007983703F071F74BE6753703F358075BE0B
:101190001123703FCBE076BE75F26F3FC84078BE3A
:1011A00094C16F3F2DA079BE6E906F3FF7FE7ABE5F
:1011B000035F6F3F275D7CBE532D6F3FBBBA7DBE83
:1011C0005FFB6E3FB2177FBE27C96E3F063A80BEF7
:1011D000AA966E3FE4E780BEE8636E3F739581BEDA
:1011E000E3306E3FB14282BE9AFD6D3F9FEF82BEFB
:1011F0000DCA6D3F3D9C83BE3C966D3F894884BEC1
:1012000028626D3F84F484BED02D6D3F2CA085BE36
:1012100035F96C3F824B86BE57C46C3F86F686BE5E
:10122000358F6C3F36A187BED1596C3F924B88BE3B
:1012300029246C3F9BF588BE3FEE6B3F4E9F89BED5
:1012400013B86B3FAD488ABEA4816B3FB7F18ABE2D
:10125000F24A6B3F6B9A8BBEFF136B3FC9428CBE49
:10126000C9DC6A3FD0EA8CBE52A56A3F81928DBE2E
:10127000996D6A3FDA398EBE9E356A3FDBE08EBEDD
:1012800061FD693F84878FBEE3C4693FD52D90BE61
:10129000248C693FCDD390BE2453693F6B7991BEB6
:1012A000E319693FB01E92BE61E0683F9AC392BEE7
:1012B0009FA6683F2A6893BE9B6C683F5F0C94BEF4
:1012C0005832683F39B094BED4F7673FB75395BEE4
:1012D00010BD673FD9F695BE0C82673F9F9996BEB9
:1012E000C846673F073C97BE440B673F12DE97BE78
:1012F00081CF663FC07F98BE7F93663F0F2199BE26
:101300003D57663F00C299BEBC1A663F93629ABEC3
:10131000FCDD653FC6029BBEFDA0653F99A29BBE5A
:10132000C063653F0C429CBE4426653F1FE19CBEE6
:1013300089E8643FD17F9DBE90AA643F221E9EBE75
:101340005A6C643F12BC9EBEE52D643F9F599FBE00
:1013500033EF633FCBF69FBE42B0633F9393A0BE93
:101360001571633FF92FA1BEAA31633FFBCBA1BE2C
:1013700002F2623F9967A2BE1CB2623FD302A3BED3
:10138000FA71623FA99DA3BE9C31623F1A38A4BE88
:1013900000F1613F25D2A4BE28B0613FCB6BA5BE52
:1013A000146F613F0A05A6BEC42D613FE39DA6BE32
:1013B00038EC603F5636A7BE70AA603F61CEA7BE2C
:1013C0006D68603F0566A8BE2E26603F41FDA8BE41
:1013D000B4E35F3F1594A9BEFEA05F3F802AAABE7A
:1013E0000E5E5F3F82C0AABEE21A5F3F1B56ABBED5
:1013F0007DD75E3F4AEBABBEDC935E3F0F80ACBE59
:1014000001505E3F6914ADBEEC0B5E3F59A8ADBE06
:101410009DC75D3FDE3BAEBE15835D3FF7CEAEBEE2
:10142000523E5D3FA561AFBE56F95C3FE6F3AFBEED
:1014300021B45C3FBB85B0BEB26E5C3F2217B1BE2B
:101440000B295C3F1DA8B1BE2AE35B3FAA38B2BEA0
:10145000119D5B3FC9C8B2BEC0565B3F7A58B3BE50
:1014600036105B3FBCE7B3BE74C95A3F8F76B4BE3B
:101470007A825A3FF304B5BE483B5A3FE792B5BE65
:10148000DEF3593F6C20B6BE3DAC593F7FADB6BED2
:101490006564593F233AB7BE551C593F55C6B7BE80
:1014A0000FD4583F1652B8BE918B583F65DDB8BE79
:1014B000DD42583F4268B9BEF3F9573FACF2B9BEBE
:1014C000D2B0573FA47CBABE7C67573F2906BBBE4B
:1014D000EF1D573F3B8FBBBE2DD4563FD917BCBE27
:1014E000358A563F03A0BCBE0740563FB827BDBE55
:1014F000A5F5553FF9AEBDBE0DAB553FC535BEBEDA
:101500004160553F1BBCBEBE4015553FFC41BFBEB0
:101510000ACA543F67C7BFBEA07E543F5C4CC0BEE2
:101520000233543FDAD0C0BE31E7533FE154C1BE6D
:101530002B9B533F70D8C1BEF24E533F895BC2BE56
:101540008502533F29DEC2BEE5B5523F5160C3BE9E
:101550001269523F00E2C3BE0D1C523F3763C4BE46
:10156000D4CE513FF5E3C4BE6A81513F3964C5BE54
:10157000CD33513F03E4C5BEFDE5503F5463C6BEC5
:10158000FC97503F2AE2C6BECA49503F8560C7BE9D
:1015900065FB4F3F65DEC7BED0AC4F3FCA5BC8BEE0
:1015A000095E4F3FB3D8C8BE110F4F3F2155C9BE8A
:1015B000E9BF4E3F12D1C9BE90704E3F874CCABEA4
:1015C00006214E3F7FC7CABE4CD14D3FFA41CBBE2C
:1015D00063814D3FF8BBCBBE49314D3F7835CCBE22
:1015E00000E14C3F79AECCBE88904C3FFD26CDBE8D
:1015F000E03F4C3F029FCDBE09EF4B3F8916CEBE68
:10160000049E4B3F908DCEBECF4C4B3F1704CFBEB8
:101610006DFB4A3F1F7ACFBEDCA94A3FA8EFCFBE81
:101620001D584A3FAF64D0BE30064A3F37D9D0BEBE
:1016300015B4493F3D4DD1BECD61493FC2C0D1BE79
:10164000580F493FC633D2BEB6BC483F49A6D2BEAA
:10165000E669483F4918D3BEEB16483FC789D3BE59
:10166000C2C3473FC3FAD3BE6E70473F3B6BD4BE85
:10167000ED1C473F31DBD4BE40C9463FA44AD5BE2E
:101680006875463F93B9D5BE6421463FFE27D6BE56
:1016900036CD453FE595D6BEDC78453F4803D7BEFD
:1016A0005724453F2670D7BEA7CF443F7FDCD7BE27
:1016B000CD7A443F5348D8BEC925443FA1B3D8BED4
:1016C0009BD0433F6A1ED9BE437B433FAD88D9BE02
:1016D000C125433F6AF2D9BE16D0423FA05BDABEB5
:1016E000427A423F50C4DABE4524423F792CDBBEE9
:1016F0001ECE413F1A94DBBED077413F34FBDBBEA8
:101700005921413FC761DCBEB9CA403FD1C7DCBEE9
:10171000F273403F532DDDBE031D403F4D92DDBEB1
:10172000EDC53F3FBEF6DDBEAF6E3F3FA65ADEBE03
:101730004A173F3F05BEDEBEBEBF3E3FDB20DFBED9
:101740000B683E3F2783DFBE32103E3FE9E4DFBE39
:1017500033B83D3F2146E0BE0D603D3FCFA6E0BE21
:10176000C2073D3FF206E1BE51AF3C3F8A66E1BE93
:10177000BA563C3F98C5E1BEFFFD3B3F1A24E2BE8E
:101780001EA53B3F1082E2BE194C3B3F7BDFE2BE11
:10179000EFF23A3F5A3CE3BEA0993A3FAC98E3BE21
:1017A0002E403A3F73F4E3BE97E6393FAC4FE4BEB8
:1017B000DD8C393F59AAE4BE0033393F7904E5BED8
:1017C000FFD8383F0B5EE5BEDB7E383F10B7E5BE85
:1017D0009424383F880FE6BE2ACA373F7167E6BEB9
:1017E0009E6F373FCCBEE6BEF014373F9915E7BE7B
:1017F00020BA363FD86BE7BE2E5F363F87C1E7BEC3
:101800001B04363FA816E8BEE6A8353F396BE8BE94
:10181000904D353F3CBFE8BE1AF2343FAE12E9BEF0
:101820008296343F9165E9BECB3A343FE4B7E9BED6
:10183000F3DE333FA709EABEFB82333FD95AEABE43
:10184000E326333F7BABEABEABCA323F8CFBEABE3A
:10185000556E323F0C4BEBBEDF11323FFB99EBBEB6
:101860004AB5313F58E8EBBE9758313F2436ECBEBD
:10187000C5FB303F5E83ECBED59E303F07D0ECBE4B
:10188000C741303F1D1CEDBE9CE42F3FA167EDBE5C
:1018900052872F3F93B2EDBEEC292F3FF2FCEDBEF5
:1018A00068CC2E3FBE46EEBEC86E2E3FF88FEEBE11
:1018B0000A112E3F9ED8EEBE31B32D3FB020EFBEB1
:1018C0003B552D3F3068EFBE29F72C3F1BAFEFBED5
:1018D000FC982C3F73F5EFBEB33A2C3F373BF0BE7C
:1018E0004EDC2B3F6680F0BECF7D2B3F01C5F0BEA6
:1018F000351F2B3F0809F1BE80C02A3F7A4CF1BE4C
:10190000B1612A3F578FF1BEC8022A3F9FD1F1BE75
:10191000C5A3293F5213F2BEA844293F7054F2BE1A
:1019200071E5283FF894F2BE2286283FEBD4F2BE40
:10193000B926283F4714F3BE38C7273F0E53F3BEDE
:101940009E67273F3F91F3BEEC07273FD9CEF3BEFA
:1019500022A8263FDD0BF4BE3F48263F4B48F4BE8D
:1019600046E8253F2284F4BE3588253F62BFF4BE99
:101970000C28253F0BFAF4BECDC7243F1D34F5BE1D
:101980007767243F976DF5BE0B07243F7BA6F5BE16
:1019900088A6233FC6DEF5BEF045233F7A16F6BE85
:1019A00042E5223F974DF6BE7E84223F1B84F6BE61
:1019B000A523223F07BAF6BEB7C2213F5BEFF6BEB2
:1019C000B461213F1724F7BE9C00213F3A58F7BE6F
:1019D000709F203FC58BF7BE303E203FB7BEF7BE9D
:1019E000DCDC1F3F10F1F7BE757B1F3FD122F8BE34
:1019F000F9191F3FF853F8BE6BB81E3F8684F8BE36
:101A0000CA561E3F7BB4F8BE16F51D3FD6E3F8BE9E
:101A100050931D3F9812F9BE77311D3FC040F9BE6B
:101A20008DCF1C3F4E6EF9BE906D1C3F439BF9BE9F
:101A3000820B1C3F9DC7F9BE63A91B3F5EF3F9BE35
:101A400033471B3F841EFABEF2E41A3F1049FABE28
:101A5000A0821A3F0273FABE3E201A3F599CFABE7A
:101A6000CCBD193F16C5FABE4A5B193F37EDFABE29
:101A7000B8F8183FBE14FBBE1796183FAB3BFBBE31
:101A80006733183FFC61FBBEA8D0173FB287FBBE8F
:101A9000DA6D173FCDACFBBEFE0A173F4DD1FBBE42
:101AA00013A8163F31F5FBBE1B45163F7A18FCBE46
:101AB00014E2153F283BFCBE017F153F3A5DFCBE9A
:101AC000E01B153FB07EFCBEB1B8143F8A9FFCBE40
:101AD0007755143FC9BFFCBE2FF2133F6CDFFCBE2D
:101AE000DC8E133F73FEFCBE7C2B133FDD1CFDBE62
:101AF00010C8123FAC3AFDBE9964123FDE57FDBEDE
:101B00001701123F7474FDBE899D113F6E90FDBE9A
:101B1000F139113FCCABFDBE4ED6103F8CC6FDBE99
:101B2000A072103FB1E0FDBEE90E103F38FAFDBED5
:101B300027AB0F3F2413FEBE5C470F3F722BFEBE48
:101B400087E30E3F2343FEBEAA7F0E3F385AFEBEF8
:101B5000C31B0E3FB070FEBED3B70D3F8B86FEBEDB
:101B6000DC530D3FC99BFEBEDBEF0C3F69B0FEBEF0
:101B7000D38B0C3F6DC4FEBEC4270C3FD4D7FEBE32
:101B8000ACC30B3F9DEAFEBE8E5F0B3FC9FCFEBEA1
:101B900068FB0A3F580EFFBE3C970A3F491FFFBE35
:101BA00009330A3F9D2FFFBED0CE093F543FFFBEF1
:101BB000906A093F6D4EFFBE4B06093FE95CFFBED0
:101BC00001A2083FC76AFFBEB13D083F0878FFBECB
:101BD0005CD9073FAB84FFBE0275073FB190FFBEE3
:101BE000A310073F189CFFBE40AC063FE3A6FFBE14
:101BF000D947063F0FB1FFBE6FE3053F9EBAFFBE58
